:020000040800F2
:10000000200E002021030008A9B7000899A70008C6
:10001000A5B70008910C000881D40008330300083C
:1000200000000000000000000000000001C0000807
:10003000F91F000800000000B9B90008E1C200087B
:100040003D0300083D0300083D0300083D03000890
:100050003D0300083D0300083D0300083D03000880
:100060003D0300083D0300083D0300083D03000870
:100070003D0300083D0300083D0300083D03000860
:100080003D0300083D0300083D0300083D03000850
:100090003D0300083D0300083D0300083D03000840
:1000A0003D0300083D0300083D0300080526000845
:1000B0003D0300083D0300083D0300083D03000820
:1000C0003D0300083D0300083D0300083D03000810
:1000D00000000000610500083D0300082120000821
:1000E0003D0300083D0300083D0300083D030008F0
:1000F0003D030008E5C400083D0300083D03000877
:10010000F5C400083D0300083D0300083D03000856
:100110003D0300083D0300083D0300083D030008BF
:100120003D0300083D0300083D0300083D030008AF
:100130003D0300083D0300083D0300083D0300089F
:100140003D0300083D0300083D0300083D0300088F
:100150003D0300083D0300083D0300083D0300087F
:1001600000000000000000003D0300083D030008FF
:100170003D0300083D0300083D0300083D0300085F
:100180003D0300083D0300083D0300080000000097
:10019000000000003D030008000000000000000017
:1001A00000000000000000003D0300083D030008BF
:1001B0003D0300083D0300083D0300083D0300081F
:1001C0003D0300083D03000800000000000000009F
:1001D0000000000000000000000000003D030008D7
:1001E0003D0300083D03000800000000000000007F
:1001F0003D030008312000083D0300080000000016
:10020000000000003D0300083D030008000000005E
:10021000000000003D030008000000003D0300084E
:100220003D03000800000000000000003D0300083E
:100230003D03000800000000000000000000000076
:100240000000000000000000000000003D03000866
:100250003D03000800F002F800F052F814A696E8FA
:10026000000CB244B344DA4501D100F049F8BAE8D1
:100270000F000FA696E83000A5EB040504EB060777
:10028000AAEB0704A7F101074FEA15154FEA34144A
:10029000A4F10104AC4201D300F032F813F0010FD5
:1002A00018BFFB1A43F0010300F001F8DBE7184721
:1002B00028DE000048DE0000103A24BF78C878C16C
:1002C000FAD8520724BF30C830C144BF04680C605C
:1002D000704700007047000000230024002500261E
:1002E000103A28BF78C1FBD8520728BF30C148BF99
:1002F0000B6070471FB50DF0CCFE1FBD10B510BDD3
:1003000000F0F3F81146FFF7F5FF0DF019FD00F0CE
:1003100011F903B4FFF7F2FF03BC00F019F9000074
:100320000A4880470A480047FEE7FEE7FEE7FEE787
:10033000FEE7FEE7FEE7FEE7FEE7FEE7FEE700007A
:1003400004480549054A064B70470000ADC3000844
:100350005502000820080020200E0020200A00205E
:10036000200A0020032A40F2308010F0030C00F035
:10037000158011F8013BBCF1020F624498BF11F8DF
:1003800001CB00F8013B38BF11F8013BA2F1040298
:1003900098BF00F801CB38BF00F8013B11F0030310
:1003A00000F07180083AC0F0088051F8043B083A28
:1003B00051F804CBA0E80810F5E7121D5CBF51F816
:1003C000043B40F8043BAFF30080D20724BF11F890
:1003D000013B11F801CB48BF11F8012B24BF00F8F5
:1003E000013B00F801CB48BF00F8012B70474FF0EC
:1003F00000020429C0F0128010F0030C00F01B80F2
:10040000CCF1040CBCF1020F18BF00F8012BA8BFFF
:1004100020F8022BA1EB0C0100F00DB85FEAC17CC3
:1004200024BF00F8012B00F8012B48BF00F8012B76
:1004300070474FF0000200B51346944696462039A7
:1004400022BFA0E80C50A0E80C50B1F12001BFF48D
:10045000F7AF090728BFA0E80C5048BF0CC05DF8F3
:1004600004EB890028BF40F8042B08BF704748BF41
:1004700020F8022B11F0804F18BF00F8012B7047B5
:1004800070477047704710B5203AC0F00B80B1E854
:100490001850A0E81850B1E81850A0E81850203AB9
:1004A000BFF4F5AF5FEA027C24BFB1E81850A0E8C2
:1004B000185044BF18C918C0BDE810405FEA827CDC
:1004C00024BF51F8043B40F8043B08BF7047D207F3
:1004D00028BF31F8023B48BF11F8012B28BF20F894
:1004E000023B48BF00F8012B7047754600F02CF81E
:1004F000AE4605006946534620F00700854618B011
:1005000020B5FFF71DFFBDE820404FF000064FF07B
:1005100000074FF000084FF0000BAC46ACE8C009F4
:10052000ACE8C009ACE8C009ACE8C00921F007019B
:100530008D46704710B50446AFF300802046BDE8F5
:100540001040FFF7E6BE00000048704700010020A1
:1005500001491820ABBEFEE72600020070470000EC
:1005600080B540F2A440C2F2000002F0AFFF80BDAF
:1005700080B58AB0089007910020059007980490F4
:10058000089800680AF0F2F90290089800680AF0EA
:10059000A3F90190029828B9FFE70198002800F01C
:1005A000A780FFE708980068C0688001002835D55B
:1005B000FFE70898407E012830D1FFE70898007EC9
:1005C00001282BD1FFE701200490FFE7089800687D
:1005D000006800F040010020B0EB911F19D1FFE747
:1005E00005980021CAF2403188420ED3FFE70899EE
:1005F000886D40F0100088650899C86D40F00100D2
:10060000C86501208DF8270076E005980130059037
:10061000DCE70898016840200860FFE7049802289A
:1006200013D0FFE7089800680AF0A0F960B1FFE76F
:10063000089800680AF082F928B9FFE7089800686E
:100640000AF0D4F9FFE7FFE7FFE70498012813D089
:10065000FFE7089800680AF03FF960B1FFE70898E3
:1006600000680AF06BF928B9FFE7089800680AF0FB
:1006700047F9FFE7FFE7FFE704980090022807D05B
:10068000FFE70098032806D1FFE70C20039005E060
:100690000820039002E004200390FFE705F0D6FF56
:1006A0000690FFE7089800688068039908421ED00A
:1006B000FFE705F0CBFF0699401A062816D3FFE79F
:1006C000089800688068039908420ED0FFE70899EF
:1006D000886D40F0100088650899C86D40F00100F1
:1006E000C86501208DF8270006E0FFE7DAE7FFE79D
:1006F00000208DF82700FFE79DF827000AB080BD95
:1007000080B582B001900198C06D00900098806D16
:1007100010F0500F4BD1FFE70099886D40F4007046
:1007200088650098006800680007002821D5FFE769
:10073000009800680AF022F9D0B1FFE7009800683D
:10074000C0688004002812D4FFE70099886D20F467
:10075000807088650098806DC004002806D4FFE78B
:100760000099886D40F001008865FFE7FFE7FFE72B
:1007700019E000980068C0688007002812D4FFE7DD
:100780000099886D20F4807088650098806DC004A1
:10079000002806D4FFE70099886D40F001008865C5
:1007A000FFE7FFE7FFE7009802F0E2FD10E00098A6
:1007B000806DC006002804D5FFE7009802F06CFEAB
:1007C00005E00098006D816E01988847FFE7FFE71C
:1007D00002B080BD80B582B001900198C06D0090DC
:1007E0000099886D40F0400088650099C86D40F020
:1007F0000400C865009802F04FFE02B080BD000002
:1008000080B582B001900198C06D0090009802F010
:100810003FFE02B080BD000080B584B00290029817
:1008200000680AF08BF80090029800680AF08EF8D1
:1008300000284BD0FFE70098002847D1FFE7029837
:100840000068806800F00D00012809D1FFE70298D8
:10085000006809F0C9FF02980168032008600DE0F4
:100860000299886D40F0100088650299C86D40F0CB
:100870000100C86501208DF80F002BE005F0E6FEB1
:100880000190FFE7029800688068C007E8B1FFE7C1
:1008900005F0DCFE0199401A032815D3FFE7029802
:1008A00000688068C00770B1FFE70299886D40F06A
:1008B000100088650299C86D40F00100C8650120EC
:1008C0008DF80F0006E0FFE7DCE7FFE700208DF87A
:1008D0000F00FFE79DF80F0004B080BD80B584B025
:1008E000029000200090029800680AF02FF800287B
:1008F00072D1FFE70298006880683F21C8F20001CA
:1009000008420ED0FFE70299886D40F0100088651C
:100910000299C86D40F00100C86501208DF80F00F4
:100920005EE00298006809F079FF48F20030C4F2F6
:10093000022009F0A9FF000200281AD5FFE740F2C3
:100940000400C2F200000068800942F66351C0F260
:100950003E51A0FB01108109022000EB41000090F4
:10096000FFE7009820B1FFE7009801380090F8E712
:10097000FFE705F06BFE0190FFE702980068006852
:10098000C00740BBFFE70298006809F0DFFF28B905
:10099000FFE70298006809F041FFFFE705F056FE07
:1009A0000199401A032815D3FFE7029800680068F0
:1009B000C00770B9FFE70299886D40F010008865A4
:1009C0000299C86D40F00100C86501208DF80F0044
:1009D00006E0FFE7D1E7FFE700208DF80F00FFE713
:1009E0009DF80F0004B080BD80B598B016901591A9
:1009F00001F064FE1490002000901390129011906A
:100A000010900F900E900D900C900B908DF82B0085
:100A1000FFE79DF82B0009286FDCFFE700208DF829
:100A20002A00FFE79DF82A0002285FDCFFE700208C
:100A300009909DF82A001499C97D884201D1FFE7E9
:100A40004EE014989DF82A1050F821000BF0C8F9D8
:100A50000990FFE7099808BBFFE714989DF82A1052
:100A600050F821000BF0BCF909900B9801300B9065
:100A70000B980B2811D3FFE714989DF82A1050F813
:100A80002110012081F82E009DF82A001499C875C4
:100A900000200B908DF85F00F5E0DBE7099B9DF8E7
:100AA0002A2010A951F82200184441F822009DF88C
:100AB0002B00092810D1FFE79DF82A2010A850F834
:100AC00022004CF6CD41CCF6CC41A0FB0110C00871
:100AD0000CA941F82200FFE70D2004F099FAFFE786
:100AE0009DF82A0001308DF82A009BE7FFE79DF86A
:100AF0002B0001308DF82B008BE70CA801F0F4FCE3
:100B0000002008900790069005908DF81300FFE7ED
:100B10009DF81300022829DCFFE79DF813001499C3
:100B2000C97D884201D1FFE71AE014989DF813109F
:100B300050F8210090ED040AB8EE400A05A800EB39
:100B4000810181ED000A9DF8131000EB810090ED0A
:100B5000001A9DED080A30EE010A8DED080AFFE744
:100B60009DF8130001308DF81300D1E700208DF8B7
:100B70001200FFE79DF8120002281FDCFFE79DF836
:100B800012001499C97D884201D1FFE710E09DF859
:100B9000121005A800EB810090ED000A9DED081AE7
:100BA00080EE010A149850F8210080ED090AFFE751
:100BB0009DF8120001308DF81200DBE70020039051
:100BC00016980BF04FFB002859D1FFE700208DF855
:100BD0000B00FFE79DF80B00022833DCFFE79DF8D0
:100BE0000B001699C97D884201D1FFE724E01698D1
:100BF0009DF80B1050F821000190019890ED050A26
:100C0000B5EE400AF1EE10FA08DAFFE7019890ED30
:100C1000050AB0EEC00A80ED050AFFE7019890EDE5
:100C2000050A90ED081A80EE011A9DED030A30EED8
:100C3000010A8DED030AFFE79DF80B0001308DF8E6
:100C40000B00C7E79DED030A9DED151AB8EE411A9A
:100C500080EE010A169880ED060A169800F1180237
:100C600046F20000C0F6010048F20001C0F60101A2
:100C700004230CF099FC01208DF85F0003E00020B4
:100C80008DF85F00FFE79DF85F0018B080BD0000A1
:100C9000FFE7FEE780B582B001F010FD019000F0A3
:100CA000E1FA019890ED040AB0EEC00ABCEEC00A69
:100CB0008DED000A01990869C86040F20000C2F297
:100CC000000001680098486040F2E850C2F200005D
:100CD0000CF080FF02B080BD81B040F2E010C2F2A3
:100CE00000000090009941F22030C0F20800086036
:100CF00000994FF080404860009900208860009A79
:100D00000821D160009908610099486100998861C3
:100D10000099C8610099086201B0704782B00190E3
:100D2000002000900198082803D8FFE70198009060
:100D300037E00198092803D1FFE70C2000902FE04D
:100D400001980A2803D1FFE71020009027E00198BE
:100D50000B2803D1FFE7142000901FE001980C2816
:100D600003D1FFE71820009017E001980D2803D168
:100D7000FFE7202000900FE001980E2803D1FFE745
:100D80003020009007E001980F2803D1FFE74020B2
:100D90000090FFE7FFE7FFE7FFE7FFE7FFE7FFE779
:100DA000FFE7009802B0704780B586B040F2E010CF
:100DB000C2F200002430059040F27820C2F2000018
:100DC000007808B9FFE712E101F078FC04900020F8
:100DD000ADF80E000290059800F00CF940F2782072
:100DE000C2F200000078E13801460091152800F2B7
:100DF000F0800099DFE811F05F00D500ED00ED0014
:100E0000ED00ED00ED00ED00ED00ED00ED00ED007A
:100E1000ED00ED00ED00ED0016001700ED001600EE
:100E2000ED003100D6E0049890ED040ABCEEC00A53
:100E30008DED020A05990298C1F8010040F2E850D0
:100E4000C2F200000CF0C6FE00F00CFA40F278216D
:100E5000C2F20001E1200870C9E04EF2CC00C0F6F9
:100E600000000279417990F807C0037A0CEB8C0CF2
:100E700003EB4C0303EB830C437A03EB4C03A3F526
:100E8000965303EB8303807A00EB4300A0F5E55013
:100E900002EB820201EB420242F2107100FB0120E0
:100EA000A0F5A470029005990120C87105990298D7
:100EB000C1F801008EE000208DF80700FFE79DF8E3
:100EC000070002282EDCFFE7002050B9FFE7049856
:100ED0009DF8071050F82100006A0CF099FB80B9CA
:100EE00019E004989DF8071050F82100006A0DF0F1
:100EF0005FF841EC100B51EC100B0CF071FB50B192
:100F0000FFE704989DF8071050F821100020C4F264
:100F1000B0200862FFE7FFE79DF8070001308DF879
:100F20000700CCE70498006890ED080ABDEEC00AFF
:100F300010EE100AADF80E000599BDF80E00A1F8EC
:100F400001000498406890ED080ABDEEC00A10EE5A
:100F5000100AADF80E000599BDF80E00A1F80300C7
:100F600005990120C87140F2E850C2F200000CF06F
:100F700031FE0498806890ED080ABDEEC00A10EEBC
:100F8000100AC0B2ADF80E000599BDF80E00A1F828
:100F9000010005990020A1F8030005990220C871FD
:100FA00018E00498006890ED070ABDEEC00A10EE44
:100FB000100AADF80E000599BDF80E00A1F8010069
:100FC00040F2B010C2F2000090F82F000599C871ED
:100FD00000E0FFE740F27821C2F200010020087033
:100FE00040F2E850C2F200000CF0F4FDFFE706B05A
:100FF00080BD000081B0009040F2E011C2F200011B
:1010000041F22230C0F20800086040F27820C2F2BB
:10101000000000780099087000990020C1F80100D4
:10102000009AFE215171009A91710099C87101B026
:101030007047000080B540F22C40C2F2000040F240
:101040007C31C2F20001B0222C230CF009FF40F2E7
:101050006830C2F2000040F2A821C2F20001C022B2
:1010600030230CF0FDFE80BD80B588B040F2B0109A
:10107000C2F200000790FFE7079940F26830C2F221
:10108000000001220CF024FF012840F0E280FFE77D
:10109000079828300690079890F82800E138014614
:1010A0000191162800F2D3800199DFE801F04D5438
:1010B0006E6F707172D0D0D0D0D0D0D0D0D00C1F85
:1010C000292A6C466D000AF0C3FB38B1FFE740F2F5
:1010D0007821C2F20001F120087006E040F2782188
:1010E000C2F2000100200870FFE7B1E006980CF0A2
:1010F0000FFA40F27821C2F20001F2200870A7E056
:10110000A6E001F0DBFA059005994FF07E5088616A
:10111000059800F1180246F20000C0F6010048F2FE
:101120000001C0F6010104230CF03EFA40F27821E0
:10113000C2F20001F42008708AE040F27821C2F285
:101140000001F620087083E040F27821C2F200012D
:10115000E12008707CE00698C1790AF09DFF40F21A
:101160007821C2F200010091E22008700698C0794F
:1011700040F61401C2F200010870FFF715FE009955
:10118000E120087064E063E062E061E060E05FE05D
:101190005EE001F093FA049000208DF80F00FFE765
:1011A0009DF80F00022845DCFFE704989DF80F101A
:1011B00050F821000290029890ED050A9FED271A41
:1011C00080EE010A80ED080A029890ED080A9FED72
:1011D000241AB4EE410AF1EE10FA0BDAFFE7029896
:1011E00090ED080AB7EE001AB4EE410AF1EE10FADB
:1011F00006DAFFE702990020C4F298200862FFE7B0
:101200009DF80F204AF20000C0F6010000EB4230CA
:101210004CF20001C0F6010101EB4231029A20328A
:1012200004230CF0C1F9FFE79DF80F0001308DF8A1
:101230000F00B5E740F27821C2F20001E720087004
:1012400040F24041C2F200010120087000E0FFE7D7
:1012500012E7FFF7A9FD08B080BD00BF00007A4487
:101260000000204381B040F2E011C2F2000101F120
:101270002400009041F22030C0F20800086000997C
:1012800000204860086001B07047000082B0019003
:101290000091019840F2E011C2F200010860009A4A
:1012A000106852688A62486202B0704780B584B0A4
:1012B000029001F003FA019000208DF80300FFE78F
:1012C0009DF80300022823DCFFE79DF80300019945
:1012D000C97D884201D1FFE714E001989DF8031011
:1012E00050F8210090F82E00C00750B1FFE7029996
:1012F0000220087002990820487001208DF80F0024
:101300000FE0FFE79DF8030001308DF80300D7E7F9
:101310000299012008700299002048708DF80F0092
:10132000FFE79DF80F0004B080BD000081B0009081
:1013300040F26412C2F20002116840F26010C2F280
:101340000000016000990969116090ED000A9FEDAD
:10135000131AB4EE410AF1EE10FA1DDDFFE740F278
:101360006010C2F2000090ED001A40F26410C2F268
:10137000000090ED000A31EE400A80EE010AB0EE66
:10138000C00A9FED071A20EE010ABDEEC00A10EE5A
:10139000100A00998882FFE701B07047BD37863593
:1013A0000000704283B040F21800C2F200000290C8
:1013B00000208DF80700FFE79DF8070002282FDCCA
:1013C000FFE79DF807000299C97D884201D1FFE738
:1013D00020E002989DF8071050F821000090009836
:1013E00090ED050AB5EE400AF1EE10FA08DAFFE7D3
:1013F000009890ED050AB0EEC00A80ED050AFFE7FF
:10140000009890ED050A90ED081A80EE010A80ED33
:10141000060AFFE79DF8070001308DF80700CBE7CB
:1014200003B0704783B002900191029B1A6958691A
:101430009969D3F81CC040EA0C00DB6B18431043D9
:1014400008430199086002980078800600281BD59F
:10145000FFE702994A6A8B6AC86A896B08430021D0
:10146000CFF6F07101EB035101F07C7108436FF08E
:101470000F0101EB021101F47C7140EA01020199B4
:10148000086810430860FFE702984168006B40F26B
:10149000FF2211400843019948600298C068B0F5E6
:1014A000806F0DD1FFE7029800788006002806D5EE
:1014B000FFE70199486840F480604860FFE70DE06D
:1014C0000298C068B0F5007F06D1FFE7019948682F
:1014D00040F40070486000E0FFE7FFE70298426BCD
:1014E00001994868104348600298406C70B1FFE76A
:1014F0000299086C4A6C896C104301F03F0140EA84
:1015000001420199486810434860FFE70298B0F82B
:10151000680001998860029800788007002859D5F2
:10152000FFE70298C16C0020CFF6FF7000EB01408E
:101530000021C0F2FF7100EA01020199886810439E
:1015400088600298006DB0F1FF3F06DCFFE701996B
:10155000886840F08050886005E00199886820F034
:1015600080508860FFE70298406DB0F1FF3F06DCD5
:10157000FFE70199886840F00050886005E0019914
:10158000886820F000508860FFE70298806DB0F115
:10159000FF3F06DCFFE70199886840F080408860E3
:1015A00005E00199886820F080408860FFE7029894
:1015B000C06DB0F1FF3F06DCFFE70199886840F09D
:1015C0000040886005E00199886820F0004088604C
:1015D000FFE7FFE70298006E0199C8600298406E2D
:1015E0000199086102980078800700286AD5FFE712
:1015F0000298006DB0F1FF3F0ADCFFE70298006D32
:101600004042009000986FF35F300199486106E016
:101610000298006D6FF35F3001994861FFE702980F
:10162000406DB0F1FF3F0FDCFFE70298406D404294
:10163000009000990020C1F6FF7000EA0142019974
:101640004869104348610BE00298416D0020C1F6E3
:10165000FF7000EA01420199486910434861FFE7C1
:101660000298806DB0F1FF3F09DCFFE70298806DC2
:1016700040420090BDF800000199886105E00298A1
:10168000B0F8580001998861FFE70298C06DB0F189
:10169000FF3F0BDCFFE70298C06D40420090009ACC
:1016A0000199886940EA0240886107E00298C26DAA
:1016B0000199886940EA02408861FFE701990020AA
:1016C000C86103E0019900204861FFE702980068C3
:1016D00001990862029800788007002806D5FFE784
:1016E0000199086A40F4E060086205E00199086A1F
:1016F00040F4A0600862FFE703B0704786B0049032
:1017000003910292049803990843029908434FF603
:10171000FF718843019000200090049818B1FFE702
:10172000049800900EE0039818B1FFE7039800902A
:1017300007E0029818B1FFE70298009000E0FFE789
:10174000FFE7FFE70198BDF80210B0EB014F03D0AF
:10175000FFE70120059002E000200590FFE70598D3
:1017600006B0704785B0039002910192002000906E
:10177000039828B1FFE7039890F82000009012E04A
:10178000029828B1FFE7029890F82000009009E045
:10179000019828B1FFE7019890F82000009000E040
:1017A000FFE7FFE7FFE7029858B1FFE700980299CB
:1017B00091F82010884203D0FFE70220049011E046
:1017C000FFE7019858B1FFE70098019991F82010C0
:1017D000884203D0FFE70320049003E0FFE70020E6
:1017E0000490FFE7049805B07047000089B00790A7
:1017F00006910592002004900390029005980068DD
:101800000190069828BBFFE7FFE7049807998968CD
:1018100088421DD2FFE7049838B9FFE707980068AF
:101820004FF6FC71084003900EE003980290039875
:101830000799498800EB0140019950F821004FF6C3
:10184000FC7108400390FFE7049801300490DCE746
:1018500034E0FFE7049907988268002091420090E5
:101860000AD2FFE7039806994FF6FC721140401A1E
:1018700018BF01200090FFE70098C007E8B1FFE71C
:10188000049838B9FFE7079800684FF6FC710840E4
:1018900003900EE00398029003980799498800EBA3
:1018A0000140019950F821004FF6FC710840039067
:1018B000FFE7049801300490CCE7FFE7069860B199
:1018C000FFE7039806994FF6FC721140884203D057
:1018D000FFE70120089029E0FFE704980599886058
:1018E00002980799498840EA0140059948600398A1
:1018F0000799498840EA01400599C8600598C06881
:10190000019950F8210070B1FFE70599C868019A64
:1019100050F822004FF6FC721040079A528840EAB5
:1019200002400861FFE700200890FFE7089809B02F
:101930007047000083B0029001910092029890F8E5
:1019400020008007002811D5FFE7019830B1FFE79C
:1019500001990020CFF601600860FFE7009820B1F0
:10196000FFE7009907200860FFE710E0019830B119
:10197000FFE701990020CFF601000860FFE700981B
:1019800020B1FFE7009905200860FFE7FFE703B0FB
:101990007047000083B002900191019890F82000F8
:1019A000029908600198006800F008000299086137
:1019B0000198006800F400200299486101980068CD
:1019C00000F00300029988610198006800F440303B
:1019D0000299C8610198006800F47C71012000EB55
:1019E0001111029A51620199096801F07C7100EBB2
:1019F0001150029988620198006800F04020029915
:101A0000C8620198006842F20001C0F60041084037
:101A1000029988630198006800F4C0500299C86375
:101A2000019840798007002807D5FFE702994FF415
:101A3000007048600299C86013E00198007902992B
:101A40004860019840794007002805D5FFE70299D2
:101A50004FF48060C86003E002990020C860FFE78F
:101A6000FFE70198406800F40060029988600198DF
:101A7000406800F44040029908640198406800F012
:101A800040700299486401984068C0F3054002998B
:101A900088640198406800F040400299086301980A
:101AA00000890299886602980078800700280CD582
:101AB000FFE7019880680021C0F2FF71014001201A
:101AC00000EB11400299C86403E002990120C86448
:101AD000FFE70198C06802990866019800690299B9
:101AE0004866029800788007002851D5FFE70198E2
:101AF00040696FF35F30ADF80200BDF80200029953
:101B0000086501984069C0F30C40ADF80200BDF8CB
:101B10000200029948650198C07AC006002805D5E0
:101B2000FFE70299086D40420865FFE70198C07A17
:101B30008006002805D5FFE70299486D40424865B8
:101B4000FFE701988069ADF80200BDF80200029934
:101B500088650198408BADF80200BDF8020002993B
:101B6000C8650198C07A4006002805D5FFE70299AC
:101B7000886D40428865FFE70198C07A000600281A
:101B800005D5FFE70299C86D4042C865FFE709E047
:101B900002990020086502994865029988650299B2
:101BA000C865FFE703B0704784B003900399886B62
:101BB000C96B084302900398016801205022C4F2C7
:101BC00002029142019000F06781FFE703980168EB
:101BD00001205022C5F202029142019000F05C8186
:101BE000FFE7039801680120D022C4F2020291426B
:101BF000019000F05181FFE7039801680120D02295
:101C0000C5F202029142019000F04681FFE703987D
:101C10000168012040F25012C4F202029142019088
:101C200000F03A81FFE703980168012040F250126A
:101C3000C5F202029142019000F02E81FFE7039865
:101C40000168012040F2D012C4F2020291420190D8
:101C500000F02281FFE703980168012040F2D012D2
:101C6000C5F202029142019000F01681FFE703984D
:101C70000168012040F25022C4F202029142019018
:101C800000F00A81FFE703980168012040F250222A
:101C9000C5F202029142019000F0FE80FFE7039836
:101CA0000168012040F2D022C4F202029142019068
:101CB00000F0F280FFE703980168012040F2D02293
:101CC000C5F202029142019000F0E680FFE703981E
:101CD0000168012040F25032C4F2020291420190A8
:101CE00000F0DA80FFE703980168012040F25032EB
:101CF000C5F202029142019000F0CE80FFE7039806
:101D00000168012040F2D032C4F2020291420190F7
:101D100000F0C280FFE703980168012040F2D03252
:101D2000C5F202029142019000F0B680FFE70398ED
:101D30000168012041F25002C4F202029142019076
:101D400000F0AA80FFE703980168012041F25002E9
:101D5000C5F202029142019000F09E80FFE70398D5
:101D60000168012041F2D002C4F2020291420190C6
:101D700000F09280FFE703980168012041F2D00251
:101D8000C5F202029142019000F08680FFE70398BD
:101D90000168012041F25012C4F202029142019006
:101DA0007AD0FFE703980168012041F25012C5F292
:101DB0000202914201906FD0FFE703980168012071
:101DC00041F2D012C4F202029142019064D0FFE7C6
:101DD00003980168012041F2D012C5F2020291423B
:101DE000019059D0FFE703980168012041F2502289
:101DF000C4F20202914201904ED0FFE703980168BD
:101E0000012041F25022C5F202029142019043D0DA
:101E1000FFE703980168012041F2D022C4F20202D8
:101E20009142019038D0FFE703980168012041F208
:101E3000D022C5F20202914201902DD0FFE7039813
:101E40000168012041F25032C4F202029142019035
:101E500022D0FFE703980168012041F25032C5F219
:101E600002029142019017D0FFE703980168012018
:101E700041F2D032C4F20202914201900CD0FFE74D
:101E8000039800684EF63041CAF6FD710844B0FA76
:101E900080F040090190FFE70198C00730B1FFE7EB
:101EA0000398016C029808430290FFE703980068CA
:101EB000406920F443000299084303990968486186
:101EC000039801680020086403990A68496C51640A
:101ED00003990968886403990968C86403990968C3
:101EE000086503980168012040F25032C4F20202F2
:101EF000914200904ED0FFE703980168012040F224
:101F00005032C5F202029142009043D0FFE703989D
:101F10000168012040F2D032C4F2020291420090E6
:101F200038D0FFE703980168012040F2D032C5F2B3
:101F30000202914200902DD0FFE703980168012032
:101F400041F25032C4F202029142009022D0FFE7E7
:101F500003980168012041F25032C5F20202914219
:101F6000009017D0FFE703980168012041F2D032BA
:101F7000C4F20202914200900CD0FFE7039800687F
:101F80004EF63041CAF6FD710844B0FA80F04009BF
:101F90000090FFE70098C00740B1FFE70398016891
:101FA00000204865039909688865FFE70398016880
:101FB0000020C86704B0704784B00390029101927A
:101FC000009303980068806C4FF6FF718843BDF85A
:101FD00000100844039909688864039801684FF465
:101FE000FE40C860029803990968C8640198039983
:101FF0000968086504B070477047000072B6FFE7D3
:10200000FEE7000080B582B00190019800780228B8
:1020100003D1FFE709F0CEFF00E0FFE702B080BD8B
:1020200080B540F28450C2F2000003F037FB80BD5F
:1020300080B540F2E850C2F2000003F02FFB80BDF3
:1020400083B002904AF60040C4F20000009002986B
:1020500000684AF60001C4F20001884205D1FFE79A
:10206000009800F554700090FFE70098029908640A
:1020700002980068D0F8800020F4F810029A1168E5
:10208000526B40EA0240C1F880000098703002991B
:10209000486402980068D0F8800020F07060029ACE
:1020A0001168926B40EA0260C1F880000098B0307D
:1020B00002998864009800F5C4700299C864009879
:1020C00000F5187002990865009800F51E700299D5
:1020D000486500980190FFE70198009901F5547157
:1020E000884208D2FFE7019900200860FFE70198C5
:1020F00004300190F0E703B07047000088B007900B
:102100000691059204930698406848B9FFE706983F
:10211000016882680069104340EA8140039009E049
:1021200006980168826800691043084340F08040C7
:102130000390FFE70698D0F820C0C1684269836920
:10214000C06940EA0C601843104340EA0140029025
:102150000798406D049901EBC10100EBC1000190AB
:102160000398019908600198043001900298019940
:10217000086001980430019000200090FFE700986B
:102180000699CA684EF2BC01C0F60001895C88421B
:102190000DD2FFE705980099405801990860019811
:1021A00004300190FFE7009804300090E7E708B0A2
:1021B0007047000083B00290019142F22800C4F2FF
:1021C000020000909DF80400C00788B1FFE7009965
:1021D00008684FF63F02C7F6FF7210400860029A87
:1021E0000099086840EA821040F0240008600FE07F
:1021F0000099086820F4F8600860029A009908685D
:1022000040EA82102422C8F2000210430860FFE76F
:1022100003B0704782B0019042F22800C4F202007D
:102220000090019800F00300032807D1FFE7009910
:10223000086848F22002104308601EE09DF8040080
:10224000C00758B1FFE7009800684FF6D771C7F68E
:10225000FF710840283000990860FFE79DF80400EE
:102260008007002808D5FFE7009908682822C8F2EF
:10227000000210430860FFE7FFE702B0704700006C
:1022800081B042F24000C4F2020000900099086858
:1022900040F00800086001B07047000083B0029071
:1022A000019142F22800C4F20200009000990868EF
:1022B00040F002000860019800880299088003B08D
:1022C0007047000089B00690059104208DF8130036
:1022D000069803900598029042F22800C4F202008A
:1022E00000900099086840F002000860EFF3108049
:1022F00007900798019072B6FFE70298006803996B
:1023000008600398043003900298043002909DF80E
:10231000130001388DF81300FFE79DF81300002823
:10232000EBD1FFE701980890089880F3108809B076
:10233000704700008AB00790069104208DF81700BE
:10234000079804900698039042F22800C4F2020015
:10235000019042F24000C4F2020000900199086826
:1023600040F00200086040F24800C2F200008068BD
:1023700000F004020099086810430860EFF3108031
:1023800008900898029072B6FFE7039800680499D5
:1023900008600498043004900398043003909DF87A
:1023A000170001388DF81700FFE79DF81700002887
:1023B000EBD1FFE702980990099880F310880AB0E2
:1023C0007047000083B00290019142F22800C4F2ED
:1023D000020000900099086840F00200086001982F
:1023E00000680299086003B07047000080B586B0AD
:1023F000049004F02BF9009042F22000C4F2020095
:102400000290FFE70298006810F00B0F15D0FFE76D
:102410000498013080B1FFE704F018F90099401AE0
:102420000499884203D8FFE7049820B9FFE7032006
:102430008DF817002EE0FFE7E4E742F23000C4F227
:10244000020001900298006800F47E000390039857
:1024500088B1FFE7039A40F24801C2F200014868E0
:1024600010434860039800F47E0001990860012041
:102470008DF817000EE002980068C003002805D50B
:10248000FFE701994FF480300860FFE700208DF8E6
:102490001700FFE79DF8170006B080BD80B582B039
:1024A00000208DF80700FFE79DF80700022816DCE2
:1024B000FFE79DF8070000EBC00140F20C20C2F2DC
:1024C000000000EB810005219FED060A09F02EF9BE
:1024D000FFE79DF8070001308DF80700E4E702B040
:1024E00080BD00BF0000000080B584B0039040F2C2
:1024F0001800C2F20000029000208DF80700FFE7EC
:102500009DF8070002285BDCFFE79DF807000299B1
:10251000C97D884201D1FFE74CE002989DF8071081
:1025200050F8210000909DF8072002EBC20140F214
:102530000C20C2F2000000EB8100039901EB820144
:1025400091ED000AB8EE400A05210BF025FC009839
:10255000BCEEC00A80ED040A0BF006FD20B1FFE7D7
:102560000099C8680861FFE70099C868096988424E
:102570000DD2FFE70098C2680169891A00EE101AAF
:10258000B8EE400AB1EE400A80ED050A11E000996C
:10259000C868096988420BD3FFE70098C1680269DF
:1025A000891A00EE101AB8EE400A80ED050AFFE71E
:1025B000FFE7FFE79DF8070001308DF807009FE770
:1025C00004B080BD80B582B000200190009040F240
:1025D0004140C2F20000D0F80900009040F267408C
:1025E000C2F20000D0F80900019041F203006946F0
:1025F000FEF74CFE40F2E850C2F200000BF0EAFA9F
:1026000002B080BD80B540F20C50C2F2000002F072
:1026100023FB80BD80B582B040F21800C2F20000FA
:10262000019000208DF80300FFE79DF803000228C9
:102630001ADCFFE79DF803000199C97D884201D1AA
:10264000FFE70BE040F26400C2F20000016801986D
:102650009DF8032050F822008847FFE79DF803000B
:1026600001308DF80300E0E700208DF80300FFE75C
:102670009DF8030002281CDCFFE79DF80300019988
:10268000C97D884201D1FFE70DE001989DF8031054
:1026900050F8210000F018F801999DF8032051F836
:1026A0002210C860FFE79DF8030001308DF8030099
:1026B000DEE701990120887502B080BD40F2180064
:1026C000C2F200007047000080B590B00E9000206C
:1026D00001900D9009900890079006900590049045
:1026E0008DF80F000C90FFE70C9804283EDCFFE704
:1026F00040F26400C2F2000001680E98884701466B
:102700000C9A04A840F822100C9950F821000A28CD
:1027100027D8FFE7FFF7D2FF02909DF80F000130A6
:102720008DF80F009DF80F000B2816DBFFE70298CD
:10273000C07D042809D0FFE70E99012081F82E0002
:1027400000208DF80F000F9062E00E9890F82F0097
:102750000299C87500200F905AE00C9801380C902F
:10276000FFE7FFE70C9801300C90BDE700200C90CC
:10277000FFE70C9803282CDCFFE70C9801300B9046
:10278000FFE70B9804281FDCFFE70C9804A951F819
:1027900020000B9A51F82210884210D9FFE70C98BC
:1027A00004A951F820000A900B9851F820000C9AC7
:1027B00041F822000A980B9A41F82200FFE7FFE750
:1027C0000B9801300B90DCE7FFE70C9801300C9080
:1027D000CFE701200C90FFE70C9803280CDCFFE703
:1027E0000C9904A850F82110099808440990FFE7B3
:1027F0000C9801300C90EFE709984AF6AB21CAF625
:10280000AA21A0FB011040080D900D980F90FFE742
:102810000F9810B080BD000084B002900020ADF889
:10282000060000900298B0F80100ADF80600BDF86F
:10283000060000EE100AB8EE400A8DED000ABDF861
:102840000600B0F57A7F09DDFFE79DED000AB2EEE4
:10285000041A80EE010A8DED000AFFE79DED000AE3
:102860009FED0E1AB4EE410AF1EE10FA0DDCFFE70F
:102870009DED000AB7EE001AB4EE410AF1EE10FA2F
:1028800003DBFFE70098039004E00020C4F2E0209F
:102890000390FFE79DED030A04B07047000020435A
:1028A00080B582B0FFF70AFF019000F019F80090A0
:1028B0000198807DC00720B9FFE7009900200870CB
:1028C000FFE700984078082804DBFFE70099022022
:1028D0000870FFE7019800990AF0D4FD02B080BDAE
:1028E00040F2E010C2F200002430704780B586B09C
:1028F000002001900590FFF7E1FE01460198049148
:102900008DF80F00FFE79DF80F00022844DCFFE779
:1029100004989DF80F1050F8210002909DF80F00C8
:102920000499C97D884201D1FFE72FE040F24400BD
:10293000C2F20000006803689DF80F104AF2000020
:10294000C0F6010000EB413005A9042298479DED37
:10295000050AB7EE001AB4EE410AF1EE10FA0ADBEE
:10296000FFE79DED050A9FED0D1AB4EE410AF1EE69
:1029700010FA06DDFFE702990020C4F2E0200862A9
:1029800003E0059802990862FFE7FFE79DF80F0052
:1029900001308DF80F00B6E706B080BD000020437F
:1029A00086B040F21800C2F20000059000200390AB
:1029B0000290019000908DF81300FFE79DF813003E
:1029C000022824DCFFE79DF813000599C97D8842A1
:1029D00001D1FFE715E005989DF8132050F822007B
:1029E0008169684640F822109DF8131000EB8100C1
:1029F00090ED001A9DED030A30EE010A8DED030AF9
:102A0000FFE79DF8130001308DF81300D6E79DED28
:102A1000030A059890ED061A80EE010A8DED030A6F
:102A20009DED030A06B0704780B586B0049003910F
:102A300000200190FFE7049890F85400012804D189
:102A4000FFE702208DF817005AE00499012081F871
:102A50005400FFE7FFE70498FDF7DEFE8DF80B005A
:102A60009DF80B00D8BBFFE70498806D40F0020092
:102A700020F488500499886504980068039908F048
:102A80007DF8FFE70498006807F048FFF0B1FFE722
:102A900001980130019001984FF60001C2F2C35134
:102AA000884212D3FFE70498806D40F0100020F0B8
:102AB000020004998865FFE70499002081F854001A
:102AC000FFE701208DF817001AE0DBE70498806D1E
:102AD00040F0010020F002000499886505E00499A7
:102AE000886D40F010008865FFE7FFE7049900203B
:102AF00081F85400FFE79DF80B008DF81700FFE701
:102B00009DF8170006B080BD81B0009001B07047FD
:102B100081B0009001B0704781B0009001B0704763
:102B200081B0009001B0704781B0009001B0704753
:102B300080B5C0B020901F9100208DF87B001B90C5
:102B40001F98C0680021C4F27F01884201D0FFE7CE
:102B500000E0FFE7FFE7209890F85400012804D137
:102B6000FFE702208DF88700FDE32099012081F81E
:102B70005400FFE7FFE72098006807F0F7FE002801
:102B800040F0DD83FFE71F980068012810D0FFE7C1
:102B90001F9800680221C0F2304188420DD1FFE742
:102BA0001F98C0680021C4F27F01884205D1FFE769
:102BB0002098006807F040FEFFE7209800681F9902
:102BC0000A68496807F0E6FE2098006807F0CEFE24
:102BD0001A902098006807F07FFE19901A98002834
:102BE00040F0B881FFE71998002840F0B381FFE773
:102BF0001F988068B0F1004F0ED1FFE72098006861
:102C00001F990968002207F0FFFE209800684FF026
:102C1000004107F0A5FF0CE0209800681F9A11689A
:102C2000926807F0F1FE20980068002107F098FFF5
:102C3000FFE71F98406920990968C96801F01801E9
:102C4000890888401D901F98006904281CD0FFE760
:102C5000209800681F990A6809691D9B07F026FFE4
:102C6000209800681F9A1169926907F051FF209817
:102C700000681F9A1169127F013AB2FA82F2520972
:102C8000520607F031FF64E120980068002107F048
:102C900013FE000348B9FFE720980068002107F001
:102CA0000BFEC0F38460189018E0209800680021A3
:102CB00007F002FE90FAA0F03E903E9820B9FFE7A0
:102CC00020208DF8FF0005E03E98B0FA80F08DF8E6
:102CD000FF00FFE79DF8FF001890FFE71898179096
:102CE0001F980068000330B9FFE71F980068C0F321
:102CF0008460169015E01F98006890FAA0F03C9050
:102D00003C9820B9FFE720208DF8F70005E03C98BB
:102D1000B0FA80F08DF8F700FFE79DF8F700169005
:102D2000FFE717981699884207D1FFE720980068B7
:102D30000022114607F000FFFFE7209800680121FC
:102D400007F0BAFD000348B9FFE7209800680121A9
:102D500007F0B2FDC0F38460159018E02098006879
:102D6000012107F0A9FD90FAA0F03A903A9820B915
:102D7000FFE720208DF8EF0005E03A98B0FA80F0E8
:102D80008DF8EF00FFE79DF8EF001590FFE715982D
:102D900014901F980068000330B9FFE71F9800687F
:102DA000C0F38460139015E01F98006890FAA0F0BB
:102DB0003890389820B9FFE720208DF8E70005E02B
:102DC0003898B0FA80F08DF8E700FFE79DF8E7004B
:102DD0001390FFE714981399884207D1FFE72098D2
:102DE00000680121002207F0A7FEFFE72098006895
:102DF000022107F061FD000348B9FFE72098006851
:102E0000022107F059FDC0F38460129018E0209869
:102E10000068022107F050FD90FAA0F03690369835
:102E200020B9FFE720208DF8DF0005E03698B0FAE2
:102E300080F08DF8DF00FFE79DF8DF001290FFE7DC
:102E4000129811901F980068000330B9FFE71F988F
:102E50000068C0F38460109015E01F98006890FA35
:102E6000A0F03490349820B9FFE720208DF8D700E7
:102E700005E03498B0FA80F08DF8D700FFE79DF8B0
:102E8000D7001090FFE711981099884207D1FFE70B
:102E9000209800680221002207F04EFEFFE72098EC
:102EA0000068032107F008FD000348B9FFE72098F8
:102EB0000068032107F000FDC0F384600F9018E064
:102EC00020980068032107F0F7FC90FAA0F03290F8
:102ED000329820B9FFE720208DF8CF0005E0329826
:102EE000B0FA80F08DF8CF00FFE79DF8CF000F908B
:102EF000FFE70F980E901F980068000330B9FFE7B6
:102F00001F980068C0F384600D9015E01F9800685A
:102F100090FAA0F03090309820B9FFE720208DF88B
:102F2000C70005E03098B0FA80F08DF8C700FFE7E1
:102F30009DF8C7000D90FFE70E980D99884207D1C4
:102F4000FFE7209800680321002207F0F5FDFFE766
:102F5000FFE7FFE72098006807F0F8FC002840F042
:102F60004481FFE7209800681F9A1168D26807F033
:102F700067FD1F98C0680021C4F27F01884240F0BD
:102F80003381FFE7209800680C901F9800680003C9
:102F900030B9FFE71F980068C0F384600B9015E01C
:102FA0001F98006890FAA0F02E902E9820B9FFE7A5
:102FB00020208DF8BF0005E02E98B0FA80F08DF843
:102FC000BF00FFE79DF8BF000B90FFE70B980130B3
:102FD00000F01F0009287DD8FFE71F980068000354
:102FE00030B9FFE71F980068C0F384600A9015E0CD
:102FF0001F98006890FAA0F02C902C9820B9FFE759
:1030000020208DF8B70005E02C98B0FA80F08DF8FC
:10301000B700FFE79DF8B7000A90FFE70A98013074
:1030200000F01F00800609901F980068000330B967
:10303000FFE71F980068C0F38460089015E01F98B0
:10304000006890FAA0F02A902A9820B9FFE7202083
:103050008DF8AF0005E02A98B0FA80F08DF8AF0047
:10306000FFE79DF8AF000890FFE709980899013144
:1030700001F01F0201219140084307901F9800684A
:10308000000330B9FFE71F980068C0F38460069022
:1030900015E01F98006890FAA0F02890289820B9B1
:1030A000FFE720208DF8A70005E02898B0FA80F00F
:1030B0008DF8A700FFE79DF8A7000690FFE70798A7
:1030C0000699013101F01F0101EB410140EA015075
:1030D000059082E01F980068000330B9FFE71F9851
:1030E0000068C0F38460049015E01F98006890FAAF
:1030F000A0F02690269820B9FFE720208DF89F00A9
:1031000005E02698B0FA80F08DF89F00FFE79DF863
:103110009F000490FFE70498013000F01F00800634
:1031200003901F980068000330B9FFE71F980068FC
:10313000C0F38460029015E01F98006890FAA0F038
:103140002490249820B9FFE720208DF8970005E00F
:103150002498B0FA80F08DF89700FFE79DF897006B
:103160000290FFE703980299013101F01F0201214B
:103170009140084301901F980068000330B9FFE7B1
:103180001F980068C0F38460009015E01F980068E5
:1031900090FAA0F02290229820B9FFE720208DF825
:1031A0008F0005E02298B0FA80F08DF88F00FFE7DD
:1031B0009DF88F000090FFE701990098013000F022
:1031C0001F0000EB40020020CFF6206000EB025011
:1031D000084340F000700590FFE70C9805991F9A8E
:1031E000926807F011FCFFE7FFE71F98408848F25C
:1031F0000801084200F0A280FFE748F20030C4F264
:10320000022007F041FB1C901F9800680021CCF2BF
:103210002131884233D1FFE79DF872000006002873
:103220002DD4FFE72098006848F20001C4F2022183
:10323000884223D1FFE71C9840F4000148F2003097
:10324000C4F2022007F024FC40F20400C2F20000A5
:103250000068800942F66351C0F23E51A0FB0110A4
:103260008109022000EB41001B90FFE71B9820B171
:10327000FFE71B9801381B90F8E7FFE75DE01F9818
:1032800000680021C4F22931884219D1FFE79DF876
:103290007300C007A0B9FFE72098006848F200114A
:1032A000C4F2022188420AD1FFE71C9840F08071E5
:1032B00048F20030C4F2022007F0EAFBFFE73BE0EF
:1032C0001F9800680021CCF2527188421AD1FFE7A2
:1032D0009DF872004006002814D4FFE7209800688B
:1032E00048F20001C4F2022188420AD1FFE71C988B
:1032F00040F4800148F20030C4F2022007F0C8FB1D
:10330000FFE718E01F9800680021C4F25A71884254
:103310000FD1FFE72098006848F20001C4F20221B3
:10332000884205D0FFE72098006807F091FAFFE790
:1033300000E0FFE7FFE7FFE7FFE7FFE708E020998E
:10334000886D40F02000886501208DF87B00FFE744
:10335000FFE72099002081F85400FFE79DF87B00EB
:103360008DF88700FFE79DF8870040B080BD000022
:1033700085B004900498006848F20001C4F202216C
:10338000884275D1FFE700208DF80F00FFE79DF818
:103390000F00042823DCFFE79DF80F1040F27A208D
:1033A000C2F2000030F8110000EE100AB8EEC00AB8
:1033B0009FED351A20EE010A9FED341A80EE010AC6
:1033C00040F29420C2F2000000EB810080ED000A80
:1033D000FFE79DF80F0001308DF80F00D7E740F2AE
:1033E0009420C2F2000090ED020A9FED222A80EEA6
:1033F000020A9FED211A20EE010A8DED020A90EDDE
:10340000000A80EE020A20EE010A8DED010A4168F1
:10341000009190ED030A9FED191A80EE010A9FEDCD
:10342000181A20EE010A40F28420C2F2000080ED5A
:10343000030A9DED000AB6EE002A30EE420A9FED27
:10344000111A20EE010A80ED020A9DED020A30EE0B
:10345000420AB1EE041A20EE010A80ED000A9DED49
:10346000010A30EE420A20EE010A80ED010AFFE770
:1034700005B070470080D4450010294600401C4626
:10348000005E97480000C8423333534000F07F4548
:1034900081B0009001B0704780B582B00190019872
:1034A00040F2A441C2F2000188420CD1FFE701982A
:1034B00000F0EAFD019840F27A21C2F200010522F3
:1034C00000F0A4FCFFE702B080BD000080B58EB024
:1034D0000D9000200C900D98006800680B900D98DE
:1034E000006840680A9048F20030C4F2022007F0F9
:1034F000DBF905909DF82C00800700281AD5FFE71E
:103500009DF828008007002814D5FFE70D98806DEE
:10351000C006002806D4FFE70D99886D40F40060CE
:103520008865FFE70D98FFF7EFFA0D980168022014
:103530000860FFE79DF82C004007002806D5FFE74C
:103540000A9800F0040004280ED0FFE79DF82C0034
:103550000007002840F19F80FFE79DF82800000742
:10356000002840F19880FFE70D98806DC006002884
:1035700006D4FFE70D99886D40F400708865FFE779
:103580000D98006807F0FAF900287CD0FFE70D9845
:10359000006848F20011C4F20221884206D1FFE718
:1035A00048F20000C4F20220049003E00D98006885
:1035B0000490FFE704980D99096888420BD0FFE753
:1035C000059840B1FFE70598052804D0FFE7059866
:1035D000092805D1FFE70D980068C068079018E03A
:1035E0000D98006848F20011C4F20221884206D109
:1035F000FFE748F20000C4F20220039003E00D98B8
:1036000000680390FFE7039806900698C06807904B
:10361000FFE7079800F40050B0F5005F32D0FFE7F5
:103620000D9800680068000700282AD5FFE70D986C
:10363000006807F09BF9C0B9FFE70D98016848687A
:1036400020F00C0048600D99886D20F4807088652A
:103650000D98806DC004002806D4FFE70D99886D91
:1036600040F001008865FFE70AE00D99886D40F0A1
:10367000100088650D99C86D40F00100C865FFE72E
:10368000FFE7FFE7FFE70D98FFF772FE0D9801686F
:103690000C200860FFE79DF82C008006002806D566
:1036A000FFE70A9800F0200020280ED0FFE79DF8E1
:1036B0002C004006002840F1B680FFE79DF8280066
:1036C0004006002840F1AF80FFE70D98806DC006EE
:1036D000002806D4FFE70D99886D40F400508865F6
:1036E000FFE70D98006807F0FFF809900D98006853
:1036F00007F044F908900D98006848F20011C4F2F0
:103700000221884206D1FFE748F20000C4F20220FD
:10371000029003E00D9800680290FFE702980D996F
:10372000096888420BD0FFE7059840B1FFE705988C
:10373000062804D0FFE70598072805D1FFE70D9874
:103740000068C068079018E00D98006848F2001102
:10375000C4F20221884206D1FFE748F20000C4F219
:103760000220019003E00D9800680190FFE70198A6
:1037700006900698C0680790FFE7099800284AD08D
:10378000FFE79DF81F00800700280AD5FFE708988B
:1037900000283FD0FFE79DF81D008006002839D49F
:1037A000FFE70D98006800684006002831D5FFE764
:1037B0009DF81E00800600282AD4FFE70D980068B7
:1037C00007F08AF8C0B9FFE70D980168486820F053
:1037D000600048600D99886D20F4805088650D98D0
:1037E000806DC005002806D4FFE70D99886D40F074
:1037F00001008865FFE70AE00D99886D40F0100030
:1038000088650D99C86D40F00100C865FFE7FFE7C6
:10381000FFE7FFE7FFE70D98FFF77AF90D980168DA
:1038200060200860FFE79DF82C000006002813D5F3
:10383000FFE79DF82800000600280DD5FFE70D9949
:10384000886D40F4803088650D9800F0FFF90D9880
:10385000016880200860FFE79DF82D00C00798B13F
:10386000FFE79DF82900C00770B1FFE70D99886D4B
:1038700040F4003088650D98FFF752F90D98016803
:103880004FF480700860FFE79DF82D008007002846
:1038900014D5FFE79DF82900800700280ED5FFE723
:1038A0000D99886D40F4802088650D98FFF73CF9EC
:1038B0000D9801684FF400700860FFE79DF82C0038
:1038C000C00600283ED5FFE79DF82800C006002866
:1038D00038D5FFE70D98806B18B9FFE701200C90F1
:1038E00019E0059860B1FFE748F20030C4F2022009
:1038F00006F0D2FF18B1FFE701200C90FFE709E0C6
:103900000D980068C068C00718B1FFE701200C904F
:10391000FFE7FFE7FFE70C9801280ED1FFE70D99BD
:10392000886D40F4806088650D99C86D40F0020094
:10393000C8650D98FFF7B0FDFFE70D9801681020EE
:103940000860FFE79DF82D004007002819D5FFE724
:103950009DF829004007002813D5FFE70D99886DD1
:1039600040F4804088650D99C86D40F00800C86536
:103970000D9801684FF4806008600D98FFF7CCF84F
:10398000FFE70EB080BD000080B588B00690002033
:103990008DF817000190069820B9FFE701208DF8F7
:1039A0001F004FE10698006940B1FFE7069890F8C4
:1039B0002000012801D1FFE7FFE7FFE70698806DAF
:1039C00050B9FFE7069800F045F906990020C86550
:1039D000069981F85400FFE70698006806F0A6FFF4
:1039E00028B1FFE70698006806F00CFFFFE706988D
:1039F000006806F0B3FFF0B9FFE70698006806F02C
:103A000033FF40F20400C2F200000068800942F671
:103A10006351C0F23E51A0FB01108109022000EB6E
:103A200041000190FFE7019820B1FFE701980138BC
:103A30000190F8E7FFE70698006806F08FFF70B97D
:103A4000FFE70699886D40F0100088650699C86DFB
:103A500040F00100C86501208DF81700FFE70698C7
:103A6000006806F083FF03900698806DC00600286A
:103A700000F1DA80FFE70398002840F0D580FFE7E7
:103A80000698806D40F0020020F4807006998865E9
:103A90000698006806F05AFFE0B9FFE748F2000018
:103AA000C4F2022006F052FF009048F20010C4F267
:103AB000022006F04BFF01460098084348B9FFE793
:103AC0000698416848F20030C4F2022006F0D2FFA6
:103AD000FFE7FFE706994A7E886B40EA42308A6832
:103AE000CB681843104391F8201040EA014004903D
:103AF000069890F8200001280BD1FFE70698416A4C
:103B00000020CFF6FE7000EB41410498084304907A
:103B1000FFE70698806A50B1FFE70699886AC96A8C
:103B200000F478700143049808430490FFE7069876
:103B30000068C06844F20701CFF6F07108400499AC
:103B4000084306990968C86006980068006920F073
:103B50004060069A1168126B10430861069800686D
:103B600006F0BAFE02900398E8BBFFE70298D0BBCC
:103B7000FFE70699087E91F83410800340EA41007F
:103B8000049006980068C06844F2020188430499D2
:103B9000084306990968C860069890F83C00012817
:103BA00019D1FFE706980068006940F2FD7120EA2C
:103BB0000102069B1968186CD3F844E0D3F848C09A
:103BC00040EA0E0040EA0C00DB6C1843104340F062
:103BD0000100086106E006980168086920F001000C
:103BE0000861FFE7FFE70698006901280CD1FFE7AD
:103BF00006980068006B20F00F00069A1168D269E1
:103C0000013A1043086306E006980168086B20F04B
:103C10000F000863FFE70698806D40F0010020F078
:103C200002000699886508E00699886D40F010004A
:103C3000886501208DF81700FFE79DF817008DF8C3
:103C40001F00FFE79DF81F0008B080BD81B0009005
:103C500001B0704780B5DAB0599000205890579065
:103C600056905590549039A86C21FCF7E2FB04A8BB
:103C7000D021FCF7DEFB5998006848F20001C4F23D
:103C80000221884240F0BF80FFE7002005904FF4FA
:103C9000001104912C9004A802F0DCFD18B1FFE79C
:103CA000FEF7ACF9FFE7FFE740F68C40C4F20240B4
:103CB000016841F480610160006800F48060039055
:103CC0000398FFE7FFE740F68C40C4F2024001682A
:103CD00041F001010160006800F0010002900298CB
:103CE000FFE7F0205490032055900020019056905B
:103CF0000020C4F2022054A902F004FB0198212103
:103D000039913A903B903C903D904FF400213E9188
:103D100001213F914FF4803240924291439144906F
:103D2000459046904A904790489040F28811C2F2E0
:103D3000000139A800F016FA18B1FFE7FEF75EF9A6
:103D4000FFE740F27010C2F2000040F28812C2F2A7
:103D50000002002100F010FC18B1FFE7FEF74EF959
:103D6000FFE740F27010C2F2000000F0A5FD18B1AC
:103D7000FFE7FEF743F9FFE740F20C50C2F2000004
:103D80005021C4F2020101604FF40001816300215F
:103D9000C163016441648121816400F02BFA18B190
:103DA000FFE7FEF72BF9FFE740F20C50C2F20000EC
:103DB00040F27011C2F2000100F0ACFC18B1FFE754
:103DC000FEF71CF9FFE7FFE7599840F20C51C2F2E9
:103DD000000101655998C865FFE740F20C50C2F236
:103DE0000000102100F0FEFE18B1FFE7FEF706F913
:103DF000FFE7252000900022114602F00BFD0098FD
:103E000002F0FEFCFFE75AB080BD000080B5A4B010
:103E100022902191209248F20030C4F2022006F054
:103E200043FD1E902298006806F0A0FD002840F097
:103E30001E81FFE7FFE7229890F85400012804D183
:103E4000FFE702208DF88F001AE12299012081F806
:103E50005400FFE7FFE71E9848B1FFE71E980528CA
:103E600005D0FFE71E98092840F0F680FFE722986A
:103E7000FCF734FD8DF87F009DF87F00002840F0AE
:103E8000E380FFE72298806D40F4807040F6016186
:103E90008843229988652298006848F20011C4F28C
:103EA0000221884206D1FFE748F20000C4F2022056
:103EB000019003E0229800680190FFE701982299A1
:103EC0000968884203D0FFE71E9830B9FFE72299BE
:103ED000886D20F480108865FFE72298806DC0040B
:103EE000002806D5FFE72299C86D20F00600C865B6
:103EF00003E022990020C865FFE72298016D40F297
:103F00000170C0F6000008662298016D40F60100BD
:103F1000C0F6000048662298016D40F2D570C0F6E8
:103F200000008866229801681C200860FFE722993B
:103F3000002081F85400FFE722980168486840F0AB
:103F40001000486022980168C86840F00100C8600D
:103F50002298006D90F85000000600284CD5FFE72D
:103F60002298006D406F002841D0FFE72298006D35
:103F7000406F0068D8B3FFE72298006D406F01687A
:103F800002A800F01DF920B1FFE701208DF88F0095
:103F900076E00898022804D1FFE7209880001D9061
:103FA0000BE00898012804D1FFE7209840001D90FD
:103FB00002E020981D90FFE7FFE71D982299096D08
:103FC000496F0968886022990868096D4030496F17
:103FD0000968C86021982299096D496F09680861CC
:103FE0002298006D00F0CEFC8DF87F0003E00120E8
:103FF0008DF88F0044E022E02298006D806902284D
:1040000004D1FFE7209880001D900DE02298006DFC
:104010008069012804D1FFE7209840001D9002E04C
:1040200020981D90FFE7FFE722980168006D40315E
:10403000219A1D9B00F07AFF8DF87F00FFE7229800
:10404000006806F0C5FC06E0FFE72299002081F831
:104050005400FFE7FFE709E001208DF87F00FFE74C
:104060002299002081F85400FFE7FFE703E00220D7
:104070008DF87F00FFE79DF87F008DF88F00FFE748
:104080009DF88F0024B080BD80B584B00290FFE71A
:10409000029890F85400012804D1FFE702208DF81F
:1040A0000F005BE00299012081F85400FFE7FFE771
:1040B00002980321FCF75CFA8DF807009DF80700D1
:1040C000002840D1FFE702980168C86820F001008D
:1040D000C8600298006D90F85400022811D1FFE7E3
:1040E0000298006D00F0F2FC8DF807009DF80700C3
:1040F00030B1FFE70299886D40F040008865FFE726
:10410000FFE702980168486820F0100048609DF8B9
:10411000070030B9FFE70298FCF77EFB8DF8070037
:1041200003E00298FCF778FBFFE79DF8070048B929
:10413000FFE70298806D40F0010020F4885002995A
:104140008865FFE7FFE7FFE70299002081F8540048
:10415000FFE79DF807008DF80F00FFE79DF80F00BF
:1041600004B080BD80B584B002900191029818B16E
:10417000FFE7019820B9FFE701208DF80F001AE052
:10418000029800788006002801D5FFE7FFE7029833
:10419000406C08B1FFE7FFE702980078800700282D
:1041A00001D5FFE7FFE702980199FDF73BF90020F1
:1041B0008DF80F00FFE79DF80F0004B080BD0000F0
:1041C00080B584B002900191029818B1FFE7019880
:1041D00020B9FFE701208DF80F0007E00298019950
:1041E000FDF7D8FB00208DF80F00FFE79DF80F00CA
:1041F00004B080BD80B584B0029002F027FA01902F
:10420000029820B9FFE701208DF80F00AFE1029876
:10421000016801205022C4F202029142009000F095
:104220006781FFE70298016801205022C5F202026F
:104230009142009000F05C81FFE702980168012044
:10424000D022C4F202029142009000F05181FFE7B7
:10425000029801680120D022C5F20202914200902A
:1042600000F04681FFE702980168012040F25012F9
:10427000C4F202029142009000F03A81FFE70298F6
:104280000168012040F25012C5F2020291420090F2
:1042900000F02E81FFE702980168012040F2D01261
:1042A000C4F202029142009000F02281FFE70298DE
:1042B0000168012040F2D012C5F202029142009042
:1042C00000F01681FFE702980168012040F25022B9
:1042D000C4F202029142009000F00A81FFE70298C6
:1042E0000168012040F25022C5F202029142009082
:1042F00000F0FE80FFE702980168012040F2D02222
:10430000C4F202029142009000F0F280FFE70298AE
:104310000168012040F2D022C5F2020291420090D1
:1043200000F0E680FFE702980168012040F2503279
:10433000C4F202029142009000F0DA80FFE7029896
:104340000168012040F25032C5F202029142009011
:1043500000F0CE80FFE702980168012040F2D032E1
:10436000C4F202029142009000F0C280FFE702987E
:104370000168012040F2D032C5F202029142009061
:1043800000F0B680FFE702980168012041F2500278
:10439000C4F202029142009000F0AA80FFE7029866
:1043A0000168012041F25002C5F2020291420090E0
:1043B00000F09E80FFE702980168012041F2D002E0
:1043C000C4F202029142009000F09280FFE702984E
:1043D0000168012041F2D002C5F202029142009030
:1043E00000F08680FFE702980168012041F2501238
:1043F000C4F20202914200907AD0FFE7029801686D
:10440000012041F25012C5F20202914200906FD099
:10441000FFE702980168012041F2D012C4F20202C3
:104420009142009064D0FFE702980168012041F2B8
:10443000D012C5F202029142009059D0FFE70298D3
:104440000168012041F25022C4F202029142009020
:104450004ED0FFE702980168012041F25022C5F2D8
:1044600002029142009043D0FFE7029801680120C8
:1044700041F2D022C4F202029142009038D0FFE70C
:1044800002980168012041F2D022C5F20202914255
:1044900000902DD0FFE702980168012041F25032D0
:1044A000C4F202029142009022D0FFE70298016814
:1044B000012041F25032C5F202029142009017D021
:1044C000FFE702980168012041F2D032C4F20202F3
:1044D000914200900CD0FFE7029800684EF6304100
:1044E000CAF6FD710844B0FA80F040090090FFE779
:1044F0000098C00708B1FFE7FFE7FFE70299002037
:1045000081F84C00FFE70299022081F854000298DC
:104510000168486940F006004861FFE702980068BA
:104520004069C00798B1FFE702F090F80199401A7E
:1045300006280BD3FFE70299102088650299032013
:1045400081F8540001208DF80F0010E0E6E7029892
:10455000FDF72AFB0299886C08650299002088659E
:10456000029A012182F854108DF80F00FFE79DF8A0
:104570000F0004B080BD000080B58CB00A90099196
:1045800008920A9818B1FFE7089820B9FFE70120C0
:104590008DF82F00B9E00A984069012807D1FFE79C
:1045A0000A990420086101208DF82F00ADE00A98D7
:1045B00000680999089AFDF7A1F838B1FFE70A9950
:1045C0000520086101208DF82F009EE00A98006800
:1045D0000999089AFDF7C6F838B1FFE70A9904204F
:1045E000086101208DF82F008FE00A9902200873DE
:1045F0000A9900200861089807A906AAFDF79AF908
:104600000A980068E0B9FFE7099838B9FFE7089809
:104610000A9908600A990120886010E009980A99AF
:10462000086008984FF6FC710840079908430999FB
:10463000069A41F822000A9902208860FFE75BE0B1
:10464000099878B9FFE70A9800684FF6FC710840AE
:10465000079908430899069A41F8220008980A9990
:10466000086044E0069801900A98099901AAFDF7AC
:10467000BDF8A0BBFFE703980A99896888421BD15F
:10468000FFE70A98406860B1FFE70A9840684FF674
:10469000FC710840079908430899069A41F82200DE
:1046A000FFE708984FF6FC710840079908430999FD
:1046B000069A41F8220011E00998069A50F8220063
:1046C000089941F8220008984FF6FC7108400799B4
:1046D00008430999069A41F82200FFE706E00A9983
:1046E0000620086101208DF82F000EE0FFE70A99EF
:1046F000886801308860FFE70A99002008610A9AFB
:10470000012111738DF82F00FFE79DF82F000CB0E9
:1047100080BD000085B003900291039818B1FFE7B7
:10472000029820B9FFE701208DF81300BFE003983D
:10473000006D20B9FFE701208DF81300B7E0039862
:1047400090F854008DF80700039890F85400022860
:1047500005D0FFE79DF8070005280DD1FFE7039975
:1047600040208865FFE70399002081F84C00FFE7AF
:1047700001208DF813009AE00298007B022806D1F0
:10478000FFE70299012008618DF813008FE003987C
:104790000168012040F25032C4F2020291420090BE
:1047A0004ED0FFE703980168012040F25032C5F275
:1047B00002029142009043D0FFE703980168012074
:1047C00040F2D032C4F202029142009038D0FFE7AA
:1047D00003980168012040F2D032C5F202029142F2
:1047E00000902DD0FFE703980168012041F250327C
:1047F000C4F202029142009022D0FFE703980168C0
:10480000012041F25032C5F202029142009017D0CD
:10481000FFE703980168012041F2D032C4F202029E
:10482000914200900CD0FFE7039800684EF63041AB
:10483000CAF6FD710844B0FA80F040090090FFE725
:104840000098C00778B9FFE70298006890F8200048
:104850008007002807D5FFE702990320086101209F
:104860008DF8130023E00398006D81280CD1FFE739
:104870000298406838B9FFE70299042008610120D6
:104880008DF8130013E00BE00298406838B1FFE7A1
:1048900002990420086101208DF8130007E0FFE76A
:1048A00002980399486700208DF81300FFE79DF8F0
:1048B000130005B07047000080B58AB008900898D2
:1048C00020B9FFE701208DF8270056E0089800681E
:1048D00038B9FFE708990220086101208DF8270008
:1048E0004BE00898406888B1FFE708980168406885
:1048F000884204D1FFE700208DF827003DE00899A9
:104900000420086101208DF8270036E008984069EE
:10491000012807D1FFE708990420086101208DF8DC
:1049200027002AE0089902200873089900200090C7
:1049300008610898006807A906AAFCF7FBFF009920
:1049400006980190089801AAFCF750FF0098089972
:1049500009684FF6FC721140079A1143049A069BAE
:1049600042F82310089A1168516008990861089A62
:10497000012111738DF82700FFE79DF827000AB089
:1049800080BD000080B586B00490049820B1FFE798
:104990000498406F20B9FFE701208DF8170090E0E0
:1049A0000498006D20B9FFE701208DF8170088E01A
:1049B000049890F854008DF80F000498006840693E
:1049C00000F4803002909DF80F00012809D0FFE725
:1049D0009DF80F00022863D1FFE7029800285FD0FE
:1049E000FFE7049890F85400012852D1FFE7FFE751
:1049F000049890F84C00012804D1FFE702208DF8BC
:104A000017005EE00499012081F84C00FFE7FFE702
:104A10000499022081F854000499496F087304999D
:104A2000002088650499496F086104980168486905
:104A300040F4BA4048610498406E38B1FFE70498EA
:104A40000168486940F400704861FFE70498006F0E
:104A500038B1FFE704980168486940F400504861A4
:104A6000FFE70498406F006801A90022FCF762FF8D
:104A700004980168406F4088000408600498016849
:104A8000406F00684FF6FC721040019A1043C867EF
:104A9000FFE704980168486940F0010048610CE0B4
:104AA000049940208865FFE70499002081F84C00B4
:104AB000FFE701208DF8170003E000208DF81700B4
:104AC000FFE79DF8170006B080BD000080B584B0F8
:104AD000029001F0BBFD0190029820B9FFE7012090
:104AE0008DF80F0079E0029890F8540002280DD05C
:104AF000FFE7029920208865FFE70299002081F8EE
:104B00004C00FFE701208DF80F0066E00298016875
:104B1000486940F0040048610299052081F854007A
:104B2000FFE70298006800698004002827D4FFE7A7
:104B300001F08CFD0199401A06281FD3FFE7029966
:104B4000886D40F0100088650299032081F85400B8
:104B5000029890F850000006002805D5FFE702985B
:104B6000416F01200873FFE7FFE70299002081F8F9
:104B70004C00FFE701208DF80F002EE0D1E70298EE
:104B80000168486940F0020048610299042081F8F8
:104B90005400029801684FF4FE40C8600299012059
:104BA00081F85400029890F850000006002809D5BA
:104BB000FFE70298416F0120087302980168002006
:104BC0008864FFE7FFE70299002081F84C00FFE7C7
:104BD000FFE700208DF80F00FFE79DF80F0004B0FD
:104BE00080BD000085B003900291039820B9FFE7D3
:104BF00001208DF813002AE00398006840F6FF7149
:104C000088430190039800685038C0F3C411012014
:104C1000884000909DF80800C006002813D5FFE7E3
:104C2000029800F01100112806D1FFE7009A0199BF
:104C300048681043486005E0009A0199486890432D
:104C40004860FFE7FFE700208DF81300FFE79DF8BD
:104C5000130005B07047000080B584B0039003983E
:104C6000006840F6FF71884302900398006850384E
:104C7000C0F3C4110120884001900298C0680199D6
:104C800008400090009808B9FFE74DE103980068DC
:104C900000694005002813D5FFE7039800684069C4
:104CA000400500280BD5FFE7039801684FF48060AA
:104CB000C8600399886D40F001008865FFE7FFE751
:104CC0000398006800690005002813D5FFE70398E2
:104CD00000684069000500280BD5FFE703980168CC
:104CE0004FF40060C8600399886D40F00200886549
:104CF000FFE7FFE7039800680069C004002813D5A8
:104D0000FFE7039800684069C00400280BD5FFE75F
:104D1000039801684FF48050C8600399886D40F093
:104D200004008865FFE7FFE7039800680069400416
:104D3000002813D5FFE70398006840694004002865
:104D40000BD5FFE7039801684FF48040C8600399D2
:104D5000886D40F008008865FFE7FFE7039800686A
:104D600000698005002816D5FFE7039800684069B0
:104D7000800500280ED5FFE7039801684FF4007006
:104D8000C8600398406E20B1FFE70398416E8847E2
:104D9000FFE7FFE7FFE70398006800698004002849
:104DA00050D5FFE70398006840698004002848D583
:104DB000FFE7039801684FF40050C860039890F82B
:104DC000540004282FD1FFE703980168486920F4B4
:104DD0000050486103980168486940F0020048614A
:104DE0000399012081F85400039890F850000006C0
:104DF000002809D5FFE70398416F01200873039845
:104E0000016800208864FFE7FFE70399002081F82C
:104E10004C00FFE70398C06E20B1FFE70398C16E16
:104E20008847FFE780E00399052081F85400039844
:104E3000006F20B1FFE70398016F8847FFE7FFE7A6
:104E4000FFE7FFE7039800680069C005002842D526
:104E5000FFE7039800684069C00500283AD5FFE7DE
:104E6000039890F850000006002814D5FFE7039837
:104E70000068C06F70B9FFE703980068806C40B9A4
:104E8000FFE70399012081F854000399496F0873E3
:104E9000FFE7FFE70AE003980068806C28B9FFE7A6
:104EA0000399012081F85400FFE7FFE703980168A8
:104EB0004FF44070C860FFE70399002081F84C0070
:104EC000FFE70398006E20B1FFE70398016E884763
:104ED000FFE7FFE7FFE70398806D28B3FFE703983C
:104EE0000168486940F0020048610399012081F897
:104EF0005400039890F850000006002805D5FFE7FD
:104F00000398416F01200873FFE7FFE70399002032
:104F100081F84C00FFE70398806E20B1FFE703980B
:104F2000816E8847FFE7FFE704B080BD80B586B09B
:104F30000490039102920193049820B9FFE70120A5
:104F40008DF817005FE00498006D20B1FFE70120A5
:104F50008DF8170057E0FFE7049890F84C000128FF
:104F600004D1FFE702208DF817004CE004990120DE
:104F700081F84C00FFE7FFE7049890F854000128FF
:104F800030D1FFE70499022081F8540004990020F1
:104F9000886504980399029A019BFDF70DF804981F
:104FA0000168486940F4BA4048610498406E38B1DD
:104FB000FFE704980168486940F400704861FFE722
:104FC0000498006F38B1FFE704980168486940F41D
:104FD00000504861FFE704980168486940F001000B
:104FE00048610CE0049940208865FFE7049900209F
:104FF00081F84C00FFE701208DF8170003E0002046
:105000008DF81700FFE79DF8170006B080BD00007F
:1050100080B584B0039001F019FB029003980190D1
:105020000198013048B1FFE740F2F800C2F20000F9
:105030000178019808440190FFE7FFE701F006FBC3
:105040000299401A0199884201D2FFE7F6E704B0BD
:1050500080BD000086B0049003910292049890F8FD
:105060005C008DF80700BDF80C0010F4C07F01D083
:10507000FFE7FFE79DF80700012806D0FFE79DF84E
:105080000700022840F0DE80FFE704980068806D8A
:1050900000909DF80C00400730B1FFE79DF800003C
:1050A000C007002847D0FFE79DF80C0010F0380F2C
:1050B00006D0FFE79DF80000800700283BD5FFE7FA
:1050C000BDF80C0010F4E07F06D0FFE79DF800006B
:1050D000400700282FD5FFE79DF80D0010F01E0FA8
:1050E00006D0FFE79DF800000007002823D5FFE762
:1050F0009DF80D0010F0E00F06D0FFE79DF80000CE
:10510000C006002817D5FFE79DF80E00800730B1D4
:10511000FFE79DF80000800600280CD5FFE79DF80A
:105120000E0010F0FC0F0DD0FFE79DF800004006C8
:10513000002807D4FFE704980168C86D40F001001B
:10514000C865FFE79DF80C00400730B1FFE79DF808
:105150000000C007002847D1FFE79DF80C0010F0C1
:10516000380F06D0FFE79DF80000800700283BD4E9
:10517000FFE7BDF80C0010F4E07F06D0FFE79DF8D4
:105180000000400700282FD4FFE79DF80D0010F025
:105190001E0F06D0FFE79DF800000007002823D46B
:1051A000FFE79DF80D0010F0E00F06D0FFE79DF837
:1051B0000000C006002817D4FFE79DF80E00800706
:1051C00030B1FFE79DF80000800600280CD4FFE70F
:1051D0009DF80E0010F0FC0F0DD0FFE79DF80000C9
:1051E0004006002807D5FFE704980168C86D40F025
:1051F0000200C865FFE79DF80C000006002809D5ED
:10520000FFE7029A04980168D1F8DC001043C1F866
:10521000DC00FFE79DF80D00C00748B1FFE7029AE8
:1052200004980168D1F8E0001043C1F8E000FFE7FE
:10523000039A04980168486D1043486500208DF872
:10524000170008E00499086E40F00200086601208B
:105250008DF81700FFE79DF8170006B070470000B3
:1052600080B586B00490039102920398406808B913
:10527000FFE700E0FFE7049890F85C0002282FD1D8
:10528000FFE704980068D0F8C4008002002809D520
:10529000FFE70499086E40F40070086601208DF85D
:1052A000170026E004980068D0F8C400C0F301405D
:1052B000019004980399029A019BFCF71FFF019942
:1052C000012000FA01F1049A1268C2F8CC10019989
:1052D000884004998865FFE700208DF8170008E0F2
:1052E0000499086E40F00800086601208DF8170048
:1052F000FFE79DF8170006B080BD000087B005905D
:105300000491059890F85C008DF803009DF8030067
:10531000012805D0FFE79DF8030002283CD1FFE7F4
:1053200004980068B8B9FFE704998868CB680A69EF
:105330004969800740EAC36040EA0240084303909D
:105340000598006C0499496800EB8100019003986E
:10535000019908601CE00498C168006940EA417046
:10536000039004988168406940EA81700290059832
:10537000406C0499496800EBC100019003980199C1
:105380000860019804300190029801990860FFE7D5
:1053900000208DF81B0008E00599086E40F002001F
:1053A000086601208DF81B00FFE79DF81B0007B081
:1053B0007047000085B0DDF814C00390029101929F
:1053C0000093039890F85C00012819D1FFE7039837
:1053D0000068D0F8800020F03F0002990901019A8E
:1053E00041EA8201009A41EA4201059A11430843C9
:1053F00003990968C1F8800000208DF8130008E0C7
:105400000399086E40F00400086601208DF813002F
:10541000FFE79DF8130005B07047000081B00090D1
:1054200001B0704782B00190009102B07047000057
:1054300083B0029001910198402808D1FFE70298BB
:105440000068D0F8900000F00F00009007E002988C
:105450000068D0F8980000F00F000090FFE7009877
:1054600003B070478AB00890079106920593002018
:105470000190089890F85C008DF803009DF80300F7
:10548000022840F0FA80FFE7079840283ED1FFE766
:1054900008980068D0F89000000748B9FFE708991D
:1054A000086E40F48070086601208DF82700EDE05A
:1054B00008980068D0F8900000F080710120B0EBEF
:1054C000116F0FD1FFE708980068D0F8800000F452
:1054D00000710120B0EB512F03D1FFE701200190B3
:1054E000FFE7FFE708980068D0F8900000F44071EB
:1054F000019800EB112001900898806C019901EB54
:10550000C10100EBC1000490FFE73DE0089800688E
:10551000D0F89800000748B9FFE70899086E40F4F2
:105520008070086601208DF82700AFE008980068B9
:10553000D0F8980000F080710120B0EB116F0FD10E
:10554000FFE708980068D0F8800000F4807101201F
:10555000B0EB112F03D1FFE701200190FFE7FFE738
:1055600008980068D0F8980000F44071019800EBAA
:10557000112001900898C06C019901EBC10100EB6A
:10558000C1000490FFE7FFE70498006800F0804046
:10559000069948600698406838B9FFE704980068A3
:1055A000C0F38A400699086006E00498006820F07D
:1055B000604006990860FFE70498006800F000501A
:1055C000069988600498006800F000400699086118
:1055D000049804300490049800880699C8610498DF
:1055E0000068C0F303400699C8600498006800F49E
:1055F0008010069948610498006800F4001006992C
:10560000886104980068C0F30660069908620498EF
:105610000068C00F0699486204980430049004980A
:10562000039000200290FFE702980699CA684EF2A4
:10563000BC01C0F60001895C88420AD2FFE70398EA
:10564000029A805C05998854FFE702980130029025
:10565000EAE70798402806D1FFE70198089909680A
:10566000C1F8940005E0019808990968C1F89C0008
:10567000FFE700208DF8270008E00899086E40F049
:105680000800086601208DF82700FFE79DF8270035
:105690000AB0704781B0009001B0704780B58AB001
:1056A000099009980068006D00F4E050089009988E
:1056B0000068416D08980840089009980068006DDE
:1056C00000F00700079009980068416D07980840AE
:1056D000079009980068006D00F03800069009985E
:1056E0000068416D06980840069009980068006DB2
:1056F00000F47100059009980068416D0598084014
:10570000059009980068006D00F4602004900998E5
:105710000068416D04980840049009980068406D45
:10572000019009980068006D00909DF8000000F05D
:1057300040010020B0EB911F12D0FFE79DF804005C
:1057400000F040010020B0EB911F08D0FFE709985E
:105750000168402008650998FFF79CFFFFE7FFE715
:105760009DF80100C007E0B1FFE79DF80500C00704
:10577000B0B1FFE709980068D0F8D8000290099806
:105780000068D0F8E010029808400290099801687B
:105790004FF4807008650998029900F02DFCFFE72E
:1057A000FFE7089848B1FFE7089809990968086574
:1057B0000998089900F02CFCFFE7079848B1FFE72B
:1057C00007980999096808650998079900F0F0FA9F
:1057D000FFE7069848B1FFE7069809990968086548
:1057E0000998069900F030FBFFE79DF8010000F0F2
:1057F00002010020B0EB510F13D0FFE79DF8050028
:1058000000F002010020B0EB510F09D0FFE709982A
:1058100001684FF400700865099800F0FFFBFFE78E
:10582000FFE79DF800100020B0EBD11F1DD0FFE76F
:105830009DF804100020B0EBD11F15D0FFE70998A8
:105840000068D0F8D400039009980068D0F8DC1004
:10585000039808400390099801688020086509981A
:10586000039900F0CFFBFFE7FFE79DF8010000F090
:1058700020010020B0EB511F13D0FFE79DF8050079
:1058800000F020010020B0EB511F09D0FFE709987C
:1058900001684FF400500865099800F0A9FBFFE784
:1058A000FFE79DF801100020B0EBD11F11D0FFE7FA
:1058B0009DF805100020B0EBD11F09D0FFE7099833
:1058C00001684FF400400865099800F08DFBFFE780
:1058D000FFE79DF8010000F040010020B0EB911FB0
:1058E00015D0FFE79DF8050000F040010020B0EB67
:1058F000911F0BD0FFE7099801684FF480400865BD
:105900000999086E40F080000866FFE7FFE70498F9
:1059100048B1FFE70498099909680865099804994E
:10592000FFF780FDFFE7059850B1FFE7059809995B
:1059300009680865059A0999086E10430866FFE72B
:105940000998006E20B1FFE70998FFF767FDFFE7B0
:105950000AB080BD80B584B00290029820B9FFE7FC
:1059600001208DF80F0057E1029800684AF20041CB
:10597000C4F20001884201D1FFE7FFE70298806886
:10598000B0F5407F01D1FFE7FFE7029890F85C0097
:1059900040B9FFE70299002081F85D00029800F00D
:1059A0003FF9FFE702980168886920F010008861DC
:1059B00000F04CFE0190FFE7029800688069000744
:1059C000002815D5FFE700F041FE0199401A0B2889
:1059D0000DD3FFE70299086E40F0010008660299B6
:1059E000032081F85C0001208DF80F0014E1E3E74B
:1059F00002980168886940F00100886100F026FE85
:105A00000190FFE7029800688069C007A8B9FFE726
:105A100000F01CFE0199401A0B280DD3FFE70299F4
:105A2000086E40F0010008660299032081F85C00CE
:105A300001208DF80F00EFE0E4E702980168886923
:105A400040F002008861029800684AF20041C4F206
:105A50000001884208D1FFE7029840684AF20051ED
:105A6000C4F200010860FFE70298007C012807D11A
:105A7000FFE702980168886920F04000886106E02D
:105A800002980168886940F040008861FFE7029849
:105A9000407C012807D1FFE702980168886940F43B
:105AA0008040886106E002980168886920F480409F
:105AB0008861FFE70298807C012807D1FFE7029800
:105AC0000168886920F48050886106E002980168C6
:105AD000886940F480508861FFE702980068806917
:105AE00020F44070029A116892681043886102980D
:105AF0000168886920F0A40088610298016808693B
:105B000020F0100008610298C068012807D1FFE763
:105B100002980168886940F0040088612BE00298CF
:105B2000C06830B3FFE70298C068022819D0FFE7C9
:105B300002980168886940F08000886102980168D5
:105B4000086940F0100008610298C068032807D176
:105B5000FFE702980168886940F020008861FFE74C
:105B600006E002980168886940F020008861FFE73C
:105B700000E0FFE7FFE7029A116853699069D2F8E5
:105B80001CE0A0F1010C6FF0FF0000EB0E2040EADA
:105B90004C60126A013A10430022CFF6FF7202EB0A
:105BA00003421043C86102988068B0F5407F1CD161
:105BB000FFE7029A1168536A906AD2F82CE0013824
:105BC0006FF0FF0C0CEB0E2C40EA0C00D2F830C04A
:105BD0006FF00F0202EB0C1210430022CFF6FF729F
:105BE00002EB03421043C860FFE702980168C26BF2
:105BF000D1F8C0001043C1F8C0000298FCF720FAA9
:105C000002990020886502990866029A012182F8AB
:105C10005C108DF80F00FFE79DF80F0004B080BD09
:105C200080B5C2B04190002040903F903E903D90A2
:105C30003C9008A8D021FAF7FCFB419800684AF292
:105C40000041C4F20001884252D1FFE704200990CC
:105C5000002008902D9008A800F0FCFD18B1FFE787
:105C6000FCF7CCF9FFE740F26810C2F200000168CF
:105C7000013101600068012810D1FFE7FFE740F61D
:105C8000A040C4F20240016841F400710160006864
:105C900000F4007007900798FFE7FFE7FFE740F682
:105CA0008C40C4F20240016841F0010101600068CB
:105CB00000F0010006900698FFE74FF4C0503C90BA
:105CC00002203D90002002903E903F90092040909D
:105CD0000020C4F202203CA900F014FB029A272005
:105CE0000390114600F096FD039800F089FD5CE0FA
:105CF000419800684AF60001C4F20001884253D17D
:105D0000FFE704200990002008902D9008A800F0DB
:105D1000A1FD18B1FFE7FCF771F9FFE740F2681049
:105D2000C2F200000168013101600068012810D151
:105D3000FFE7FFE740F6A040C4F20240016841F4EB
:105D400000710160006800F4007005900598FFE79D
:105D5000FFE7FFE740F68C40C4F20240016841F0E3
:105D600002010160006800F0020004900498FFE75F
:105D70004FF440503C9002203D90002000903E9017
:105D80003F900920409040F20040C4F202203CA91C
:105D900000F0B8FA009A6D200190114600F03AFD2B
:105DA000019800F02DFDFFE7FFE742B080BD000045
:105DB00080B59EB01D901C910CA84021FAF717FBEE
:105DC00002A82821FAF735FB9DF87000C00760B3E0
:105DD000FFE7FFE71D98402102AA0CABFFF742FB4B
:105DE000FFE71D984021FFF723FB0028F2D1FFE7D2
:105DF0000598FAF793FFADF806000398B0F1804FCD
:105E000012D1FFE7BDF90600092801DBFFE719E021
:105E100002980CA9FBF73AFA40F2E850C2F20000EF
:105E200007F0D8FEFFE7FFE7FFE79DF870004007A7
:105E3000002807D5FFE71D98402102AA0CABFFF709
:105E400011FBFFE71EB080BD80B5ACB02B902A914E
:105E50001AA84021FAF7CBFA10A82821FAF7E9FA94
:105E60009DF8A8000007002840F18880FFE7FFE7C1
:105E70002B98412110AA1AABFFF7F4FAFFE72B98F1
:105E80004121FFF7D5FA0028F2D1FFE71398FAF77E
:105E900045FFADF83E001198B0F1804F6DD1FFE79E
:105EA000BDF93E00092801DBFFE774E0109801907E
:105EB000B0F5805F33D0FFE7019841F201018842DD
:105EC0003ED0FFE7019841F22131C0F2080188423B
:105ED00047D1FFE710981199129A139BDDF850C033
:105EE000DDF854E0CDF820E0CDF81CC00693059213
:105EF0000491039016981799189A199B0C930B927A
:105F00000A9109901A981B990E910D9040F26830F1
:105F1000C2F2000003A9012207F082FF2CE0BDF8C5
:105F20006800ADF80A00BDF90A0005F075FCBDF87F
:105F30006A00ADF80A00BDF90A0005F07BFC1BE021
:105F4000BDF86800ADF80800BDF9080006F03CF89F
:105F5000BDF86A00ADF80800BDF9080006F042F887
:105F60000AE010981AA9FBF791F940F28450C2F2A6
:105F7000000007F02FFEFFE7FFE7FFE79DF8A8000E
:105F80008006002807D5FFE72B98412110AA1AABFD
:105F9000FFF768FAFFE72CB080BD000082B00090E8
:105FA000009890F85C00012810D1FFE700990220CA
:105FB00081F85C0000980168886920F00100886120
:105FC0000099002008668DF8070008E00099086E27
:105FD00040F00400086601208DF80700FFE79DF8F7
:105FE000070002B07047000081B0009001B0704718
:105FF00081B0009001B0704782B00190009102B072
:106000007047000082B00190009102B0704700001C
:1060100082B00190009102B07047000081B0009002
:1060200001B0704780B586B004900391FFE740F25D
:106030004800C2F200000078012804D1FFE70220E6
:106040008DF817008BE040F24801C2F200010120F8
:106050000870FFE7FFE740F24801C2F200010020AC
:1060600048604FF47A70FCF7C1F98DF80B009DF889
:106070000B00002866D1FFE70498006840F2480151
:10608000C2F20001886042F22800C4F202000090CF
:106090000498006820F0004048F2080188420BD1C3
:1060A000FFE704984068FCF7B5F84FF47A70FCF706
:1060B0009DF98DF80B003AE0049800680821C8F2B9
:1060C0000001884209D1FFE7FCF7DAF84FF47A7053
:1060D000FCF78CF98DF80B0028E003994FF0FF30A6
:1060E0000860049880680190FFE7019804998A6825
:1060F000C9681144884218D2FFE701980499496899
:10610000FCF758F84FF47A70FCF770F98DF80B0033
:106110009DF80B0020B1FFE701980399086004E0A7
:10612000FFE7019801300190DFE7FFE7FFE7049800
:1061300001684FF0004060EA0102009908681040D1
:106140000860FFE7FFE740F24801C2F200010020CB
:106150000870FFE79DF80B008DF81700FFE79DF82A
:10616000170006B080BD000081B000208DF803004C
:1061700042F22800C4F20200016841F0010101600E
:106180000068C00720B9FFE701208DF80300FFE792
:106190009DF8030001B0704780B586B0059004916A
:1061A000039240F24801C2F20001002048604FF41F
:1061B0007A70FCF71BF98DF80B009DF80B00002896
:1061C00070D1FFE7059840F24801C2F200018860F3
:1061D00042F22800C4F202000190059820F000402D
:1061E000022805D1FFE704980399FCF76BF836E025
:1061F00005980221C1F20001884207D0FFE7059807
:106200000621C1F20001884205D1FFE704980399F5
:10621000FCF790F822E0059820F000400221C4F23B
:106220000001884205D1FFE704980399FCF736F88E
:1062300013E0059820F000400221C6F200018842D8
:1062400005D1FFE704980399FCF7BCF804E0049833
:106250000399FCF723F8FFE7FFE7FFE7FFE74FF4B9
:106260007A70FCF7C3F88DF80B0005990420CBF287
:10627000000060EA01020199086810400860059872
:106280000621C1F2000188420BD1FFE742F2400033
:10629000C4F2020000900099086820F00400086031
:1062A000FFE7FFE79DF80B0006B080BD81B000203E
:1062B0008DF8030042F22800C4F202000068C00713
:1062C000D8B1FFE742F20401C4F2020140F2231008
:1062D000C4F26750086048F6AB10CCF6EF50086087
:1062E00042F22800C4F202000068C00720B1FFE7B4
:1062F00001208DF80300FFE7FFE79DF8030001B0E0
:106300007047000085B00490039100200090FFE7E3
:10631000039800680099C840002800F06681FFE7F4
:1063200003980068009A012191400840019001986B
:10633000002800F05681FFE703984068022805D046
:10634000FFE703984068122828D1FFE704980099D6
:106350006FF0030202EA51010844006A02900098BB
:1063600000F0070081000F2000FA01F10298884335
:1063700002900398006900F00F00009901F00701F6
:10638000890000FA01F102980843029002980499EA
:10639000009B02EA530211440862FFE70498006878
:1063A000029000984100032000FA01F1029888430E
:1063B00002900398406800F003000099490000FA39
:1063C00001F102980843029002980499086003982A
:1063D000406801280FD0FFE70398406802280AD0E0
:1063E000FFE703984068112805D0FFE7039840684D
:1063F00012282FD1FFE7049880680290009841008E
:10640000032000FA01F10298884302900398C068C3
:106410000099490000FA01F102980843029002989D
:10642000049988600498406802900099012000FA5D
:1064300001F102988843029003984068C0F300106D
:10644000009900FA01F10298084302900298049919
:106450004860FFE70398406800F0030003280CD170
:10646000FFE70398406800F0030003281DD1FFE711
:1064700003988068012818D0FFE70498C06802904C
:1064800000984100032000FA01F10298884302902D
:10649000039880680099490000FA01F102980843C6
:1064A000029002980499C860FFE70398C079C0067B
:1064B000002840F19580FFE7009820F0030042F2A9
:1064C0006002C4F2024280580290009800F003007B
:1064D000C1000F2000FA01F102988843029004984D
:1064E0004FF60041CBF6FD510840800A009901F0BB
:1064F0000301C90000FA01F10298084302900298D2
:10650000009921F00301885042F20000C4F20240D9
:10651000006802900199029888430290039880795C
:10652000C006002805D5FFE70199029808430290AC
:10653000FFE7029842F20001C4F20241086042F211
:106540000400C4F202400068029001990298884356
:106550000290039880798006002805D5FFE701990D
:10656000029808430290FFE7029842F20401C4F245
:106570000241086042F28400C4F2024000680290C6
:106580000199029888430290039880798007002837
:1065900005D5FFE70199029808430290FFE70298AA
:1065A00042F28401C4F20241086042F28000C4F267
:1065B0000240006802900199029888430290039873
:1065C0008079C00728B1FFE701990298084302903B
:1065D000FFE7029842F28001C4F202410860FFE73F
:1065E000FFE700980130009092E605B07047000088
:1065F00082B00190ADF8021001980069BDF8021058
:10660000084204D0FFE701208DF8010003E00020DC
:106610008DF80100FFE79DF8010002B0704700000F
:1066200082B00190ADF802108DF801209DF80100B4
:1066300028B1FFE7BDF802000199886104E0BDF8C8
:10664000020001998862FFE702B0704740F6180027
:10665000C2F200000068704740F20041C4F203013A
:10666000086840F0010008600020704740F2F80020
:10667000C2F20000027840F61801C2F20001086878
:10668000104408607047000080B582B0032000F01D
:10669000D9F801F013FB40F62041C4F20241096829
:1066A00001F00F024EF2AC01C0F60001895CC84057
:1066B00040F20401C2F200010860042002F062F915
:1066C0000F2000F011F820B1FFE701208DF807003E
:1066D00005E000F093F800208DF80700FFE79DF833
:1066E000070002B080BD000080B586B00490002095
:1066F000039040F2F800C2F20000007820B9FFE7F2
:1067000001208DF8170075E04EF21000CEF2000067
:1067100000684007002812D5FFE740F20400C2F2EB
:106720000000006840F2F801C2F200010A784FF45C
:106730007A71B1FBF2F1B0FBF1F0039040E002F0AE
:1067400095F902900298019040B1FFE70198012865
:1067500016D0FFE70198022821D02FE040F2040074
:10676000C2F20000006840F2F801C2F200010A78AB
:106770004FF4FA51B1FBF2F1B0FBF1F003901EE0DF
:1067800040F2F800C2F2000001784FF47A70B0FBDA
:10679000F1F14FF4FA40B0FBF1F003900FE040F25A
:1067A000F800C2F2000001784FF47A70B0FBF1F10A
:1067B0004FF40040B0FBF1F0039000E0FFE7FFE78B
:1067C000039802F02DF920B1FFE701208DF81700A2
:1067D00010E004994FF0FF300022009200F01AF808
:1067E0000098049940F2FC02C2F2000211608DF898
:1067F0001700FFE79DF8170006B080BD7047000046
:1068000080B582B0ADF80600BDF9060006F00CFFB9
:1068100002B080BD80B586B0ADF816000491039239
:1068200006F01AFF0290BDF9160001900298049933
:10683000039A04F0BBFF0146019806F015FF06B06D
:1068400080BD000080B582B00190019806F02EFF57
:1068500002B080BD80B59EB01D9000208DF86B0009
:106860008DF86A001D98C078C00760B1FFE740F658
:10687000E841C4F20241086820F040401D9A926D40
:1068800010430860FFE71D980068C007002837D054
:10689000FFE71D98C06D1990052817D81999DFE8F2
:1068A00001F003040B12131414E01D98083005F0D6
:1068B000F9F88DF86B000DE01D98303005F0A8F95F
:1068C0008DF86B0006E005E004E003E001208DF8A0
:1068D0006B00FFE79DF86B0060B9FFE740F6D84119
:1068E000C4F20241086820F007001D9AD26D1043DF
:1068F000086004E09DF86B008DF86A00FFE7FFE791
:106900001D9800788007002840F14A80FFE71D9815
:10691000006E1890282829D81899DFE801F015276B
:1069200027272727272716272727272727271D2712
:1069300027272727272724272727272727272527EC
:10694000272727272727260014E01D98083005F061
:10695000A9F88DF86B000DE01D98303005F058F95E
:106960008DF86B0006E005E004E003E001208DF8FF
:106970006B00FFE79DF86B0060B9FFE740F6D84178
:10698000C4F20241086820F038001D9A126E1043CC
:10699000086004E09DF86B008DF86A00FFE7FFE7F0
:1069A0001D9800784007002847D5FFE71D98406EE6
:1069B0001790B0B1FFE71798402813D0FFE717985A
:1069C000802816D0FFE71798C02819D0FFE717983E
:1069D000B0F5807F15D0FFE71798B0F5A07F11D0F4
:1069E00011E014E01D98083005F05CF88DF86B009C
:1069F0000DE01D98303005F00BF98DF86B0006E0C6
:106A000005E004E003E001208DF86B00FFE79DF84E
:106A10006B0060B9FFE740F6D841C4F20241086854
:106A200020F4E0701D9A526E1043086004E09DF857
:106A30006B008DF86A00FFE7FFE71D9800780007FC
:106A400000284AD5FFE71D98806E1690C8B1FFE771
:106A50001698B0F5007F15D0FFE71698B0F5806F57
:106A600017D0FFE71698B0F5C06F19D0FFE716985A
:106A7000B0F5006F15D0FFE71698B0F5206F11D074
:106A800011E014E01D98083005F00CF88DF86B004B
:106A90000DE01D98303005F0BBF88DF86B0006E076
:106AA00005E004E003E001208DF86B00FFE79DF8AE
:106AB0006B0060B9FFE740F6D841C4F202410868B4
:106AC00020F460601D9A926E1043086004E09DF807
:106AD0006B008DF86A00FFE7FFE71D980078C0069D
:106AE00000284AD5FFE71D98C06E1590C8B1FFE792
:106AF0001598B0F5805F15D0FFE71598B0F5005FE9
:106B000017D0FFE71598B0F5405F19D0FFE715984B
:106B1000B0F5804F15D0FFE71598B0F5A04F11D014
:106B200011E014E01D98083004F0BCFF8DF86B00F4
:106B30000DE01D98303005F06BF88DF86B0006E025
:106B400005E004E003E001208DF86B00FFE79DF80D
:106B50006B0060B9FFE740F6D841C4F20241086813
:106B600020F4E0401D9AD26E1043086004E09DF8C6
:106B70006B008DF86A00FFE7FFE71D98007880063C
:106B800000284AD5FFE71D98006F1490C8B1FFE7B1
:106B90001498B0F5004F15D0FFE71498B0F5803F7A
:106BA00017D0FFE71498B0F5C03F19D0FFE714984D
:106BB000B0F5003F15D0FFE71498B0F5203F11D095
:106BC00011E014E01D98083004F06CFF8DF86B00A4
:106BD0000DE01D98303005F01BF88DF86B0006E0D5
:106BE00005E004E003E001208DF86B00FFE79DF86D
:106BF0006B0060B9FFE740F6D841C4F20241086873
:106C000020F460301D9A126F1043086004E09DF874
:106C10006B008DF86A00FFE7FFE71D984078C0061B
:106C200000284AD5FFE71D98406F1390C8B1FFE7D1
:106C30001398B0F1807F15D0FFE71398B0F1007F73
:106C400017D0FFE71398B0F1407F19D0FFE71398F2
:106C5000B0F1806F15D0FFE71398B0F1A06F11D09D
:106C600011E014E01D98083004F01CFF8DF86B0053
:106C70000DE01D98303004F0CBFF8DF86B0006E07E
:106C800005E004E003E001208DF86B00FFE79DF8CC
:106C90006B0060B9FFE740F6E041C4F202410868CA
:106CA00020F0E0601D9A526F1043086004E09DF8E8
:106CB0006B008DF86A00FFE7FFE71D9840788006BB
:106CC000002838D5FFE71D98806F129078B1FFE754
:106CD0001298B0F5803F0BD0FFE71298B0F5003F57
:106CE0000DD0FFE71298B0F5403F09D009E00CE065
:106CF0001D98303004F08CFF8DF86B0005E004E047
:106D000003E001208DF86B00FFE79DF86B0060B990
:106D1000FFE740F6E441C4F20241086820F4403045
:106D20001D9A926F1043086004E09DF86B008DF887
:106D30006A00FFE7FFE71D9840784006002838D535
:106D4000FFE71D98C06F119078B1FFE71198B0F57B
:106D5000802F0BD0FFE71198B0F5002F0DD0FFE783
:106D60001198B0F5402F09D009E00CE01D983030A3
:106D700004F04EFF8DF86B0005E004E003E0012015
:106D80008DF86B00FFE79DF86B0060B9FFE740F6F8
:106D9000E441C4F20241086820F440201D9AD26FF9
:106DA0001043086004E09DF86B008DF86A00FFE76F
:106DB000FFE71D984078000600283AD5FFE71D98A8
:106DC000D0F88000109078B1FFE71098B0F5801FE0
:106DD0000BD0FFE71098B0F5001F0DD0FFE710981B
:106DE000B0F5401F09D009E00CE01D98303004F0E8
:106DF0000FFF8DF86B0005E004E003E001208DF843
:106E00006B00FFE79DF86B0068B9FFE740F6E441CF
:106E1000C4F20241086820F440101D9AD2F8802084
:106E20001043086004E09DF86B008DF86A00FFE7EE
:106E3000FFE71D988078C007A0B3FFE71D98D0F842
:106E400084000F9050B1FFE70F98B0F1807F06D01B
:106E5000FFE70F98B0F1007F08D008E00BE01D9825
:106E6000303004F0D5FE8DF86B0004E003E0012023
:106E70008DF86B00FFE79DF86B0068B9FFE740F6FF
:106E8000E441C4F20241086820F040701D9AD2F833
:106E900084201043086004E09DF86B008DF86A00C0
:106EA000FFE7FFE71D984079C006002834D5FFE7CB
:106EB0001D98D0F888000E9050B1FFE70E98B0F101
:106EC000806F06D0FFE70E98B0F1006F08D008E0A1
:106ED0000BE01D98303004F09BFE8DF86B0004E051
:106EE00003E001208DF86B00FFE79DF86B0068B9A7
:106EF000FFE740F6E441C4F20241086820F0406038
:106F00001D9AD2F888201043086004E09DF86B00B9
:106F10008DF86A00FFE7FFE71D9840790007002819
:106F200011D5FFE7FFE740F61C41C4F202410868B3
:106F300020F4004008601D98D0F8C820086810436D
:106F40000860FFE7FFE71D988078800700284CD590
:106F5000FFE71D98D0F88C000D90C8B1FFE70D98A1
:106F6000B0F5807F15D0FFE70D98B0F5007F17D002
:106F7000FFE70D98B0F5407F19D0FFE70D98B0F509
:106F8000806F15D0FFE70D98B0F5A06F11D011E01C
:106F900014E01D98083004F085FD8DF86B000DE0BD
:106FA0001D98303004F034FE8DF86B0006E005E0EB
:106FB00004E003E001208DF86B00FFE79DF86B0013
:106FC00068B9FFE740F6DC41C4F20241086820F4EA
:106FD000E0601D9AD2F88C201043086004E09DF810
:106FE0006B008DF86A00FFE7FFE71D988078400787
:106FF00000284CD5FFE71D98D0F890000C90C8B140
:10700000FFE70C98B0F5805F15D0FFE70C98B0F55E
:10701000005F17D0FFE70C98B0F5405F19D0FFE78D
:107020000C98B0F5804F15D0FFE70C98B0F5A04F45
:1070300011D011E014E01D98083004F033FD8DF8F4
:107040006B000DE01D98303004F0E2FD8DF86B0010
:1070500006E005E004E003E001208DF86B00FFE7A7
:107060009DF86B0068B9FFE740F6DC41C4F20241CD
:10707000086820F4E0401D9AD2F890201043086080
:1070800004E09DF86B008DF86A00FFE7FFE71D98AC
:1070900080788006002834D5FFE71D98D0F8A0003E
:1070A0000B90022809D3FFE70B98022806D0FFE7D0
:1070B0000B980338032808D308E00BE01D9808302C
:1070C00004F0F0FC8DF86B0004E003E001208DF883
:1070D0006B00FFE79DF86B0068B9FFE740F6E841F9
:1070E000C4F20241086820F007001D9AD2F8A020DF
:1070F0001043086004E09DF86B008DF86A00FFE71C
:10710000FFE71D9840798007002827D5FFE71D98E5
:10711000D0F8A4000A9020B1FFE70A98082801D00F
:1071200001E004E003E001208DF86B00FFE79DF82B
:107130006B0068B9FFE740F6E841C4F20241086815
:1071400020F008001D9AD2F8A4201043086004E043
:107150009DF86B008DF86A00FFE7FFE71D98C07887
:107160008007002840F1B580FFE740F62401C4F213
:107170000241086840F001000860FFF767FA1B90C1
:10718000FFE740F62400C4F202400068C00760B97F
:10719000FFE7FFF75BFA1B99401A032804D3FFE7C8
:1071A00003208DF86B0000E0EBE79DF86B000028F2
:1071B00040F08980FFE740F6F040C4F202400068EA
:1071C00000F440701C901C98D0B1FFE71C981D99EA
:1071D000D1F8BC10884213D0FFE740F6F041C4F26A
:1071E0000241086820F440701C90086840F4803028
:1071F0000860086820F4803008601C980860FFE789
:107200009DF87000C007E0B1FFE7FFF71FFA1B9081
:10721000FFE740F6F040C4F2024000688007002813
:107220000ED4FFE7FFF712FA1B99401A41F2893199
:10723000884204D3FFE703208DF86B0000E0E8E705
:10724000FFE79DF86B00C0BBFFE7FFE71D98D0F894
:10725000BC0000F44070B0F5407F13D1FFE740F66A
:107260001C41C4F20241086820F47C501D9AD2F8F7
:10727000BC204FF6F043C0F6FF731A4040EA1210EC
:10728000086008E040F61C41C4F20241086820F49E
:107290007C500860FFE740F6F041C4F20241086804
:1072A00020F4407008601D98D0F8BC206FF31F32A6
:1072B000086810430860FFE704E09DF86B008DF854
:1072C0006A00FFE704E09DF86B008DF86A00FFE7B5
:1072D000FFE71D98C0784007002839D5FFE71D98C3
:1072E000D0F89800099060B1FFE70998102809D0FC
:1072F000FFE7099820280ED0FFE7099830280BD027
:107300000BE00EE040F62841C4F20241086840F468
:107310000030086005E004E003E001208DF86B0018
:10732000FFE79DF86B0068B9FFE740F6E841C4F25B
:107330000241086820F030001D9AD2F898201043CE
:10734000086004E09DF86B008DF86A00FFE7FFE736
:107350001D9880784006002835D5FFE71D98D0F8A5
:107360009C00089020B1FFE70898402809D00FE062
:1073700040F62841C4F20241086840F40030086039
:107380000AE01D98083004F08DFB8DF86B0003E0D7
:1073900001208DF86B00FFE79DF86B0068B9FFE7EF
:1073A00040F6E441C4F20241086820F040001D9A12
:1073B000D2F89C201043086004E09DF86B008DF823
:1073C0006A00FFE7FFE71D98C0780007002840D556
:1073D000FFE71D98D0F8AC00079004281ED8079945
:1073E000DFE801F0030C131A1B0040F62841C4F239
:1073F0000241086840F40030086013E01D9808302E
:1074000004F050FB8DF86B000CE01D98303004F058
:10741000FFFB8DF86B0005E004E003E001208DF830
:107420006B00FFE79DF86B0068B9FFE740F6E041AD
:10743000C4F20241086820F007001D9AD2F8AC207F
:107440001043086004E09DF86B008DF86A00FFE7C8
:10745000FFE71D98C078C006002840F14F80FFE785
:107460001D98D0F8B000069020282CD80699DFE8A7
:1074700001F0112A2A2A2A2A2A2A1A2A2A2A2A2AF8
:107480002A2A212A2A2A2A2A2A2A282A2A2A2A2A67
:107490002A2A290040F62841C4F20241086840F433
:1074A0000030086013E01D98083004F0FBFA8DF8F6
:1074B0006B000CE01D98303004F0AAFB8DF86B00D7
:1074C00005E004E003E001208DF86B00FFE79DF884
:1074D0006B0068B9FFE740F6E041C4F2024108687A
:1074E00020F038001D9AD2F8B0201043086004E064
:1074F0009DF86B008DF86A00FFE7FFE71D98C078E4
:10750000800600284BD5FFE71D98D0F8B400059001
:1075100088B1FFE70598402816D0FFE70598802836
:1075200019D0FFE70598C0281CD0FFE70598B0F5F3
:10753000807F18D018E040F62841C4F20241086864
:1075400040F40030086013E01D98083004F0AAFAF7
:107550008DF86B000CE01D98303004F059FB8DF86D
:107560006B0005E004E003E001208DF86B00FFE70D
:107570009DF86B0068B9FFE740F6E041C4F20241B4
:10758000086820F4E0701D9AD2F8B4201043086017
:1075900004E09DF86B008DF86A00FFE7FFE71D9897
:1075A000C078400600284CD5FFE71D98D0F8B800F9
:1075B0000490C8B1FFE70498B0F5007F15D0FFE74D
:1075C0000498B0F5806F17D0FFE70498B0F5C06F4E
:1075D00019D0FFE70498B0F5006F15D0FFE70498C5
:1075E000B0F5206F11D011E014E01D98083004F0C0
:1075F00059FA8DF86B000DE01D98303004F008FB4F
:107600008DF86B0006E005E004E003E001208DF852
:107610006B00FFE79DF86B0068B9FFE740F6E041BB
:10762000C4F20241086820F460601D9AD2F8B820C4
:107630001043086004E09DF86B008DF86A00FFE7D6
:10764000FFE71D9800798007002838D5FFE71D98CF
:10765000D0F8A8000390032816D80399DFE801F0BA
:1076600002030C1314E040F62841C4F202410868FA
:1076700040F4003008600BE01D98083004F012FA66
:107680008DF86B0004E003E001208DF86B00FFE74C
:107690009DF86B0068B9FFE740F6E441C4F202418F
:1076A000086820F003001D9AD2F8A8201043086053
:1076B00004E09DF86B008DF86A00FFE7FFE71D9876
:1076C0000079400700283CD5FFE71D98D0F89400CA
:1076D000029050B1FFE70298B0F5807F06D0FFE737
:1076E0000298B0F5007F0AD010E013E040F6284180
:1076F000C4F20241086840F4003008600AE01D98B6
:10770000083004F0CFF98DF86B0003E001208DF80C
:107710006B00FFE79DF86B0068B9FFE740F6E841B2
:10772000C4F20241086820F440701D9AD2F89420F7
:107730001043086004E09DF86B008DF86A00FFE7D5
:10774000FFE71D980079C00600283BD5FFE71D988C
:10775000D0F8C4000190102808D0FFE70198202835
:107760000DD0FFE70198302810D010E040F62841F6
:10777000C4F20241086840F4003008600BE01D9834
:10778000303004F045FA8DF86B0004E003E001208E
:107790008DF86B00FFE79DF86B0068B9FFE740F6D6
:1077A000E441C4F20241086820F030001D9AD2F88A
:1077B000C4201043086004E09DF86B008DF86A0057
:1077C000FFE7FFE71D980079000700280DD5FFE7C8
:1077D00040F6E841C4F20241086820F0C0001D9A5A
:1077E000D2F8C02010430860FFE79DF86A001EB081
:1077F00080BD000080B586B004900391049820B944
:10780000FFE701208DF817003AE2039842F20001E9
:10781000C4F20201096801F00F01884216D9FFE79E
:1078200042F20000C4F20200016821F00F01039A45
:1078300011430160006800F00F000399884204D0F2
:10784000FFE701208DF817001AE2FFE7049800789F
:10785000C00600281BD5FFE70498406940F6204188
:10786000C4F20241096801F4E041B0EB112F0DD9D7
:10787000FFE740F62041C4F20241086820F4E040EE
:10788000049A526940EA02200860FFE7FFE7049883
:107890000078000700281BD5FFE70498006940F630
:1078A0002041C4F20241096801F4E061B0EB111F0C
:1078B0000DD9FFE740F62041C4F20241086820F4E8
:1078C000E060049A126940EA02100860FFE7FFE7EF
:1078D000049800784007002819D5FFE70498C0688D
:1078E00040F62041C4F20241096801F0700188426B
:1078F0000CD9FFE740F62041C4F20241086820F0AD
:107900007000049AD26810430860FFE7FFE704980C
:1079100000788007002819D5FFE70498806840F6B2
:107920002041C4F20241096801F00F0188420CD9DC
:10793000FFE740F62041C4F20241086820F00F0042
:10794000049A926810430860FFE7FFE70498007804
:10795000C007002800F0D180FFE7049840680328A2
:107960000ED1FFE740F60040C4F2024000688001FB
:10797000002804D4FFE701208DF8170080E135E0EE
:107980000498406802280ED1FFE740F60040C4F298
:10799000024000688003002804D4FFE701208DF82E
:1079A00017006DE121E00498406801280ED1FFE73F
:1079B00040F60040C4F2024000688005002804D46C
:1079C000FFE701208DF817005AE10DE040F6004076
:1079D000C4F2024000688007002804D4FFE70120B9
:1079E0008DF817004CE1FFE7FFE7FFE740F61C4189
:1079F000C4F20241086820F00300049A5268104360
:107A00000860FEF723FE01900498406803281AD10D
:107A1000FFE7FFE740F61C40C4F20240006800F0B8
:107A2000180018280ED0FFE7FEF710FE0199401A43
:107A300041F28931884204D3FFE703208DF8170013
:107A40001EE1E7E758E00498406802281AD1FFE7F2
:107A5000FFE740F61C40C4F20240006800F0180046
:107A600010280ED0FFE7FEF7F1FD0199401A41F210
:107A70008931884204D3FFE703208DF81700FFE027
:107A8000E7E738E00498406801281AD1FFE7FFE7EC
:107A900040F61C40C4F20240006800F018000828BC
:107AA0000ED0FFE7FEF7D2FD0199401A41F289316D
:107AB000884204D3FFE703208DF81700E0E0E7E7F2
:107AC00018E0FFE740F61C40C4F20240006810F0E6
:107AD000180F0ED0FFE7FEF7B9FD0199401A41F2E9
:107AE0008931884204D3FFE703208DF81700C7E0EF
:107AF000E8E7FFE7FFE7FFE7FFE704980078800784
:107B0000002819D5FFE70498806840F62041C4F2A8
:107B10000241096801F00F0188420CD2FFE740F6EC
:107B20002041C4F20241086820F00F00049A9268D4
:107B300010430860FFE7FFE7039842F20001C4F238
:107B40000201096801F00F01884216D2FFE742F2F4
:107B50000000C4F20200016821F00F01039A1143F2
:107B60000160006800F00F000399884204D0FFE72D
:107B700001208DF8170083E0FFE7049800784007A4
:107B8000002819D5FFE70498C06840F62041C4F2E8
:107B90000241096801F0700188420CD2FFE740F60B
:107BA0002041C4F20241086820F07000049AD268B3
:107BB00010430860FFE7FFE70498007800070028FB
:107BC0001BD5FFE70498006940F62041C4F202414A
:107BD000096801F4E061B0EB111F0DD2FFE740F638
:107BE0002041C4F20241086820F4E060049A12695E
:107BF00040EA02100860FFE7FFE704980078C0063B
:107C000000281BD5FFE70498406940F62041C4F2E4
:107C10000241096801F4E041B0EB112F0DD2FFE7FA
:107C200040F62041C4F20241086820F4E040049A82
:107C3000526940EA02200860FFE7FFE700F03EF8E3
:107C400040F62041C4F20241096801F00F024EF2F1
:107C5000AC01C0F60001895CC84040F20401C2F2E8
:107C60000001086040F2FC00C2F200000068FEF76C
:107C70003BFD8DF80B009DF80B008DF81700FFE71A
:107C80009DF8170006B080BD80B500F017F840F6EB
:107C90002041C4F20241096801F00F024EF2AC012A
:107CA000C0F60001895C01F01F0120FA01F140F2E9
:107CB0000400C2F200000160006880BD89B040F697
:107CC0001C40C4F20240006800F01800082806D1E9
:107CD000FFE740F60010C0F23D00049048E140F696
:107CE0001C40C4F20240006810F0180F21D1FFE7D9
:107CF00040F60040C4F20240006800F0200100207D
:107D0000B0EB511F0ED0FFE740F60040C4F2024036
:107D10000068C0F3C10149F20000C0F2D030C84091
:107D2000049005E049F20000C0F2D0300490FFE773
:107D30001DE140F61C40C4F20240006800F018004B
:107D4000102806D1FFE747F64000C0F27D100490EE
:107D50000CE140F61C40C4F20240006800F018003C
:107D6000182840F0FC80FFE740F62840C4F20240AB
:107D7000016801F0030108910168C1F30521069132
:107D80000068C0F300100590059840F63841C4F231
:107D90000241096889B2C90800FB01F000EE100A2F
:107DA000B8EE400A8DED020A0698002800F0D38054
:107DB000FFE708980090012809D0FFE70098022803
:107DC00000F08D80FFE70098032864D088E040F63B
:107DD0000040C4F20240006800F020010020B0EB37
:107DE000511F33D0FFE740F60040C4F20240006864
:107DF000C0F3C10149F20000C0F2D030C840039086
:107E00009DED030AB8EE400A9DED061AB8EE411A40
:107E100080EE010A40F63440C4F2024000686FF37D
:107E20005F2001EE100AB8EE411A9DED022A9FED87
:107E3000533A22EE032A31EE021AB7EE002A31EE4F
:107E4000021A20EE010A8DED010A23E09DED060ADB
:107E5000B8EE401A9FED4A0A80EE010A40F634401F
:107E6000C4F2024000686FF35F2001EE100AB8EE22
:107E7000411A9DED022A9FED413A22EE032A31EE8E
:107E8000021AB7EE002A31EE021A20EE010A8DED39
:107E9000010AFFE748E09DED060AB8EE401A9FEDA3
:107EA000360A80EE010A40F63440C4F2024000680F
:107EB0006FF35F2001EE100AB8EE411A9DED022A21
:107EC0009FED2E3A22EE032A31EE021AB7EE002A77
:107ED00031EE021A20EE010A8DED010A24E0FFE7DF
:107EE0009DED060AB8EE401A9FED260A80EE010AC3
:107EF00040F63440C4F2024000686FF35F2001EEA8
:107F0000100AB8EE411A9DED022A9FED1C3A22EEAE
:107F1000032A31EE021AB7EE002A31EE021A20EEE1
:107F2000010A8DED010AFFE740F63440C4F2024039
:107F3000006881B2012000EB512007909DED010AFD
:107F40009DED071AB8EE411A80EE010ABCEEC00A98
:107F50008DED040A02E000200490FFE705E049F2FD
:107F60000000C0F2D0300490FFE7FFE7FFE7FFE733
:107F7000049809B0704700BF20BCBE4B0000003918
:107F80000024744C0024744A80B588B0069006988A
:107F900028B9FFE701208DF81F0000F0EFBC40F684
:107FA0001C40C4F20240006800F01800049040F643
:107FB0002840C4F20240006800F0030003900698D5
:107FC0000078C006002840F18080FFE70498082868
:107FD00008D0FFE7049818281DD1FFE7039802286E
:107FE00019D1FFE70698C06928B9FFE701208DF88D
:107FF0001F0000F0C3BCFFE740F61841C4F2024185
:10800000086820F47C10069A126A40EA0240086070
:10801000FFE7FFE758E00698C06988B3FFE740F63E
:108020000041C4F20241086840F480700860FEF725
:108030000DFB0590FFE740F60040C4F202400068E7
:10804000800500280DD4FFE7FEF700FB0599401AD4
:10805000032805D3FFE703208DF81F0000F08EBC36
:10806000E9E7FFE740F61841C4F20241086820F44E
:108070007C10069A126A40EA02400860FFE722E09C
:1080800040F60041C4F20241086820F480700860A4
:10809000FEF7DCFA0590FFE740F60040C4F202402C
:1080A0000068800500280DD5FFE7FEF7CFFA059997
:1080B000401A032805D3FFE703208DF81F0000F0C6
:1080C0005DBCE9E7FFE7FFE7FFE706980078C00738
:1080D000002800F0B980FFE70498102808D0FFE7D7
:1080E000049818280ED1FFE7039803280AD1FFE768
:1080F0000698406828B9FFE701208DF81F0000F0BE
:108100003DBCA0E0FFE706984068B0F5803F09D18C
:10811000FFE740F60041C4F20241086840F48030B5
:10812000086056E00698406888B9FFE740F60041CD
:10813000C4F20241086820F480300860086820F426
:1081400080100860086820F48020086040E00698ED
:108150004068B0F5A02F11D1FFE740F60041C4F20E
:108160000241086840F480200860086820F480100C
:108170000860086840F48030086028E0069840688D
:10818000B0F5A81F11D1FFE740F60041C4F202414B
:10819000086840F480200860086840F48010086097
:1081A000086840F48030086010E040F60041C4F2F6
:1081B0000241086820F480300860086820F48020BC
:1081C0000860086820F480100860FFE7FFE7FFE719
:1081D000FFE7FFE706984068D0B1FFE7FEF736FA01
:1081E0000590FFE740F60040C4F2024000688003BB
:1081F00000280CD4FFE7FEF729FA0599401A6528F4
:1082000004D3FFE703208DF81F00B7E3EAE719E086
:10821000FEF71CFA0590FFE740F60040C4F202406A
:108220000068800300280CD5FFE7FEF70FFA0599D8
:10823000401A652804D3FFE703208DF81F009DE353
:10824000EAE7FFE7FFE7FFE70698007880070028E6
:1082500040F1C380FFE7049840B1FFE70498182875
:108260005ED1FFE7039801285AD1FFE70698C0685E
:1082700020B9FFE701208DF81F007FE3049840BB81
:10828000FFE740F60040C4F20240006800F018002A
:108290000699096988421BD0FFE740F60041C4F205
:1082A0000241086820F01800069A1269104308601D
:1082B000FFF7EAFC40F2FC00C2F200000068FEF7A3
:1082C00013FA20B1FFE701208DF81F0056E3FFE706
:1082D000FFE7FEF7BBF90590FFE740F60040C4F268
:1082E00002400068800700280CD4FFE7FEF7AEF9D3
:1082F0000599401A032804D3FFE703208DF81F00D7
:108300003CE3EAE740F61041C4F20241086820F479
:10831000FE00069A526940EA02400860FFE75BE00F
:108320000698C068A8B3FFE740F60041C4F20241D6
:10833000086820F01800069A12691043086008685F
:1083400040F001000860FEF781F90590FFE740F674
:108350000040C4F202400068800700280CD4FFE708
:10836000FEF774F90599401A032804D3FFE70320A8
:108370008DF81F0002E3EAE740F61041C4F2024123
:10838000086820F4FE00069A526940EA024008603C
:1083900021E040F60041C4F20241086820F00100EB
:1083A0000860FEF753F90590FFE740F60040C4F27D
:1083B00002400068800700280CD5FFE7FEF746F969
:1083C0000599401A032804D3FFE703208DF81F0006
:1083D000D4E2EAE7FFE7FFE7FFE706980078000747
:1083E000002849D5FFE70698806910B3FFE740F6FB
:1083F000F041C4F20241086840F080600860FEF776
:1084000025F90590FFE740F6F040C4F2024000680D
:10841000000100280CD4FFE7FEF718F90599401A6F
:10842000032804D3FFE703208DF81F00A6E2EAE744
:1084300021E040F6F041C4F20241086820F080607B
:108440000860FEF703F90590FFE740F6F040C4F23C
:1084500002400068000100280CD5FFE7FEF7F6F89F
:108460000599401A032804D3FFE703208DF81F0065
:1084700084E2EAE7FFE7FFE7069800784007002874
:1084800040F1CC80FFE740F62400C4F202400068CF
:10849000C00708BBFFE740F62401C4F202410868A8
:1084A00040F001000860FEF7D1F80590FFE740F6C4
:1084B0002400C4F202400068C00760B9FFE7FEF77D
:1084C000C5F80599401A032804D3FFE703208DF867
:1084D0001F0053E2EBE7FFE7FFE7069880680128FB
:1084E00009D1FFE740F6F041C4F20241086840F0CC
:1084F0000100086054E00698806888B9FFE740F6FC
:10850000F041C4F20241086820F0010008600868E8
:1085100020F080000860086820F0040008603EE059
:1085200006988068052811D1FFE740F6F041C4F2B3
:108530000241086840F004000860086820F08000EC
:108540000860086840F00100086027E0069880682D
:10855000852811D1FFE740F6F041C4F202410868D6
:1085600040F004000860086840F080000860086877
:1085700040F00100086010E040F6F041C4F2024112
:10858000086820F001000860086820F00400086016
:10859000086820F080000860FFE7FFE7FFE7FFE7DB
:1085A000FFE706988068E0B1FFE7FEF74FF8059017
:1085B000FFE740F6F040C4F2024000688007002860
:1085C0000ED4FFE7FEF742F80599401A41F28931CF
:1085D000884204D3FFE703208DF81F00CEE1E8E7CF
:1085E0001BE0FEF733F80590FFE740F6F040C4F2D9
:1085F00002400068800700280ED5FFE7FEF726F846
:108600000599401A41F28931884204D3FFE70320DB
:108610008DF81F00B2E1E8E7FFE7FFE70698007872
:108620008006002849D5FFE70698406A10B3FFE7A7
:1086300040F60041C4F20241086840F480500860EE
:10864000FEF704F80590FFE740F60040C4F2024050
:108650000068800400280CD4FFE7FDF7F7FF0599B8
:10866000401A032804D3FFE703208DF81F0085E19B
:10867000EAE721E040F60041C4F20241086820F434
:1086800080500860FDF7E2FF0590FFE740F60040EC
:10869000C4F202400068800400280CD5FFE7FDF713
:1086A000D5FF0599401A032804D3FFE703208DF86E
:1086B0001F0063E1EAE7FFE7FFE70698806A00280A
:1086C00000F05881FFE70498182800F0D580FFE7F4
:1086D0000698806A022840F0A180FFE740F600413A
:1086E000C4F20241086820F080700860FDF7AEFF18
:1086F0000590FFE740F60040C4F2024000688001A8
:1087000000280CD5FFE7FDF7A1FF0599401A0328C3
:1087100004D3FFE703208DF81F002FE1EAE7FFE70E
:1087200040F62841C4F20241086843F603729043C0
:10873000069BDA6A1B6B42EA032210430860069923
:10874000486BD1F838C0CB6B0A6C01386FF35F20EF
:108750004FF60061CFF6FF7101EB4C2189B208445E
:108760000021CFF6FF7101EB034101F4FE01084443
:108770004FF07F4101EB026101F0FE41084440F6F9
:108780003441C4F202410860FFE740F62841C4F2D8
:1087900002410091086820F0100008600698C06C43
:1087A000C00040F63842C4F202421060086840F04F
:1087B00010000860086820F00C00069A526C104304
:1087C0000860086820F02000069A926C1043086048
:1087D000086840F48030086040F60041C4F202416D
:1087E000086840F080700860FDF730FF0590FFE7F3
:1087F00040F60040C4F202400068800100280CD41A
:10880000FFE7FDF723FF0599401A032804D3FFE78C
:1088100003208DF81F00B1E0EAE72CE040F60041AC
:10882000C4F20241086820F080700860FDF70EFF76
:108830000590FFE740F60040C4F202400068800166
:1088400000280CD5FFE7FDF701FF0599401A032822
:1088500004D3FFE703208DF81F008FE0EAE740F61E
:108860002841C4F2024108684FF6FC72CFF6F87254
:1088700010400860FFE77CE040F62840C4F2024068
:108880000068029040F63440C4F202400068019053
:108890000698806A012837D0FFE7029800F00300AD
:1088A0000699C96A88422FD1FFE7029800F47C51EB
:1088B0000698006BB0EB112F26D1FFE701986FF3FC
:1088C0005F200699496B013988421DD1FFE7BDF849
:1088D00004100698806B0138B0EB512F14D1FFE7DC
:1088E000019800F4FE010698C06B0138B0EB114FFF
:1088F0000AD1FFE7019800F0FE410698006C0138AC
:10890000B0EB116F04D0FFE701208DF81F0035E0B8
:1089100040F63840C4F20240006881B20698C06C4C
:10892000B0EBD10F24D0FFE740F62841C4F202415A
:10893000086820F010000860FDF788FE0590FFE74A
:10894000FDF784FE0599401A08B9FFE7F8E7069895
:10895000C06CC00040F63841C4F20241086040F6E5
:108960002841C4F20241086840F010000860FFE7A7
:10897000FFE7FFE700208DF81F00FFE79DF81F00CD
:1089800008B080BD82B0019001980090042843D8BF
:108990000099DFE801F00C1D2F4103004EF2100199
:1089A000CEF20001086840F00400086035E04EF2A5
:1089B0001001CEF20001086820F00400086040F6C3
:1089C000E441C4F20241086820F00C00086024E091
:1089D0004EF21001CEF20001086820F00400086099
:1089E00040F6E441C4F202410868012262F38300C8
:1089F000086012E04EF21001CEF20001086820F08B
:108A00000400086040F6E441C4F202410868022212
:108A100062F38300086000E0FFE702B070470000E7
:108A200082B0009000980138B0F1807F03D3FFE757
:108A30000120019016E0009801384EF21401CEF2A8
:108A4000000108604EF21801CEF20001002008601B
:108A50004EF21002CEF20002116841F003011160E3
:108A60000190FFE7019802B07047000083B04EF21A
:108A70001000CEF2000000684007002803D5FFE791
:108A80000420029020E040F6E440C4F20240006876
:108A900000F00C0001900198009040B1FFE70098B1
:108AA000042807D0FFE70098082806D008E0002037
:108AB000029008E00120029005E00220029002E00E
:108AC00000200290FFE7FFE7029803B07047000024
:108AD00081B0009001B0704781B0009001B0704744
:108AE00081B0009001B0704784B0029001910020E5
:108AF0000090FFE7029890F83C00012804D1FFE7BE
:108B000002208DF80F0095E00299012081F83C00C9
:108B1000FFE7FFE7009820F0FF000199C9680843CC
:108B20000090009820F440700199896808430090F3
:108B3000009820F4806001994968084300900098EB
:108B400020F400600199096808430090009820F41F
:108B500080500199096908430090009820F4005062
:108B60000199496908430090009820F480400199D8
:108B7000096B08430090009820F4702001998969DE
:108B800040EA01400090009820F080500199C969A6
:108B9000084300900298006842F60041C4F20101C7
:108BA00088421BD0FFE70298006842F60041C5F2F8
:108BB0000101884212D0FFE70298006843F20041A9
:108BC000C4F20101884209D0FFE70298006843F22D
:108BD0000041C5F2010188421ED1FFE7009820F450
:108BE00070000199896A40EA01500090009820F0D5
:108BF00080700199096A08430090009820F0007085
:108C00000199496A08430090009820F000500199AA
:108C1000C96A08430090FFE7009802990968486410
:108C2000FFE70299002081F83C00FFE700208DF863
:108C30000F00FFE79DF80F0004B0704781B000906F
:108C400001B0704781B0009001B0704781B00090D2
:108C500001B0704785B003900291FFE7039890F848
:108C60003C00012804D1FFE702208DF81300F6E054
:108C70000399012081F83C00FFE7FFE703990220F8
:108C800081F83D00039800684068019003980068EF
:108C9000806800900398006842F60041C4F2010128
:108CA00088421BD0FFE70398006842F60041C5F2F6
:108CB0000101884212D0FFE70398006843F20041A7
:108CC000C4F20101884209D0FFE70398006843F22B
:108CD0000041C5F2010188420AD1FFE7019820F462
:108CE0007000019002984168019808430190FFE7E5
:108CF00001984FF68F71CFF6FF510840019002980E
:108D00000168019808430190019803990968486037
:108D10000398006842F60041C4F20101884200F065
:108D20008280FFE70398006842F60041C5F2010126
:108D3000884278D0FFE703980068B0F1804F72D086
:108D4000FFE703980068B0F1A04F6CD0FFE70398ED
:108D5000006840F20041C4F20001884263D0FFE79E
:108D60000398006840F20041C5F2000188425AD0E1
:108D7000FFE70398006840F60001C4F20001884252
:108D800051D0FFE70398006840F60001C5F20001EA
:108D9000884248D0FFE70398006840F60041C4F2DB
:108DA000000188423FD0FFE70398006840F6004189
:108DB000C5F20001884236D0FFE70398006843F20D
:108DC0000041C4F2010188422DD0FFE703980068FA
:108DD00043F20041C5F20101884224D0FFE7039825
:108DE000006841F60001C4F2000188421BD0FFE791
:108DF0000398006841F60001C5F20001884212D0D4
:108E0000FFE70398006844F20001C4F201018842C0
:108E100009D0FFE70398006844F20001C5F20101A0
:108E200088420ED1FFE7009820F080000090029861
:108E30008168009808430090009803990968886049
:108E4000FFE70399012081F83D00FFE70399002027
:108E500081F83C00FFE700208DF81300FFE79DF844
:108E6000130005B07047000081B0009001B070475A
:108E700080B582B00090009820B9FFE701208DF8FE
:108E8000070045E0009890F83D0040B9FFE70099E1
:108E9000002081F83C00009800F03EF8FFE70099C0
:108EA000022081F83D00009951F8040B03F02AFBE1
:108EB0000099012081F84800FFE70099012081F81E
:108EC0003E00009981F83F00009981F84000009928
:108ED00081F84100009981F84200009981F843002F
:108EE000FFE7FFE70099012081F84400009981F82D
:108EF0004500009981F84600009981F84700FFE796
:108F00000099012081F83D0000208DF80700FFE75F
:108F10009DF8070002B080BD80B584B0039003982F
:108F2000006840F20041C4F20001884210D1FFE71E
:108F3000FFE740F69C40C4F20240016841F00201A4
:108F40000160006800F0020002900298FFE722E052
:108F50000398006840F60041C4F20001884219D12C
:108F6000FFE7FFE740F69C40C4F20240016841F091
:108F700008010160006800F0080001900198FFE717
:108F80003020009000221146FDF744FC0098FDF7C8
:108F900037FCFFE7FFE704B080BD000083B001901D
:108FA000019890F83D00012804D0FFE701208DF8DA
:108FB0000B00B2E00199022081F83D0001980068A1
:108FC00042F60041C4F20101884200F08280FFE7CE
:108FD0000198006842F60041C5F20101884278D04C
:108FE000FFE701980068B0F1804F72D0FFE7019869
:108FF0000068B0F1A04F6CD0FFE70198006840F224
:109000000041C4F20001884263D0FFE70198006884
:1090100040F20041C5F2000188425AD0FFE70198B2
:10902000006840F60001C4F20001884251D0FFE719
:109030000198006840F60001C5F20001884248D05E
:10904000FFE70198006840F60041C4F20001884241
:109050003FD0FFE70198006840F60041C5F20001EB
:10906000884236D0FFE70198006843F20041C4F21D
:10907000010188422DD0FFE70198006843F20041CA
:10908000C5F20101884224D0FFE70198006841F64B
:109090000001C4F2000188421BD0FFE7019800687C
:1090A00041F60001C5F20001884212D0FFE70198A5
:1090B000006844F20001C4F20101884209D0FFE7D0
:1090C0000198006844F20001C5F20101884219D1FB
:1090D000FFE70198006880680721C0F2010108409D
:1090E0000090009806280CD0FFE70098B0F5803F6C
:1090F00007D0FFE701980168086840F001000860A8
:10910000FFE706E001980168086840F00100086088
:10911000FFE700208DF80B00FFE79DF80B0003B080
:109120007047000083B00190019890F83D0001283D
:1091300004D0FFE701208DF80B00B8E00199022070
:1091400081F83D0001980168C86840F00100C860DE
:109150000198006842F60041C4F20101884200F023
:109160008280FFE70198006842F60041C5F20101E4
:10917000884278D0FFE701980068B0F1804F72D044
:10918000FFE701980068B0F1A04F6CD0FFE70198AD
:10919000006840F20041C4F20001884263D0FFE75A
:1091A0000198006840F20041C5F2000188425AD09F
:1091B000FFE70198006840F60001C4F20001884210
:1091C00051D0FFE70198006840F60001C5F20001A8
:1091D000884248D0FFE70198006840F60041C4F299
:1091E000000188423FD0FFE70198006840F6004147
:1091F000C5F20001884236D0FFE70198006843F2CB
:109200000041C4F2010188422DD0FFE701980068B7
:1092100043F20041C5F20101884224D0FFE70198E2
:10922000006841F60001C4F2000188421BD0FFE74C
:109230000198006841F60001C5F20001884212D091
:10924000FFE70198006844F20001C4F2010188427E
:1092500009D0FFE70198006844F20001C5F201015E
:10926000884219D1FFE70198006880680721C0F2A1
:10927000010108400090009806280CD0FFE70098F4
:10928000B0F5803F07D0FFE701980168086840F01B
:1092900001000860FFE706E001980168086840F0F7
:1092A00001000860FFE700208DF80B00FFE79DF844
:1092B0000B0003B07047000081B00090FFE70098FA
:1092C0000068006A41F21111084210D1FFE70098CE
:1092D0000068006A44F24441084207D1FFE7009861
:1092E0000168086820F001000860FFE7FFE7FFE77A
:1092F0000099012081F83D00002001B07047000076
:1093000080B586B00490039100208DF80B00FFE734
:10931000049890F83C00012804D1FFE702208DF862
:109320001700EDE00499012081F83C00FFE7FFE71A
:109330000499022081F83D0004980068806801903B
:1093400001984FF68871CFF6CE71084001900198D0
:1093500020F47F400190019804990968886003987F
:1093600000680090002800F0B180FFE70098102806
:1093700000F0AC80FFE70098202800F0A780FFE70E
:109380000098302800F0A280FFE70098402800F005
:109390009080FFE70098502871D0FFE70098602880
:1093A0007AD0FFE70098702845D0FFE70098B0F525
:1093B000805F3FD0FFE70098B0F5005F50D0FFE737
:1093C0000098B0F5801F00F08180FFE70098B0F1B1
:1093D000101F7BD0FFE700982021C0F210018842C7
:1093E00074D0FFE700983021C0F2100188426DD0A0
:1093F000FFE700984021C0F21001884266D0FFE7E5
:1094000000985021C0F2100188425FD0FFE7009819
:109410006021C0F21001884258D0FFE70098702107
:10942000C0F21001884251D0FFE70098B0F5001F4C
:109430004CD052E055E004980068039B5A68996844
:10944000DB6803F0C1F90498006880680190019816
:1094500040F077000190019804990968886040E025
:1094600004980068039B5A689968DB6803F0ACF9BC
:1094700004980168886840F48040886031E004986E
:109480000068039A5168D26803F0B4FD049800683C
:10949000502103F0B3F924E004980068039A51685E
:1094A000D26803F0ABFE04980068602103F0A6F9CF
:1094B00017E004980068039A5168D26803F09AFD97
:1094C00004980068402103F099F90AE004980068C4
:1094D0000399096803F092F903E001208DF80B006D
:1094E000FFE70499012081F83D00FFE7049900207F
:1094F00081F83C00FFE79DF80B008DF81700FFE7AF
:109500009DF8170006B080BD80B58AB00990099813
:109510000068B0F1804F36D1FFE70998007F04283A
:1095200031D1FFE740F29840C2F200000890006895
:10953000069009980821059101F0FEF80599034667
:10954000069844F6206200FB023040F29C42C2F2D0
:10955000000207921268801A40F29042C2F20002A2
:109560005060099801F0E8F8079A089950600020C7
:10957000086040F26741C2F20001D1F809000130F1
:10958000C1F80900FFE709980068B0F1804F36D1B3
:10959000FFE70998007F082831D1FFE740F29840A3
:1095A000C2F2000004900068029009980C21019119
:1095B00001F0C2F801990346029844F6206200FBCC
:1095C000023040F29C42C2F2000203925268801ABA
:1095D00040F29042C2F200021060099801F0ACF82B
:1095E000039A049910600020086040F24141C2F2E1
:1095F0000001D1F809000130C1F80900FFE70AB005
:1096000080BD000080B586B00490039102920020D6
:109610008DF80700FFE7049890F83C00012804D17A
:10962000FFE702208DF8170080E00499012081F8FF
:109630003C00FFE7FFE70298B0B9FFE70498006835
:10964000039B19685A68DB6803F0FCFC0498016806
:10965000886920F00C00886103988268049801688A
:1096600088691043886156E00298042817D1FFE703
:1096700004980068039B19685A68DB6803F0E8FDEA
:1096800004980168886920F44060886103988268C2
:1096900004980168886940EA022088613AE00298EB
:1096A000082816D1FFE704980068039B19685A68D8
:1096B000DB6803F003FE04980168C86920F00C0021
:1096C000C8610398826804980168C8691043C8613A
:1096D0001FE002980C2817D1FFE704980068039B4D
:1096E00019685A68DB6803F01FFE04980168C869AE
:1096F00020F44060C8610398826804980168C869D2
:1097000040EA0220C86103E001208DF80700FFE76E
:10971000FFE7FFE7FFE7FFE70499002081F83C003F
:10972000FFE79DF807008DF81700FFE79DF8170089
:1097300006B080BD80B582B00090009820B9FFE7E8
:1097400001208DF8070045E0009890F83D0040B9F1
:10975000FFE70099002081F83C00009800F03EF8F7
:10976000FFE70099022081F83D00009951F8040BB1
:1097700002F0C8FE0099012081F84800FFE7009937
:10978000012081F83E00009981F83F00009981F89E
:109790004000009981F84100009981F84200009949
:1097A00081F84300FFE7FFE70099012081F84400BA
:1097B000009981F84500009981F84600009981F8E8
:1097C0004700FFE70099012081F83D0000208DF857
:1097D0000700FFE79DF8070002B080BD81B0009050
:1097E00001B0704780B596B01490139100208DF8A9
:1097F0004B00139828B9FFE7149890F83E000F909B
:1098000034E01398042805D1FFE7149890F83F003E
:109810000E9028E01398082805D1FFE7149890F8D7
:1098200040000D901CE013980C2805D1FFE7149818
:1098300090F841000C9010E01398102805D1FFE734
:10984000149890F842000B9004E0149890F84300AC
:109850000B90FFE70B980C90FFE70C980D90FFE73B
:109860000D980E90FFE70E980F90FFE70F988DF878
:109870004300139828B9FFE7149890F844000A9021
:109880001CE01398042805D1FFE7149890F84500D0
:10989000099010E01398082805D1FFE7149890F874
:1098A0004600089004E0149890F847000890FFE7FD
:1098B00008980990FFE709980A90FFE70A988DF841
:1098C00042009DF84300012805D1FFE79DF84200C2
:1098D000012804D0FFE701208DF8570052E11398CA
:1098E00028B9FFE71499022081F83E0038E0139868
:1098F000042806D1FFE71499022081F83F00079061
:109900002CE01398082806D1FFE71499022081F86B
:10991000400006901FE013980C2806D1FFE7149929
:10992000022081F84100059012E01398102806D11A
:10993000FFE71499022081F84200049005E0149991
:10994000022081F843000490FFE704980590FFE7A8
:1099500005980690FFE706980790FFE70798FFE74E
:10996000139828B9FFE71499022081F844001EE0FB
:109970001398042806D1FFE71499022081F84500C6
:10998000039012E01398082806D1FFE714990220EB
:1099900081F84600029005E01499022081F8470002
:1099A0000290FFE702980390FFE70398FFE7139800
:1099B00001900C2825D80199DFE801F00723232323
:1099C0000E232323152323231C0014980168C86841
:1099D00040F00200C86018E014980168C86840F0C0
:1099E0000400C86011E014980168C86840F00800DD
:1099F000C8600AE014980168C86840F01000C860A8
:109A000003E001208DF84B00FFE79DF84B00002894
:109A100040F0B380FFE7149800681399012202F028
:109A2000B7FE1498006842F60041C4F20101884272
:109A300000F08280FFE71498006842F60041C5F20A
:109A40000101884278D0FFE714980068B0F1804F98
:109A500072D0FFE714980068B0F1A04F6CD0FFE718
:109A60001498006840F20041C4F20001884263D0BB
:109A7000FFE71498006840F20041C5F200018842F7
:109A80005AD0FFE71498006840F60001C4F20001C4
:109A9000884251D0FFE71498006840F60001C5F2F3
:109AA0000001884248D0FFE71498006840F6004162
:109AB000C4F2000188423FD0FFE71498006840F6E6
:109AC0000041C5F20001884236D0FFE714980068D3
:109AD00043F20041C4F2010188422DD0FFE71498FF
:109AE000006843F20041C5F20101884224D0FFE73B
:109AF0001498006841F60001C4F2000188421BD0AE
:109B0000FFE71498006841F60001C5F200018842A1
:109B100012D0FFE71498006844F20001C4F201017A
:109B2000884209D0FFE71498006844F20001C5F2AA
:109B30000101884219D1FFE7149800688068072165
:109B4000C0F2010108401190119806280CD0FFE7DF
:109B50001198B0F5803F07D0FFE7149801680868B6
:109B600040F001000860FFE706E01498016808680B
:109B700040F001000860FFE7FFE79DF84B008DF81B
:109B80005700FFE79DF8570016B080BD80B584B040
:109B9000039003980068C068029003980068006909
:109BA00001909DF804008007002824D5FFE79DF868
:109BB0000800800700281DD5FFE7039801686FF0B3
:109BC0000200086103990120087703980068806902
:109BD000800720B1FFE70398FFF796FC06E00398A3
:109BE00000F0D8F9039800F09DFBFFE703990020EF
:109BF0000877FFE7FFE79DF804004007002825D518
:109C0000FFE79DF80800400700281ED5FFE70398EE
:109C100001686FF004000861039902200877039837
:109C20000068806910F4407F04D0FFE70398FFF7D5
:109C30006BFC06E0039800F0ADF9039800F072FBAE
:109C4000FFE7039900200877FFE7FFE79DF804008E
:109C50000007002824D5FFE79DF80800000700282A
:109C60001DD5FFE7039801686FF0080008610399AC
:109C70000420087703980068C069800720B1FFE7D7
:109C80000398FFF741FC06E0039800F083F903987E
:109C900000F048FBFFE7039900200877FFE7FFE7A4
:109CA0009DF80400C006002825D5FFE79DF80800B0
:109CB000C00600281ED5FFE7039801686FF010006A
:109CC000086103990820087703980068C06910F4B8
:109CD000407F04D0FFE70398FFF716FC06E00398E7
:109CE00000F058F9039800F01DFBFFE703990020EE
:109CF0000877FFE7FFE79DF80400C00778B1FFE7AA
:109D00009DF80800C00748B1FFE7039801686FF0AD
:109D100001000861039800F09BFCFFE7FFE7019852
:109D200000F08000802806D0FFE79DF8050080063F
:109D3000002810D5FFE79DF808000006002809D587
:109D4000FFE7039801686FF4025008610398FEF77B
:109D5000C3FEFFE7FFE79DF80500C00780B1FFE7FE
:109D60009DF808000006002809D5FFE70398016860
:109D70006FF4807008610398FEF7AAFEFFE7FFE723
:109D80009DF804004006002810D5FFE79DF8080064
:109D90004006002809D5FFE7039801686FF04000EE
:109DA0000861039800F0F4FCFFE7FFE79DF804006A
:109DB0008006002810D5FFE79DF8080080060028DF
:109DC00009D5FFE7039801686FF020000861039848
:109DD000FEF786FEFFE7FFE79DF80600C0060028B5
:109DE00010D5FFE79DF80A00C006002809D5FFE757
:109DF000039801686FF4801008610398FEF722FF52
:109E0000FFE7FFE79DF806008006002810D5FFE772
:109E10009DF80A008006002809D5FFE7039801682D
:109E20006FF4001008610398FEF708FFFFE7FFE7F3
:109E30009DF806004006002810D5FFE79DF80A00AF
:109E40004006002809D5FFE7039801686FF48000F9
:109E500008610398FEF7FAFEFFE7FFE79DF80600AA
:109E60000006002810D5FFE79DF80A00000600282C
:109E700009D5FFE7039801686FF4000008610398B3
:109E8000FEF7F2FFFFE7FFE704B080BD80B58AB0C0
:109E9000099000200890079006900590049009987A
:109EA000006842F60041C4F20101884220D1FFE778
:109EB000FFE740F68C40C4F20240016841F0010126
:109EC0000160006800F0010003900398FFE74FF481
:109ED0004070049002200590002006900790012019
:109EE00008900020C4F2022004A9FCF70BFA4FE00E
:109EF00009980068B0F1804F1FD1FFE7FFE740F6F7
:109F00008C40C4F20240016841F001010160006828
:109F100000F0010002900298FFE703200490022065
:109F20000590002006900790012008900020C4F2C0
:109F3000022004A9FCF7E6F929E00998006841F637
:109F40000001C4F20001884220D1FFE7FFE740F69C
:109F50008C40C4F20240016841F0020101600068D7
:109F600000F0020001900198FFE74FF44040049098
:109F700002200590002106910791089040F20040D0
:109F8000C4F2022004A9FCF7BDF9FFE7FFE7FFE7F1
:109F90000AB080BD81B0009001B0704780B586B036
:109FA00004900391029200208DF80700FFE70498C7
:109FB00090F83C00012804D1FFE702208DF817003B
:109FC000C0E00499012081F83C00FFE7FFE7029818
:109FD0000090142800F2A7800099DFE801F00BA49C
:109FE000A4A424A4A4A43EA4A4A457A4A4A471A497
:109FF000A4A48A0004980068039902F017FC04984E
:10A000000168886940F008008861049801688869DF
:10A0100020F0040088610398026904980168886947
:10A020001043886183E004980068039902F0B8FC4B
:10A0300004980168886940F40060886104980168A8
:10A04000886920F480608861039802690498016837
:10A05000886940EA0220886169E0049800680399F1
:10A0600002F060FD04980168C86940F00800C8610A
:10A0700004980168C86920F00400C8610398026967
:10A0800004980168C8691043C86150E004980068EA
:10A09000039902F009FE04980168C86940F4006061
:10A0A000C86104980168C86920F48060C861039899
:10A0B000026904980168C86940EA0220C86136E074
:10A0C00004980068039902F0B1FE04980168086DD5
:10A0D00040F00800086504980168086D20F004004D
:10A0E00008650398026904980168086D10430865C3
:10A0F0001DE004980068039902F00AFF04980168C3
:10A10000086D40F40060086504980168086D20F44B
:10A11000806008650398026904980168086D40EA48
:10A120000220086503E001208DF80700FFE7FFE744
:10A130000499002081F83C00FFE79DF807008DF8A6
:10A140001700FFE79DF8170006B080BD80B582B00C
:10A150000090009820B9FFE701208DF8070045E046
:10A16000009890F83D0040B9FFE70099002081F881
:10A170003C00009800F03EF8FFE70099022081F8CB
:10A180003D00009951F8040B02F0BCF90099012040
:10A1900081F84800FFE70099012081F83E0000990E
:10A1A00081F83F00009981F84000009981F8410052
:10A1B000009981F84200009981F84300FFE7FFE72A
:10A1C0000099012081F84400009981F84500009928
:10A1D00081F84600009981F84700FFE700990120C7
:10A1E00081F83D0000208DF80700FFE79DF807008B
:10A1F00002B080BD80B58EB00D9000200C900B9009
:10A200000A90099008900D98006842F60041C4F247
:10A210000101884210D1FFE7FFE740F6A440C4F2F5
:10A220000240016841F400610160006800F40060D0
:10A2300007900798FFE772E00D980068B0F1804F33
:10A2400038D1FFE7FFE740F69C40C4F202400168C6
:10A2500041F001010160006800F0010006900698DD
:10A26000FFE7FFE740F68C40C4F20240016841F08E
:10A2700001010160006800F0010005900598FFE70A
:10A280000C200890022009900A90002001900B9069
:10A2900001200C900020C4F2022008A9FCF732F83B
:10A2A000019A2D2002901146FCF7B4FA0298FCF7AF
:10A2B000A7FA33E00D98006840F60001C4F20001EF
:10A2C000884210D1FFE7FFE740F69C40C4F202400D
:10A2D000016841F004010160006800F0040004908E
:10A2E0000498FFE719E00D98006841F60001C4F2F8
:10A2F0000001884210D1FFE7FFE740F69C40C4F21E
:10A300000240016841F040010160006800F0400037
:10A3100003900398FFE7FFE7FFE7FFE7FFE70EB0D3
:10A3200080BD000081B0009001B0704780B590B052
:10A330000E900D910D9828B9FFE70E9890F83E0009
:10A340000B9034E00D98042805D1FFE70E9890F8A3
:10A350003F000A9028E00D98082805D1FFE70E98E5
:10A3600090F8400009901CE00D980C2805D1FFE7FB
:10A370000E9890F84100089010E00D98102805D133
:10A38000FFE70E9890F84200079004E00E9890F8CE
:10A3900043000790FFE707980890FFE708980990A7
:10A3A000FFE709980A90FFE70A980B90FFE70B98E0
:10A3B000012804D0FFE701208DF83F0044E10D980B
:10A3C00028B9FFE70E99022081F83E0038E00D9889
:10A3D000042806D1FFE70E99022081F83F0006907D
:10A3E0002CE00D98082806D1FFE70E99022081F88D
:10A3F000400005901FE00D980C2806D1FFE70E994C
:10A40000022081F84100049012E00D98102806D136
:10A41000FFE70E99022081F84200039005E00E99B3
:10A42000022081F843000390FFE703980490FFE7C0
:10A4300004980590FFE705980690FFE70698FFE768
:10A440000E9800680D990122019202F0A1F901987D
:10A450000E99096842F60042C4F20102914202904C
:10A4600038D0FFE70E980168012042F60042C5F29D
:10A470000102914202902DD0FFE70E980168012061
:10A4800043F20042C4F201029142029022D0FFE75F
:10A490000E980168012043F20042C5F20102914288
:10A4A000029017D0FFE70E980168012044F20002E5
:10A4B000C4F20102914202900CD0FFE70E980068AE
:10A4C0004CF20001CAF6FE710844B0FA80F040096F
:10A4D0000290FFE70298C00738B1FFE70E980168C5
:10A4E000486C40F400404864FFE70E98006842F66C
:10A4F0000041C4F20101884200F08280FFE70E981B
:10A50000006842F60041C5F20101884278D0FFE7B9
:10A510000E980068B0F1804F72D0FFE70E98006887
:10A52000B0F1A04F6CD0FFE70E98006840F20041F8
:10A53000C4F20001884263D0FFE70E98006840F241
:10A540000041C5F2000188425AD0FFE70E9800682A
:10A5500040F60001C4F20001884251D0FFE70E9896
:10A56000006840F60001C5F20001884248D0FFE7CC
:10A570000E98006840F60041C4F2000188423FD0C6
:10A58000FFE70E98006840F60041C5F200018842DE
:10A5900036D0FFE70E98006843F20041C4F2010193
:10A5A00088422DD0FFE70E98006843F20041C5F2C3
:10A5B0000101884224D0FFE70E98006841F60001AF
:10A5C000C4F2000188421BD0FFE70E98006841F6F4
:10A5D0000001C5F20001884212D0FFE70E98006822
:10A5E00044F20001C4F20101884209D0FFE70E984D
:10A5F000006844F20001C5F20101884219D1FFE769
:10A600000E98006880680721C0F2010108400C9094
:10A610000C9806280CD0FFE70C98B0F5803F07D0C7
:10A62000FFE70E980168086840F001000860FFE746
:10A6300006E00E980168086840F001000860FFE736
:10A6400000208DF83F00FFE79DF83F0010B080BD6F
:10A6500081B0009000980068B0F1804F08D1FFE70A
:10A6600040F29841C2F20001086801300860FFE73B
:10A670000098006840F60041C4F20001884259D1B8
:10A68000FFE740F2AF11C2F200010120087040F272
:10A690006C10C2F2000001780131017000784007AF
:10A6A00038B9FFE740F2AC11C2F200010120087096
:10A6B000FFE740F26C10C2F20000007849F68851C2
:10A6C000C0F6D81144F6C562CCF2EC4200FB021091
:10A6D0004FEA7000884207D8FFE740F2AE11C2F29D
:10A6E000000101200870FFE740F26C10C2F2000088
:10A6F000007849F69012C1F699124CF6CD41CCF68D
:10A70000CC4100FB01204FEA301043F23231C0F25D
:10A71000333188420DD8FFE740F2AD11C2F200019B
:10A720000120087040F26C11C2F200010020087094
:10A73000FFE7FFE701B0704784B00390029100206B
:10A740000190029800900C281DD80099DFE801F0D4
:10A75000071B1B1B0C1B1B1B111B1B1B1600039831
:10A760000068406B01900FE003980068806B0190D7
:10A770000AE003980068C06B019005E00398006848
:10A78000006C019000E0FFE7019804B07047000002
:10A7900081B0009001B07047FFE7FEE782B0019002
:10A7A00000208DF80300FFE79DF80300022818DC65
:10A7B000FFE79DF803000199C97D884201D1FFE7B9
:10A7C00009E001989DF8031050F821100020C4F210
:10A7D000E020C861FFE79DF8030001308DF8030019
:10A7E000E2E702B07047000081B0009000988068F6
:10A7F0004FF6C071C7F6FF710840023000998860BB
:10A8000001B0704781B00090009988684FF6C0721F
:10A81000C5F6FF721040886001B0704781B00090AB
:10A82000009880684FF6C071C7F6FF71084001308C
:10A830000099886001B0704781B0009048F2C8016B
:10A84000C4F20221086840F00100086001B07047BE
:10A8500081B000900099D1F8C80040F00100C1F823
:10A86000C80001B07047000081B000900098806877
:10A8700040F080504FF6C071C7F6FF710840009954
:10A88000886001B07047000081B000900098806837
:10A8900000F0E07001B0704781B0009000988068CF
:10A8A00000F4604001B0704781B00090009880686B
:10A8B00000F01F0001B0704783B002900191029830
:10A8C000019900EB8100603000900098006800F072
:10A8D000F84003B07047000081B000900098806895
:10A8E000C0F3C00001B0704781B000900098C06C08
:10A8F00000F4C070B0FA80F0400901B07047000069
:10A9000081B00090009880684FF6C071C7F6FF7163
:10A91000084020300099886001B0704781B00090F5
:10A9200000988068C00F01B07047000081B00090AF
:10A9300000988068C0F3407001B0704781B000900B
:10A9400000988068C0F3400001B0704781B000906B
:10A950000098806800F0010001B0704781B000905D
:10A9600000988068C0F3007001B0704781B000901B
:10A9700000988068C0F3800001B0704781B00090FB
:10A980000098C06800F44060B0FA80F0400901B05F
:10A990007047000084B003900291019203980299DD
:10A9A00001F4407100EB9110303000900098006885
:10A9B000029901F01F021F21914088430199C1F3C0
:10A9C0008461914008430099086004B0704700001A
:10A9D00081B00090009880684FF6C071C7F6FF7193
:10A9E000084004300099886001B0704781B0009041
:10A9F000009880684FF6C071C7F6FF7108401030AC
:10AA00000099886001B0704784B003900291019270
:10AA10000398029901F0007100EBD15014300090BE
:10AA2000009800680299C1F30452072191408843BD
:10AA30000199914008430099086004B070470000F4
:10AA400083B00290019100920298D0F8B000019971
:10AA50006FF31F518843009A02F018034FF6FF72FC
:10AA6000C0F20F02DA40114008440299C1F8B00068
:10AA700003B0704782B0019000910198806820F483
:10AA80007C10009908430199886002B0704700006B
:10AA900082B0019000910198806820F0E0700099E8
:10AAA00008430199886002B07047000085B00490A7
:10AAB0000391029201930498039900EB81006030A6
:10AAC0000090009800684FF20001C0F2FF31014091
:10AAD000029800F0F840019A1043084340F000400B
:10AAE0000099086005B0704784B00390029101920C
:10AAF0000398029900EB8100603000900098006894
:10AB000020F00070019908430099086004B0704774
:10AB100084B00390029101920398029900EB8100A6
:10AB2000603000900098006820F080700199084320
:10AB30000099086004B0704784B0039002910192BC
:10AB40000398029900EB8100603000900098006843
:10AB500020F00040019908430099086004B0704754
:10AB600082B0019000910198406920F00040009966
:10AB700008430199486102B07047000082B001901B
:10AB80000091019880684FF6C071C3F6FF710140D3
:10AB9000009800F08040084400F10040019988606E
:10ABA00002B0704780B58AB000208DF81B00F7F71F
:10ABB00085FD059040F24400C2F200000068036881
:10ABC00044F20000C0F6010009A904229847099840
:10ABD00046F26661C3F23331884240F08080FFE77D
:10ABE00040F24400C2F200000068036844F2000032
:10ABF000C0F602000DF11B01012298479DF81B00D1
:10AC0000032805DCFFE79DF81B000599C875FFE7E1
:10AC100000208DF81B00FFE79DF81B00022838DCA0
:10AC2000FFE705989DF81B1050F8210004909DF84F
:10AC30001B000599C97D884204D1FFE704990020D3
:10AC4000086220E040F24400C2F20000006803689D
:10AC50009DF81B1048F20000C0F6010040EA811088
:10AC600008A9042298470898013058B1FFE70898CE
:10AC700040B1FFE7089805999DF81B2051F8221074
:10AC8000C860FFE7FFE79DF81B0001308DF81B004F
:10AC9000C2E740F24400C2F200000190006803687D
:10ACA00046F20000C0F60100039007A904220292B8
:10ACB00098470199029A0398079BDDF814C0CCF8D5
:10ACC000183009680B6808A998470898013028B916
:10ACD000FFE705994FF07E508861FFE7FFE70AB074
:10ACE00080BD000080B58AB00021009109910891D3
:10ACF00007910691059104910391029140F2A440BD
:10AD0000C2F20000019048F20002C4F20222026086
:10AD10004FF4002242608160C16001220261082379
:10AD20004361027641760523C36180F820104FF419
:10AD3000946383624FF48063C36280F834200163BC
:10AD40004FF48052826380F83C10F8F71DFE18B172
:10AD5000FFE7F7F753F9FFE70820C0F690400290AD
:10AD600006200390072004907F2005900420069081
:10AD70000020079040F2A440C2F2000002A9F7F7B9
:10AD8000D7FE18B1FFE7F7F739F9FFE78020C1F6E2
:10AD9000505002900C20039040F2A440C2F20000F8
:10ADA00002A9F7F7C5FE18B1FFE7F7F727F9FFE7A4
:10ADB0000020C4F6843002901220039040F2A44098
:10ADC000C2F2000002A9F7F7B3FE18B1FFE7F7F7E8
:10ADD00015F9FFE70020C4F6B87002901820039020
:10ADE00040F2A440C2F2000002A9F7F7A1FE18B198
:10ADF000FFE7F7F703F9FFE70020CCF2527002906B
:10AE00004FF48070039040F2A440C2F2000002A907
:10AE1000F7F78EFE18B1FFE7F7F7F0F8FFE70AB093
:10AE200080BD000080B582B040F28450C2F20000C4
:10AE300001904AF20041C4F200010160002141602A
:10AE40008160C16001744174012282744261826137
:10AE50004FF0150CC0F81CC00323036242628262EB
:10AE6000C0F82CC0036342638263C163FAF772FDCA
:10AE700018B1FFE7F7F7C2F8FFE702B080BD0000A6
:10AE800080B582B040F2E850C2F2000001904AF66C
:10AE90000001C4F200010160002141608160C160D5
:10AEA0000174417401228274426182614FF0150C79
:10AEB000C0F81CC00323036242628262C0F82CC047
:10AEC000036342638263C163FAF744FD18B1FFE78D
:10AED000F7F794F8FFE702B080BD000080B582B0BC
:10AEE000FFE740F68840C4F20240016841F00101EA
:10AEF0000160006800F0010001900198FFE71B204D
:10AF0000009000221146FBF785FC0098FBF778FCC7
:10AF100002B080BD80B590B000200F900E900D90D3
:10AF20000C900B90FFE740F68C40C4F202400168A1
:10AF300041F080010160006800F080000A900A98EA
:10AF4000FFE7FFE740F68C40C4F20240016841F0A1
:10AF500001010160006800F0010009900998FFE715
:10AF6000FFE740F68C40C4F20240016841F0020164
:10AF70000160006800F0020008900898FFE740F2C6
:10AF80000040C4F20220069040F2064100910022E7
:10AF90000592FBF745FB059A0020C4F202200290BF
:10AFA0004FF480610191FBF73BFB0698A8210391C8
:10AFB00001220492FBF734FB009B049A0599069842
:10AFC0000B930C920D910E910BA90791FBF79AF937
:10AFD000DDF804C00298049B059A0799CDF82CC0AF
:10AFE0000C930D930E92FBF78DF90298059A079931
:10AFF0004FF400430B930C920D92FBF783F9DDF8AD
:10B000000CC0049B059A06980799CDF82CC00C93A8
:10B010000D9202220E92FBF775F9059A0698079990
:10B0200050230B930C920D92FBF76CF910B080BD7E
:10B0300080B5FBF711FB18B1FFE7F6F7DFFFFFE77D
:10B0400080BD000080B588B0002100910791069175
:10B050000591049103910291019140F29860C2F22E
:10B06000000041F60002C4F200020260F9224260D0
:10B07000816044F61F62C260016180218161FFF737
:10B0800065F818B1FFE7F6F7B9FFFFE76020019018
:10B090004FF47A70029000220392059240F2986079
:10B0A000C2F2000001A9FEF779FF18B1FFE7F6F739
:10B0B000A5FFFFE740F29860C2F2000001A9042258
:10B0C000FEF76CFF18B1FFE7F6F798FFFFE740F2D5
:10B0D0009860C2F20000FEF7D9FE08B080BD000003
:10B0E00080B59AB000200190199018901790169092
:10B0F00015901490139012901190109003A8342181
:10B10000F5F797F9019940F24C60C2F20000029005
:10B1100042F60042C4F201020260F92242608160FC
:10B1200044F61F62C2600161416180218161FFF7C5
:10B130000DF818B1FFE7F6F761FFFFE70020179061
:10B140001890199040F24C60C2F2000017A9FDF768
:10B1500081FD18B1FFE7F6F751FFFFE7602010907F
:10B160004FF47A7011900022129213921492159259
:10B17000169240F24C60C2F2000010A9FEF70EFFDA
:10B1800018B1FFE7F6F73AFFFFE740F24C60C2F272
:10B19000000010A90422FEF701FF18B1FFE7F6F73F
:10B1A0002DFFFFE70020009003900490059006908B
:10B1B00007904FF40051089109900A900B904FF0BE
:10B1C00000710C910D900E900F9040F24C60C2F205
:10B1D000000003A9FDF788FC18B1FFE7F6F70EFFA2
:10B1E000FFE740F24C60C2F20000FEF74FFE1AB0DB
:10B1F00080BD000080B590B0002101910F910E91AB
:10B200000D910C910B910A9109910891079106916A
:10B21000059104910391029140F2E460C2F20000B2
:10B220004FF080420260F9224260816044F61F6262
:10B23000C260016180218161FEF788FF18B1FFE7DC
:10B24000F6F7DCFEFFE740F2E460C2F20000FEF732
:10B2500071FA18B1FFE7F6F7D1FEFFE700200D9075
:10B260000F9040F2E460C2F200000DA9FDF7F2FC7D
:10B2700018B1FFE7F6F7C2FEFFE7602006904FF433
:10B280007A700790002208920A9240F2E460C2F2BB
:10B29000000006A9FEF782FE18B1FFE7F6F7AEFE42
:10B2A000FFE740F2E460C2F2000006A90422FEF7C4
:10B2B00075FE18B1FFE7F6F7A1FEFFE70020029048
:10B2C000012103910490059040F2E460C2F2000075
:10B2D00002A90822FEF796F918B1FFE7F6F78EFEED
:10B2E000FFE740F2E460C2F2000002A90C22FEF780
:10B2F00089F918B1FFE7F6F781FEFFE740F2E46055
:10B30000C2F20000FEF7C2FD10B080BD80B588B06B
:10B3100000210091079106910591049103910291FA
:10B32000019140F23070C2F2000040F20042C4F2DB
:10B3300000020260F922426081604FF6FF72C26033
:10B34000016180218161FDF793FD18B1FFE7F6F7F8
:10B3500055FEFFE74FF48050049040F23070C2F287
:10B36000000004A9FDF7CCFF18B1FFE7F6F746FE91
:10B37000FFE700200190039040F23070C2F200001D
:10B3800001A9FDF767FC18B1FFE7F6F737FEFFE705
:10B3900008B080BD80B58CB0002101910B910A915D
:10B3A00009910891079106910591049103910291E9
:10B3B00040F27C70C2F2000040F60002C4F20002CB
:10B3C0000260F922426081604CF25032C260016139
:10B3D00080218161FEF7BAFE18B1FFE7F6F70EFE95
:10B3E000FFE7002009900B9040F27C70C2F2000051
:10B3F00009A9FDF72FFC18B1FFE7F6F7FFFDFFE7FE
:10B400006020029040F6C410039000200490069043
:10B4100040F27C70C2F2000002A90C22FEF7BEFDD1
:10B4200018B1FFE7F6F7EAFDFFE70CB080BD0000BA
:10B4300080B588B000210091079106910591049193
:10B4400003910291019140F2C870C2F2000040F6EF
:10B450000042C4F200020260F9224260816043F2BD
:10B46000D302C26001618161FDF702FD18B1FFE7FF
:10B47000F6F7C4FDFFE74FF48050049040F2C87027
:10B48000C2F2000004A9FDF73BFF18B1FFE7F6F791
:10B49000B5FDFFE700200190039040F2C870C2F2B2
:10B4A000000001A9FDF7D6FB18B1FFE7F6F7A6FDEE
:10B4B000FFE708B080BD000080B58AB0002003908F
:10B4C00009900890079006900590049004900590CC
:10B4D00002210691012107910890099040F28450C1
:10B4E000C2F2000004A9F9F709FF18B1FFE7F6F767
:10B4F00085FDFFE74FF08040049000200590022179
:10B500000691012107910890099040F28450C2F2FF
:10B51000000004A9F9F7F2FE18B1FFE7F6F76EFD97
:10B52000FFE7684600230193036040F28450C2F2B3
:10B530000000029002221146F9F73CFF019A02989E
:10B540000121F9F787FD019A02984FF40021F9F7DC
:10B5500081FD019A02980421F9F77CFD0298FAF71F
:10B560001DFD0AB080BD000080B58AB000200390A8
:10B57000099008900790069005900490049005901B
:10B580000221069107910890099040F2E850C2F21A
:10B59000000004A9F9F7B2FE18B1FFE7F6F72EFD97
:10B5A000FFE74FF0804004900020059002210691B3
:10B5B00007910890099040F2E850C2F2000004A9F7
:10B5C000F9F79CFE18B1FFE7F6F718FDFFE76846AC
:10B5D00000230193036040F2E850C2F200000290A1
:10B5E00002221146F9F7E6FE019A02980821F9F7BE
:10B5F00031FD019A02984FF40021F9F72BFD019AD1
:10B6000002982021F9F726FD0298FAF7C7FC0AB044
:10B6100080BD000080B582B040F2A440C2F20000BC
:10B6200001907F21F7F700FA019840F27A21C2F2E7
:10B6300000010522F8F7EAFB40F27C70C2F200003C
:10B640000C21FEF773FE02B080BD000080B5FFF74D
:10B6500033FFFFF789FFF5F7EDFCF5F73DFB80BD04
:10B6600080B586B040F24C60C2F200000390002129
:10B670000191FEF75BFE039804210291FEF756FE4E
:10B68000019940F2E460C2F200000490FEF74EFE21
:10B6900002990498FEF74AFE019940F29860C2F2BE
:10B6A00000000590FEF742FE02990598FEF73EFE67
:10B6B0000498FDF737FD04980821FEF793F80498E5
:10B6C0000C21FEF78FF840F2C870C2F20000FDF7BF
:10B6D00029FD039B049A0599D3F800C04FF47A70B2
:10B6E000CCF834001B689863136858631268906341
:10B6F0000A685063096888630020C4F202204FF48E
:10B7000080610122FAF78CFF06B080BD80B582B05F
:10B71000F6F7D4FF01900198C069C068804700F037
:10B720002DFBE12000F0D0FD02B080BD85B002AA63
:10B7300000920246009804928DF80F1080ED000AE6
:10B7400000208DF80700FFE79DF807009DF80F1017
:10B7500088420EDAFFE7029804999DF8072001EB72
:10B7600082014860FFE79DF8070001308DF807006F
:10B77000EAE70098049A0021117690ED000A9DF8FE
:10B780000F0001EE100AB8EEC11A20EE010A04986B
:10B7900080ED070A02980499086204990120087054
:10B7A00005B07047FFE7FEE7FFE7FEE788B00790C8
:10B7B00006910592079800F0070004900498C0F1E4
:10B7C0000700052803D3FFE70420019004E0049854
:10B7D000C0F107000190FFE701980390049804303E
:10B7E000062803D8FFE70020009003E00498033800
:10B7F0000090FFE70098029006980399012202FA50
:10B8000001F101390840029B984005999A40013A9C
:10B810001140084308B0704781B0ADF80200BDF98F
:10B82000020040F29861C2F200010968886301B029
:10B830007047000081B0ADF80200BDF9020040F28F
:10B840009861C2F200010968486301B070470000C6
:10B8500080B590B0F6F732FF0E90002001900D9069
:10B860000C900B900A900990089007900690059014
:10B870008DF81300FFE79DF8130009286FDCFFE740
:10B8800000208DF81200FFE79DF8120002285FDC0F
:10B89000FFE7002003909DF812000E99C97D8842B1
:10B8A00001D1FFE74EE00E989DF8121050F82100EC
:10B8B00000F096FA0390FFE7039808BBFFE70E98A5
:10B8C0009DF8121050F8210000F08AFA03900598B4
:10B8D0000130059005980B2811D3FFE70E989DF8CD
:10B8E000121050F82110012081F82E009DF812004E
:10B8F0000E99C875002005908DF83F0058E0DBE7F1
:10B90000039B9DF812200AA951F82200184441F81F
:10B9100022009DF81300092810D1FFE79DF812209E
:10B920000AA850F822004CF6CD41CCF6CC41A0FB41
:10B930000110C00806A941F82200FFE70D20F9F721
:10B9400067FBFFE79DF8120001308DF812009BE7BE
:10B95000FFE79DF8130001308DF813008BE706A870
:10B96000F6F7C2FD00208DF80B00FFE79DF80B00F5
:10B97000022816DCFFE79DF80B000E99C97D88426E
:10B9800001D1FFE707E00E989DF80B1050F8211049
:10B990000869C860FFE79DF80B0001308DF80B00C7
:10B9A000E4E70E9800F02EFB01208DF83F00FFE742
:10B9B0009DF83F0010B080BD7047000080B586B094
:10B9C00000208DF8160040F21801C2F20001049127
:10B9D0000390029001908DF81700FFE79DF8170083
:10B9E000022857DCFFE79DF817000499C97D8842BB
:10B9F00001D1FFE748E040F26400C2F200000168B4
:10BA000004989DF8172050F8220088479DF81720C9
:10BA100001A941F82200FFE79DF8171001A850F88E
:10BA2000210080BBFFE740F26400C2F20000016821
:10BA300004989DF8172050F8220088479DF8172099
:10BA400001A941F822009DF8160001308DF816007A
:10BA50009DF816000B2815DBFFE70498C07D04282D
:10BA600010D1FFE704989DF8171050F8211001201D
:10BA700081F82E009DF817000499C87500208DF8F4
:10BA800016000DE0C8E7FFE79DF8170001308DF8BC
:10BA90001700A3E701A8F6F727FDF5F783FCFFE7FA
:10BAA00006B080BD80B584B0029040F60041C4F27B
:10BAB0000241086820F080600860FAF7C7FD019035
:10BAC000FFE740F60040C4F20240006800F0006169
:10BAD0000020B0EBD16F0CD0FFE7FAF7B7FD01996A
:10BAE000401A032804D3FFE703208DF80F008BE0F2
:10BAF000E7E7FFE740F62C41C4F20241086843F64D
:10BB000003729043029B1A685B6842EA0322104367
:10BB1000086002998868D1F80CC00B694A6901383D
:10BB20006FF35F204FF60061CFF6FF7101EB4C2100
:10BB300089B208440021CFF6FF7101EB034101F403
:10BB4000FE0108444FF07F4101EB026101F0FE412C
:10BB5000084440F63C41C4F202410860FFE740F669
:10BB60002C41C4F202410091086820F00C00029AB6
:10BB7000926910430860086820F02000029AD26998
:10BB8000104308600298426A086810430860086819
:10BB900020F01000086040F64042C4F202421068F3
:10BBA0004FF6F8739843029B1B6A40EAC30010608B
:10BBB000086840F01000086040F60041C4F20241FD
:10BBC000086840F080600860FAF740FD0190FFE7E8
:10BBD00040F60040C4F20240006800F0006100201E
:10BBE000B0EBD16F0CD1FFE7FAF730FD0199401AA5
:10BBF000032804D3FFE703208DF80F0004E0E7E7F4
:10BC000000208DF80F00FFE79DF80F0004B080BD05
:10BC100080B584B0029040F60041C4F20241086849
:10BC200020F080500860FAF711FD0190FFE740F620
:10BC30000040C4F20240006800F000510020B0EB68
:10BC4000517F0CD0FFE7FAF701FD0199401A032854
:10BC500004D3FFE703208DF80F008BE0E7E7FFE751
:10BC600040F63041C4F20241086843F60372904343
:10BC7000029B1A685B6842EA03221043086002993B
:10BC80008868D1F80CC00B694A6901386FF35F20EE
:10BC90004FF60061CFF6FF7101EB4C2189B20844E9
:10BCA0000021CFF6FF7101EB034101F4FE010844CE
:10BCB0004FF07F4101EB026101F0FE41084440F684
:10BCC0004441C4F202410860FFE740F63041C4F24B
:10BCD00002410091086820F00C00029A926910431A
:10BCE0000860086820F02000029AD26910430860BA
:10BCF0000298426A086810430860086820F0100043
:10BD0000086040F64842C4F2024210684FF6F873E9
:10BD10009843029B1B6A40EAC3001060086840F029
:10BD20001000086040F60041C4F20241086840F08B
:10BD300080500860FAF78AFC0190FFE740F6004067
:10BD4000C4F20240006800F000510020B0EB517FC7
:10BD50000CD1FFE7FAF77AFC0199401A032804D3C3
:10BD6000FFE703208DF80F0004E0E7E700208DF8DF
:10BD70000F00FFE79DF80F0004B080BD80B584B0D0
:10BD8000F6F79CFC03900398C06940688047C82080
:10BD900001F048FF00F092F8F6F7A8FDFEF702FF69
:10BDA00000208DF80B00FFE79DF80B00022815DC42
:10BDB000FFE79DF80B000399C97D884201D1FFE799
:10BDC00006E003989DF80B1050F821000190FFE762
:10BDD0009DF80B0001308DF80B00E5E704B080BD45
:10BDE00080B586B0049000220392049908680989FE
:10BDF000FAF716FCFAF72AFC0190FFE70499486865
:10BE00004989FAF7F5FB58B1FFE7FAF71FFC0199EA
:10BE1000401A652803D3FFE7002005904BE0EDE7CB
:10BE200000208DF80B00FFE79DF80B00172828DC99
:10BE3000FFE70499086809890122FAF7F1FB052058
:10BE4000009001F0EFFE0398400003900499086809
:10BE500009890022FAF7E4FB009801F0E3FE049957
:10BE600048684989FAF7C4FB20B1FFE7039801301D
:10BE70000390FFE7FFE79DF80B0001308DF80B0002
:10BE8000D2E70499086809890122FAF7C9FB0398E7
:10BE900080F40000039003984FF6C071C0F2FF01D8
:10BEA000084003900499086809890022FAF7B8FB52
:10BEB00003980590FFE7059806B080BD80B584B073
:10BEC000F6F7FCFB039000208DF80B00FFE79DF8D0
:10BED0000B00022842DCFFE79DF80B000399C97DA7
:10BEE000884201D1FFE733E003989DF80B1050F82A
:10BEF0002100019040F24400C2F200000068036893
:10BF00009DF80B104AF20000C0F6010000EB811012
:10BF100001992831042298470198806A0130B0B90C
:10BF2000FFE70199C868886240F24400C2F200004D
:10BF3000006843689DF80B104AF20000C0F601004B
:10BF400000EB81100199283104229847FFE7FFE7B1
:10BF50009DF80B0001308DF80B00B8E704B080BDF0
:10BF600080B582B000208DF80700FFE79DF807003C
:10BF70000B281CDCFFE740F24400C2F2000000681E
:10BF800082689DF8073042F20000C0F6010000EB25
:10BF9000433044F20001C0F6010101EB4331904708
:10BFA000FFE79DF8070001308DF80700DEE702B0DB
:10BFB00080BD000080B540F20040C4F202200221A2
:10BFC0000122FAF72DFB80BD81B0ADF80200BDF96A
:10BFD000020040F24C61C2F200010968886301B0BE
:10BFE0007047000081B0ADF80200BDF9020040F2D8
:10BFF0004C61C2F200010968486301B0704700005B
:10C000007047000080B584B00390002000908DF848
:10C010000B0001F0B3FA40F24400C2F200000068E5
:10C02000826848F20000C0F601004CF20001C0F640
:10C030000101904700988DF80B00FFE79DF80B0079
:10C04000022827DCFFE79DF80B000399C97D884291
:10C0500001D1FFE718E003989DF80B1050F821007C
:10C06000019040F24400C2F20000006843689DF86D
:10C070000B1048F20000C0F6010040EA811001995F
:10C080000C3104229847FFE79DF80B0001308DF832
:10C090000B00D3E704B080BD80B58AB009908DF85D
:10C0A0002310F6F70BFB079007989DF8231050F824
:10C0B00021000690002005900998D0F80100059015
:10C0C00001F05CFA09980078E22840F0B180FFE7BF
:10C0D0000598049001280ED0FFE70498032843D068
:10C0E000FFE70498042861D0FFE7049840F29A2102
:10C0F000884278D081E0069890ED050A9FED571AA6
:10C1000080EE010A80ED080A069890ED080A9FED7E
:10C11000541AB4EE410AF1EE10FA0BDAFFE7069872
:10C1200090ED080AB7EE001AB4EE410AF1EE10FAEB
:10C1300006DAFFE706990020C4F296200862FFE7BE
:10C140009DF823204AF20000C0F6010000EB4230C7
:10C150004CF20001C0F6010101EB4231069A203297
:10C16000042301F021FA62E09DF823000799C875C5
:10C1700040F24400C2F2000002900068826844F27B
:10C180000000C0F60200039046F20001C0F6020172
:10C19000904702990398069B002283F82E20096895
:10C1A0004B68079917310122984755E040F2440047
:10C1B000C2F2000000900068826844F20000C0F6FD
:10C1C0000200019046F20001C0F60201904700997A
:10C1D0000198079B0322DA7509684B6807991731A4
:10C1E0000122984723E09DF82300032804D1FFE7AC
:10C1F000FFF7B6FE01F078FA19E00998F6F70CFBA4
:10C20000069880ED080A9DF823204AF20000C0F647
:10C21000010000EB42304CF20001C0F6010101EBDD
:10C220004231069A2032042301F0BEF9FFE7FFE70E
:10C230009DF823204AF20000C0F6010000EB4230D6
:10C240004CF20001C0F6010101EB4231069A2032A6
:10C25000042301F0A9F9FFE70AB080BD00007A4489
:10C260000000204380B584B0029000208DF80700C4
:10C27000FFE79DF8070002281EDCFFE79DF8070096
:10C280000299C97D884201D1FFE70FE002989DF82D
:10C29000071050F82100406A01F0BAF9012804D1D2
:10C2A000FFE701208DF80F000AE0FFE79DF8070087
:10C2B00001308DF80700DCE700208DF80F00FFE764
:10C2C0009DF80F0004B080BD81B08DF803009DF88B
:10C2D000030040F27821C2F20001087001B07047FB
:10C2E00080B5FAF7C3F980BD80B59CB008A850218D
:10C2F000F4F79FF8002007900690059004900390B3
:10C300000290FFE740F61000C4F20240016841F0DD
:10C3100030010160006800F0300001900198FFE7F3
:10C32000FFE740F61400C4F20240006800F0080085
:10C33000082801D0FFE7F4E7012008904FF480308F
:10C340000990022012900321139114902821159135
:10C350001690179018900C20199000201A901B909E
:10C3600008A8FBF711FE18B1FFE7F5F747FEFFE756
:10C370001F20029003200390002004900590069057
:10C38000079002A80521FBF735FA18B1FFE7F5F78A
:10C3900035FEFFE742F20001C4F202010868022202
:10C3A00062F3051008601CB080BD000082B04EF63C
:10C3B0008851CEF20001086840F47000086040F631
:10C3C0000042C4F202420120106040F61C41C4F257
:10C3D000024100200090086040F62041C4F2024172
:10C3E000086011684EF6E323CEF6E223194011608F
:10C3F00040F62841C4F20241086040F62C41C4F2E4
:10C400000241086040F63041C4F20241086040F643
:10C410003443C4F2024340F28021C0F2011119609A
:10C4200040F63843C4F20243186040F63C43C4F27D
:10C430000243196040F64043C4F20243186040F6DC
:10C440004443C4F20243196040F64841C4F2024139
:10C450000860116821F48021116040F65041C4F257
:10C46000024108604EF60851CEF200014FF0006024
:10C47000086042F21800C4F20200006800F0604058
:10C4800001900198B0F1604F05D0FFE70198B0F13D
:10C49000404F24D1FFE742F21C00C4F202000068C2
:10C4A000C00778B1FFE742F20C01C4F2020142F684
:10C4B0003B20C0F61900086046F67F60C4F65D4078
:10C4C0000860FFE742F21C01C4F20201086840F074
:10C4D00002000860086840F001000860FFE702B051
:10C4E0007047000080B540F2E460C2F20000FDF742
:10C4F0004DFB80BD80B540F2C870C2F20000FDF770
:10C5000045FB80BD83B002900191029800680090C5
:10C51000029842F60041C4F20101884252D0FFE77E
:10C52000029842F60041C5F2010188424AD0FFE775
:10C530000298B0F1804F45D0FFE70298B0F1A04FCC
:10C5400040D0FFE7029840F20041C4F20001884267
:10C5500038D0FFE7029840F20041C5F2000188425E
:10C5600030D0FFE7029840F60001C4F20001884293
:10C5700028D0FFE7029840F60001C5F2000188428A
:10C5800020D0FFE7029840F60041C4F20001884243
:10C5900018D0FFE7029840F60041C5F2000188423A
:10C5A00010D0FFE7029843F20041C4F20101884233
:10C5B00008D0FFE7029843F20041C5F2010188422A
:10C5C0000AD1FFE7009820F07000009001984168C0
:10C5D000009808430090FFE7029842F60041C4F239
:10C5E0000101884272D0FFE7029842F60041C5F28D
:10C5F000010188426AD0FFE70298B0F1804F65D010
:10C60000FFE70298B0F1A04F60D0FFE7029840F238
:10C610000041C4F20001884258D0FFE7029840F27E
:10C620000041C5F20001884250D0FFE7029840F671
:10C630000001C4F20001884248D0FFE7029840F6AA
:10C640000001C5F20001884240D0FFE7029840F6A1
:10C650000041C4F20001884238D0FFE7029840F65A
:10C660000041C5F20001884230D0FFE7029843F252
:10C670000041C4F20101884228D0FFE7029843F24A
:10C680000041C5F20101884220D0FFE7029841F63F
:10C690000001C4F20001884218D0FFE7029841F679
:10C6A0000001C5F20001884210D0FFE7029844F271
:10C6B0000001C4F20101884208D0FFE7029844F269
:10C6C0000001C5F2010188420AD1FFE7009820F479
:10C6D000407000900198C168009808430090FFE7FF
:10C6E000009820F080000199496908430090009863
:10C6F00002990860019880680299C86201980068F0
:10C7000002998862029842F60041C4F2010188420F
:10C7100028D0FFE7029842F60041C5F201018842A5
:10C7200020D0FFE7029843F20041C4F201018842A1
:10C7300018D0FFE7029843F20041C5F20101884298
:10C7400010D0FFE7029844F20001C4F201018842D0
:10C7500008D0FFE7029844F20001C5F201018842C7
:10C7600005D1FFE70198006902990863FFE7029984
:10C770000120486102980069C00730B1FFE70299C3
:10C78000086920F001000861FFE703B0704700006E
:10C7900084B0039002910192029800F01F010120E1
:10C7A00088400090009A0399086A904308620198B3
:10C7B000029901F01F0100FA01F20399086A10437F
:10C7C000086204B07047000085B0049003910292A3
:10C7D0000193049880680090009820F47F400090B6
:10C7E00003980299019A41EA022101430098084303
:10C7F000009000980499886005B0704783B002905B
:10C80000019102988068009000984FF68F71CFF6E2
:10C81000CF710840009001980099084340F007004C
:10C82000009000980299886003B0704785B004902A
:10C8300003910498006A01900499086A20F00100AD
:10C8400008620498406800900498806902900298F9
:10C850004FF68F71CFF6FE7108400290029820F0DB
:10C86000030002900398016802980843029001981F
:10C8700020F002000190039881680198084301901C
:10C88000049842F60041C4F20101884228D0FFE733
:10C89000049842F60041C5F20101884220D0FFE72A
:10C8A000049843F20041C4F20101884218D0FFE726
:10C8B000049843F20041C5F20101884210D0FFE71D
:10C8C000049844F20001C4F20101884208D0FFE755
:10C8D000049844F20001C5F2010188420ED1FFE73D
:10C8E000019820F0080001900398C168019808435E
:10C8F0000190019820F004000190FFE7049842F6AF
:10C900000041C4F20101884228D0FFE7049842F6B2
:10C910000041C5F20101884220D0FFE7049843F2AC
:10C920000041C4F20101884218D0FFE7049843F2A5
:10C930000041C5F20101884210D0FFE7049844F29B
:10C940000001C4F20101884208D0FFE7049844F2D4
:10C950000001C5F20101884213D1FFE7009820F4DD
:10C9600080700090009820F4007000900398416956
:10C97000009808430090039881690098084300904C
:10C98000FFE7009804994860029804998861039829
:10C9900040680499486301980499086205B070479B
:10C9A00085B0049003910498006A01900499086A84
:10C9B00020F0100008620498406800900498806994
:10C9C0000290029848F6FF71CFF6FF61084002908E
:10C9D000029820F44070029003980168029840EA9F
:10C9E00001200290019820F02000019003988168B6
:10C9F000019840EA01100190049842F60041C4F207
:10CA0000010188422BD0FFE7049842F60041C5F2AD
:10CA10000101884223D0FFE7049843F20041C4F2A9
:10CA2000010188421BD0FFE7049843F20041C5F2A0
:10CA30000101884213D0FFE7049844F20001C4F2D8
:10CA40000101884208D0FFE7049844F20001C5F2D2
:10CA50000101884212D1FFE7012078B9FFE7019870
:10CA600020F0800001900398C168019840EA01100D
:10CA70000190019820F040000190FFE7049842F6F1
:10CA80000041C4F20101884228D0FFE7049842F631
:10CA90000041C5F20101884220D0FFE7049843F22B
:10CAA0000041C4F20101884218D0FFE7049843F224
:10CAB0000041C5F20101884210D0FFE7049844F21A
:10CAC0000001C4F20101884208D0FFE7049844F253
:10CAD0000001C5F20101884215D1FFE7009820F45A
:10CAE00080600090009820F40060009003984169F5
:10CAF000009840EA8100009003988169009840EA1C
:10CB000081000090FFE7009804994860029804991A
:10CB100088610398406804998863019804990862C1
:10CB200005B0704785B0049003910498006A0190A5
:10CB30000499086A20F480700862049840680090A4
:10CB40000498C069029002984FF68F71CFF6FE717B
:10CB500008400290029820F00300029003980168B8
:10CB6000029808430290019820F400700190039805
:10CB70008168019840EA01200190049842F6004142
:10CB8000C4F2010188422BD0FFE7049842F600412D
:10CB9000C5F20101884223D0FFE7049843F2004127
:10CBA000C4F2010188421BD0FFE7049843F2004120
:10CBB000C5F20101884213D0FFE7049844F2000156
:10CBC000C4F20101884208D0FFE7049844F2000152
:10CBD000C5F20101884212D1FFE7012078B9FFE7D1
:10CBE000019820F4006001900398C168019840EA20
:10CBF00001200190019820F480600190FFE70498E3
:10CC000042F60041C4F20101884228D0FFE70498AF
:10CC100042F60041C5F20101884220D0FFE70498A6
:10CC200043F20041C4F20101884218D0FFE70498A2
:10CC300043F20041C5F20101884210D0FFE7049899
:10CC400044F20001C4F20101884208D0FFE70498D1
:10CC500044F20001C5F20101884215D1FFE70098B6
:10CC600020F480500090009820F400500090039829
:10CC70004169009840EA011000900398816900988A
:10CC800040EA01100090FFE700980499486002987C
:10CC90000499C861039840680499C863019804998D
:10CCA000086205B07047000085B0049003910498B5
:10CCB000006A01900499086A20F480500862049880
:10CCC000406800900498C0690290029848F6FF718D
:10CCD000CFF6FF6108400290029820F44070029065
:10CCE00003980168029840EA01200290019820F41C
:10CCF0000050019003988168019840EA013001904A
:10CD0000049842F60041C4F2010188422BD0FFE7AB
:10CD1000049842F60041C5F20101884223D0FFE7A2
:10CD2000049843F20041C4F2010188421BD0FFE79E
:10CD3000049843F20041C5F20101884213D0FFE795
:10CD4000049844F20001C4F20101884208D0FFE7D0
:10CD5000049844F20001C5F20101884212D1FFE7B4
:10CD6000012078B9FFE7019820F400400190039872
:10CD7000C168019840EA01300190019820F4804098
:10CD80000190FFE7049842F60041C4F20101884295
:10CD900028D0FFE7049842F60041C5F2010188421D
:10CDA00020D0FFE7049843F20041C4F20101884219
:10CDB00018D0FFE7049843F20041C5F20101884210
:10CDC00010D0FFE7049844F20001C4F20101884248
:10CDD00008D0FFE7049844F20001C5F2010188423F
:10CDE00015D1FFE7009820F480400090009820F4CF
:10CDF0000040009003984169009840EA811000903B
:10CE000003988169009840EA81100090FFE700983C
:10CE10000499486002980499C8610398406804998D
:10CE2000086401980499086205B0704785B00490C1
:10CE300003910498006A01900499086A20F48030F4
:10CE400008620498406800900498006D029002986F
:10CE50004FF68F71CFF6FE7108400290039801687B
:10CE6000029808430290019820F400300190039842
:10CE70008168019840EA01400190049842F600411F
:10CE8000C4F20101884228D0FFE7049842F600412D
:10CE9000C5F20101884220D0FFE7049843F2004127
:10CEA000C4F20101884218D0FFE7049843F2004120
:10CEB000C5F20101884210D0FFE7049844F2000156
:10CEC000C4F20101884208D0FFE7049844F200014F
:10CED000C5F2010188420BD1FFE7009820F48030B1
:10CEE000009003984169009840EA01200090FFE714
:10CEF000009804994860029804990865039840686E
:10CF00000499886401980499086205B0704700008C
:10CF100085B0049003910498006A01900499086A0E
:10CF200020F4801008620498406800900498006D16
:10CF30000290029848F6FF71CFF6FF610840029018
:10CF400003980168029840EA01200290019820F4B9
:10CF50000010019003988168019840EA0150019007
:10CF6000049842F60041C4F20101884228D0FFE74C
:10CF7000049842F60041C5F20101884220D0FFE743
:10CF8000049843F20041C4F20101884218D0FFE73F
:10CF9000049843F20041C5F20101884210D0FFE736
:10CFA000049844F20001C4F20101884208D0FFE76E
:10CFB000049844F20001C5F2010188420BD1FFE759
:10CFC000009820F48020009003984169009840EA7E
:10CFD00081200090FFE70098049948600298049926
:10CFE0000865039840680499C86401980499086228
:10CFF00005B0704785B00490039102920498006ACE
:10D0000000900499086A20F0010008620498806981
:10D010000190019820F0F00001900299019840EAF7
:10D0200001100190009820F00A00009003990098E8
:10D030000843009001980499886100980499086257
:10D0400005B0704787B00690059104920393069847
:10D05000006A01900699086A20F0010008620698AB
:10D06000806902900699012042F60042C4F2010252
:10D070009142009000F09480FFE70699012042F66B
:10D080000042C5F201029142009000F08980FFE762
:10D0900006990120B1F1804F009000F08180FFE7F8
:10D0A00006990120B1F1A04F009079D0FFE70699D1
:10D0B000012040F20042C4F20002914200906FD081
:10D0C000FFE70699012040F20042C5F200029142BA
:10D0D000009065D0FFE70699012040F60002C4F2F7
:10D0E0000002914200905BD0FFE70699012040F6D4
:10D0F0000002C5F200029142009051D0FFE706996C
:10D10000012040F60042C4F200029142009047D054
:10D11000FFE70699012040F60042C5F20002914265
:10D1200000903DD0FFE70699012043F20042C4F28F
:10D1300001029142009033D0FFE70699012043F2AB
:10D140000042C5F201029142009029D0FFE7069902
:10D15000012041F60002C4F20002914200901FD06B
:10D16000FFE70699012041F60002C5F20002914254
:10D17000009015D0FFE70699012044F20002C4F2A6
:10D180000102914200900BD0FFE706984CF200019B
:10D19000CAF6FE710844B0FA80F040090090FFE73B
:10D1A0000098C00748B1FFE7029820F00300029002
:10D1B000049902980843029004E0029840F00100AC
:10D1C0000290FFE7029820F0F0000290039800011F
:10D1D000C1B2029808430290019820F00A00019021
:10D1E000059800F00A0101980843019002980699F9
:10D1F000886101980699086207B0704785B004906D
:10D20000039102920498006A00900499086A20F041
:10D2100010000862049880690190019820F4704021
:10D2200001900299019840EA01300190009820F0A5
:10D23000A00000900399009840EA01100090019826
:10D240000499886100980499086205B0704700004D
:10D2500086B005900491039202930598006A0090AD
:10D260000599086A20F0100008620598806901900D
:10D27000019820F4407001900399019840EA012040
:10D280000190019820F4704001900298000381B24F
:10D29000019808430190009820F0A00000900498A5
:10D2A00000F00A01009840EA0110009001980599E9
:10D2B000886100980599086206B0704786B00590AD
:10D2C0000491039202930598006A00900599086AF8
:10D2D00020F4807008620598C0690190019820F0E0
:10D2E000030001900399019808430190019820F0F0
:10D2F000F000019002980001C1B20198084301902A
:10D30000009820F420600090049800F00A01009832
:10D3100040EA0120009001980599C861009805999C
:10D32000086206B07047000086B005900491039231
:10D3300002930598006A00900599086A20F48050CD
:10D3400008620598C0690190019820F4407001902E
:10D350000399019840EA01200190019820F470405F
:10D3600001900298000381B201980843019000984F
:10D3700020F420400090049800F00A01009840EA50
:10D380000130009001980599C861009805990862DC
:10D3900006B0704780B5F5F783FAF3F77BFC80BDE4
:10D3A00080B582B001900198F3F7C0FF02B080BD54
:10D3B00080B582B001900198C0698068804702B052
:10D3C00080BD000080B582B0F5F778F90190F3F7E1
:10D3D0004BFE40F2AF10C2F200000078C00738B137
:10D3E000FFE740F2AF11C2F2000100200870FFE732
:10D3F00040F2AC10C2F200000078C00760B1FFE755
:10D400000198FFF7D5FFFFF7C5FF40F2AC11C2F25C
:10D41000000100200870FFE740F2AE10C2F20000E9
:10D420000078C007B8B1FFE700F08AFB40F2AE1108
:10D43000C2F2000100200870F5F7C4F840F2404045
:10D44000C2F200000078C00720B1FFE7E120FEF73C
:10D450003BFFFFE7FFE740F2AD10C2F200000078AB
:10D46000C00750B1FFE70198FFF79AFF40F2AD11F6
:10D47000C2F2000100200870FFE702B080BD00008A
:10D48000FFE7FEE780B582B0019000910098F3F7C6
:10D490000DFF0198C06900688047019880ED040A7B
:10D4A000019890ED030A9FED191AB4EE410AF1EECE
:10D4B00010FA25DDFFE700984078082820D0FFE724
:10D4C000019890ED040AB2EE041AB4EE410AF1EEAE
:10D4D00010FA05DDFFE700990198808A4880FFE790
:10D4E000019890ED030AB2EE041AB4EE410AF1EE8F
:10D4F00010FA04DAFFE7009900204880FFE7FFE711
:10D500000098F4F77FFD02B080BD00BFBD378635BF
:10D5100080B584B00390F5F7D1F800900398D0F867
:10D520000100029000980299F3F75EFA20B9FFE734
:10D530000098FDF733F9FFE700F020F800208DF8A0
:10D540000700FFE79DF80700022814DCFFE79DF8BD
:10D5500007000099C97D884201D1FFE705E00398E3
:10D560009DF80710FEF798FDFFE79DF807000130D2
:10D570008DF80700E6E704B080BD000080B582B0FA
:10D5800046F26660C3F23330019044F20000C0F608
:10D59000010046F20001C0F6010101AA042300F0D7
:10D5A00003F802B080BD000080B586B005900491FC
:10D5B00003928DF80B3040F24400C2F2000001905B
:10D5C000006882680598049990470198006843684C
:10D5D000059803999DF80B20984706B080BD000080
:10D5E00084B041EC100B8DED020B029A039941F0CF
:10D5F0000100002A08BF08460190019820F0004170
:10D600000020C7F6F070401AC00F04B07047000049
:10D6100081B000EE100A0090009820F00040C0F1A8
:10D62000FF40C00F01B0704781B0ADF80200BDF9F6
:10D63000020000280ED4FFE7BDF9021001F01F021E
:10D64000012090404A094EF20011CEF2000141F84B
:10D650002200FFE701B070474EF60C50CEF20000FA
:10D660000068C0F30220704782B0ADF80600009158
:10D67000BDF9060000280AD4FFE700980001BDF9B3
:10D6800006104EF20042CEF2000288540BE00098E1
:10D690000001BDF8061001F00F014EF61452CEF253
:10D6A00000028854FFE702B07047000083B0029088
:10D6B000029800F0070000904EF60C51CEF20001E7
:10D6C0000868019001984FF6FF0210400190019800
:10D6D000009A40EA02200022C0F2FA521043019060
:10D6E0000198086003B07047BFF34F8F4EF60C519E
:10D6F000CEF20001086800F4E0600422C0F2FA52A1
:10D7000010430860BFF34F8FFFE700BFFDE7000045
:10D7100080B58CB00B900A91099208930B988068A1
:10D72000013007900B98C06806900B9881680898A4
:10D73000084008900698012810D0FFE7069908983D
:10D7400000FB01F008900699079800FB01F0079094
:10D750000699099800FB01F00990FFE709980490E9
:10D7600007980899401A039004980399884203D2B5
:10D77000FFE70498019002E003980190FFE7019809
:10D780000290029805900B980069089908440A993C
:10D79000059AF2F7E7FD0B9800690A99059B194471
:10D7A000099AD21AF2F7DEFD0CB080BD80B58CB0BC
:10D7B0000B900A91099208930B98806801300790AA
:10D7C0000B98C06806900B988168089808400890EC
:10D7D0000698012810D0FFE70699089800FB01F091
:10D7E00008900699079800FB01F0079006990998A0
:10D7F00000FB01F00990FFE7099804900798089949
:10D80000401A039004980399884203D2FFE70498D2
:10D81000019002E003980190FFE7019802900298BE
:10D8200005900A980B990969089A1144059AF2F72C
:10D8300099FD0A98059B18440B990969099AD21A0F
:10D84000F2F790FD0CB080BD86B004900391029277
:10D850000498029908440121C0F60801884204D3C3
:10D86000FFE703208DF8170042E0029820B9FFE798
:10D8700000208DF817003BE001208DF80300002008
:10D880000190FFE701980299884224D2FFE70498AB
:10D8900000788DF802009DF802000399097888420B
:10D8A0000ED0FFE79DF80200FF2804D0FFE702201A
:10D8B0008DF817001CE000208DF80300FFE7FFE75C
:10D8C000049801300490039801300390FFE7019819
:10D8D00001300190D6E79DF80300012804D1FFE74D
:10D8E00000208DF8170003E001208DF81700FFE7F6
:10D8F0009DF8170006B0704780B58EB00B900A9166
:10D900000020099008900790029001200D900D983A
:10D9100080F31088F8F7CAFC0B9800F02DF80990F6
:10D920000A9800F029F8079007980999401A28B139
:10D93000FFE707980999401A009002E00120009043
:10D94000FFE70098089004200390012004900998B4
:10D9500005900898069003A802A9F8F763FB8DF8D4
:10D960000700F8F701FC00200C900C9880F3108859
:10D970009DF807000EB080BD82B00190002000909D
:10D98000019800F17840400B0090009802B0704779
:10D9900085B00390029101920398019908440121F6
:10D9A000C0F60801884204D3FFE701208DF8130078
:10D9B0001FE0019820B9FFE701208DF8130018E05F
:10D9C00000200090FFE70098019988420DD2FFE700
:10D9D0000398411C0391007802994A1C0292087036
:10D9E000FFE7009801300090EDE700208DF813006C
:10D9F000FFE79DF8130005B07047000080B594B0B4
:10DA00000F900E910D920F980D9908440021C0F6C9
:10DA10000801884206D8FFE70F990020B0EBD16FCC
:10DA200004D1FFE701208DF8430084E00D9820B970
:10DA3000FFE700208DF843007DE09DF83C000007E3
:10DA400020B1FFE701208DF8430074E00F980E9994
:10DA50000D9AFFF7F9FE8DF82F009DF82F0020B9E1
:10DA6000FFE700208DF8430065E001201390139834
:10DA700080F31088F8F71AFC00200C90FFE70C9850
:10DA80000D99B0EB111F22D2FFE700200A900990F8
:10DA9000089007900E9B186859689A68DB680A938B
:10DAA0000992089107900E9810300E900F9902205D
:10DAB00007AAF8F771FB20B9FFE70F9810300F9015
:10DAC00000E02DE0FFE70C9801300C90D7E79DF8BF
:10DAD00034000007B8B1FFE70020069005900490DD
:10DAE00003900E990D9800F00F0203A80190F2F731
:10DAF00039FC019A02920F990220F8F74DFB08B108
:10DB0000FFE70DE0FFE7F8F72FFB08B1FFE707E0BD
:10DB100000201290129981F310888DF843000AE0DA
:10DB2000F8F722FB00201190119880F31088012053
:10DB30008DF84300FFE79DF8430014B080BD00005E
:10DB400080B582B0F4F7BAFD019040F2E011C2F264
:10DB5000000141F22630C0F208000860002088620F
:10DB60004862ADF802000198006890ED060AB2EE36
:10DB7000041A80EE010ABDEEC00A10EE100AADF8DC
:10DB80000200BDF8020088840198406890ED060A02
:10DB900080EE010ABDEEC00A10EE100AADF80200D8
:10DBA000BDF80200C8840198806890ED060A80EEF6
:10DBB000010ABDEEC00A10EE100AADF80200BDF871
:10DBC0000200088540F2E850C2F2000000F002F8BE
:10DBD00002B080BD80B584B0029000208DF80700AF
:10DBE000FFE7029840F2E011C2F2000101F12402C5
:10DBF000F7F736FB70B1FFE79DF8070001308DF8AD
:10DC00000700C0B2142804DBFFE700208DF80F00E6
:10DC100004E0E6E701208DF80F00FFE79DF80F0014
:10DC200004B080BD80B584B0ADF80E0040F2307015
:10DC3000C2F200000290FBF7B1F9029801680020DF
:10DC40004862BDF80E00052805DBFFE7BDF80E00B1
:10DC50000238019002E001200190FFE70198ADF841
:10DC60000E00FFE7BDF80E0040F23071C2F2000175
:10DC70000968496A884201D9FFE7F3E740F230704A
:10DC8000C2F20000FBF718FB04B080BD83B0019026
:10DC900020200090019818B9FFE7002002903FE093
:10DCA000BDF8060038B9FFE701980004019000981C
:10DCB00010380090FFE79DF8070038B9FFE701989A
:10DCC00000020190009808380090FFE79DF80700D7
:10DCD00010F0F00F07D1FFE70198000101900098C4
:10DCE00004380090FFE79DF8070010F0C00F07D13F
:10DCF000FFE7019880000190009802380090FFE74C
:10DD00009DF807000006002807D4FFE701984000AF
:10DD10000190009801380090FFE700980290FFE71B
:10DD2000029803B07047000081B00090009802682C
:10DD300041688068891A0844013001B070470000CA
:10DD400080B582B000200190F8F79EFCFEF7CCFA77
:10DD5000FDF7E0F8FDF7C2F8FCF7C4FFFDF762F845
:10DD6000FDF78EF8FDF7BCF9FDF744FAFDF7CEFAA2
:10DD7000FDF710FBFDF75CFBFDF764F9FDF758F9C3
:10DD8000FDF748FCFDF762FCFDF76AFCFDF7BEFC01
:10DD9000FFE7FFF717FBFCE784B002AA00920246F8
:10DDA0000098039280ED000A8DF8071003990A7E0F
:10DDB00001EB820292ED011A91ED070A30EE410A61
:10DDC00081ED070A90ED001A039890ED070A30EEF6
:10DDD000010A80ED070A039890ED070A9DF80710E5
:10DDE00001EE101AB8EEC11A80EE010A80ED080AA1
:10DDF000029803990A7E01EB820148600399087E2C
:10DE00000130087603990B7E9DF80720B3FBF2F0F2
:10DE100000FB12300876039890ED080A04B07047B2
:10DE200080B584B00390029101920398FFF77CFFC4
:10DE3000009001980099884203D9FFE7009801906B
:10DE4000FFE703980299019A0368FFF761FC019AC2
:10DE50000399086810440860019804B080BD000070
:10DE600080B586B0049003910292019301990298C3
:10DE7000B0FBF1F00290029828B1FFE70298411E32
:10DE8000084205D0FFE7029800F052F80290FFE741
:10DE90000499002008600499486001980499C860BA
:10DEA0000398049908610298012807D8FFE70499AC
:10DEB000002088606FF01500059006E00298013898
:10DEC0000499886000200590FFE7059806B080BDA2
:10DED00080B584B003900291019203980299019A4F
:10DEE00000F00AF80190019A0399486810444860CC
:10DEF000019804B080BD000080B584B00390029109
:10DF00000192039908684968401A009001980099A5
:10DF1000884203D9FFE700980190FFE70398029930
:10DF2000019A4368FFF742FC019804B080BD0000ED
:10DF300080B582B00090009840B1FFE7009840B1F2
:10DF4000FFE70098411E084203D1FFE700980190C7
:10DF500007E00098FFF79AFE411E012088400190DB
:10DF6000FFE7019802B080BD81B040F61C00C2F20C
:10DF7000000001780131017000780F280ADBFFE70B
:10DF800040F61C01C2F200010F20087000208DF83D
:10DF9000030003E001208DF80300FFE79DF8030074
:10DFA00001B070470808A0F500114FEA3101704731
:10DFB00043004FEAD30C4FEA3C0C43401FBF4007DD
:10DFC0000CF1605113F0FE4F70471CF0006F03D14D
:10DFD0000CF00041002070470CF0004343EA507001
:10DFE00040EACC0010B500F00EF800BF000000922F
:10DFF0004FEA0001FFF7D6BF4FF00041A1F5002125
:10E000004FF0000070470EF1020E2EF0030E5EF886
:10E01000044B244204D44FEA4102B2F17F4F11D89D
:10E020004FEA4003B3F17F4F0CD80ED14FEAD07CBA
:10E030000CEB4C0C0CF1020CB2F17F4F08BF4CEB17
:10E04000D17C04E04FF0080C01E04FEAD17C0CEBEE
:10E050004C0324FA03F404F00704B4F1040C06D2D0
:10E060000EEB840CBDE810404CF0010C6047DFE87B
:10E070000CF0070802024FF00040A0F5800010BD30
:10E080000846420018BFD2F1807288BF00F00040FD
:10E0900010BDF1EE100A4FF6FF71C0F2C03120EA58
:10E0A000010040F04070E1EE100A704700000000EF
:10E0B0000000000001020304060708090001020332
:10E0C00004050607080C101418203040466562202D
:10E0D0003236203230323600F8E0000800000020EE
:10E0E00000010000B8020008F8E10008000100206B
:10E0F000200D0000D8020008040200200090D00388
:10E10000A129000815260008BDB900089D240008B3
:10E110006800002098000020C800002000000000D7
:10E1200000000000000000040000803F0800002004
:10E1300091D90008FDD90008F9D80008380000205E
:10E1400000000000000000000000000000000000CF
:10E15000010000000000000000000000E1BD000818
:10E16000000402420000024208000080000000009B
:10E170000000000000000000000000000000E0427D
:10E180000000E0420000000000000000000000006D
:10E1900000040242000402422000100000000000BF
:10E1A0000000000000000000000000000000E0424D
:10E1B0000000E0420000000000000000000000013C
:10E1C00000040242000402428000400000000000FF
:10E1D0000000000000000000000000000000E0421D
:10E1E0000000E0420000000000000000000000020B
:08E1F000010000001000000016
:040000050800025598
:00000001FF
